S00D00006473703234342E68313614
S12340000FF043B87FFE0000420042004200420042004200420042004200420042004234D9
S123402042004200420042004200983042004200421A4200420042004200420042004200BC
S123404042004200420042004200420042004200420042004200420042004200420042003C
S1234060420042004200420042004200420042009E9A420042004200420042004200420026
S123408042008BA84200420042004D7A420080C842009E0C42004200420042004200420018
S12340A08CE270BC42004200420042004200420042004200420042004200420042004200C6
S12340C04200420042004200420042004200420042004200420042004200420042004200BC
S12340E042004200420042004200420042004200420042004200420042004200420042009C
S123410042004200420042004200420042004200420042004200420042004200420042007B
S123412042004200420042004200420042004200420042004200420042004200420042005B
S123414042004200420042004200420042004200420042004200420042004200420042003B
S123416042004200420042004200420042004200420042004200420042004200420042001B
S12341804200420042004200420042004200420042004200420042004200420042004200FB
S12341A04200420042004200420042004200420042004200420042004200420042004200DB
S12341C04200420042004200420042004200420042004200420042004200420042004200BB
S12341E042004200420042004200420042004200420042004200420042004200420042009B
S1234200343F37AF379C27FA3FFE274FF501CA01C501B6F83F02357E2777343F37AF379CA7
S123422027FA3FFE274FF501CA01C501B6F83F02357E2777343F37AF379C27FA3FFE274FDF
S1234240F501CA01C501B6F83F02357E277737B540CF37FAFA0037B5660037FAFA041735A0
S1234260FA2137B52AEB37FAFA4437B5008037FAFA4637B5000537FAFA4837B56BB037FA36
S1234280FA4A37B5FF0337FAFA4C37B5783037FAFA4E37B5FB0137FAFA5037B578F037FA7C
S12342A0FA5237B5000537FAFA5437B5703037FAFA5637B5FA1037FAFA5837B5587037FAD3
S12342C0FA5A37B5FA1037FAFA5C37B54C7037FAFA5E37B5FA1037FAFA6037B5547037FA76
S12342E0FA6237B5FFFB37FAFA6837B5680137FAFA6A37B5FC0037FAFA7037B5DBF037FA90
S1234300FA72F57F17FAFA41F57B17FAF907F5FC17FAF906F51017FAFA171735FA11F5E197
S123432017FAFA15F52017FAFA1FF5FF17FAFA19F5DF17FAFA1D37B5000D37FAFC00F5509B
S123434017FAFC05F51C17FAFC04F57F17FAFC1617FAFC15F57E17FAFC1737B5820437FA32
S1234360FC1837B5040237FAFC1A37B58F0037FAFC1C1735FC1E37B5000F37FAFC0837B5A6
S1234380000C37FAFC0AF55017FAF926F58017FAF927F54017FAF92537B5208E37FAF90093
S12343A037B5024037FAF904F58017FAF9211735F9203901F91F27F7F50F27FA379C379D5C
S12343C0379E37B500FF37FAFB0437B5F00037FAFB061735FB00F50F379F37BFF3FEFA00D9
S12343E0424E37BC4000F500379CC501371F371F371F371F379FCF04F500379C379DF50FC7
S1234400379E37BCEE92CD003C02C500B716BA023C02C500379ECE019500AA003D023E0292
S12344204D03B5F03C05B0DEF50F379C27FA37BC049827F5B0008A003C02377C598CB5F25A
S1234440FA00A92EB0FA3424274F37DC277A379D3745000C8508CC0A379C2776B0068500F1
S12344609A003D023C027CFFB6F0351227F74556204478333800332E323000576564204D69
S1234480617220333120323030340030393A34363A343300000F0502000F04F4000F04E617
S12344A0340C274F27050000850037B80009B434F50F37BD0510379D850037350108372679
S12344C027FF37DD37DDB4FE3D018500373501083726277537B106183733000F9A02375AFB
S12344E0000027030000B0BCF50F27FA27350E5827350E5A37AC27FA3735000F37B50510F7
S12345002773050237B50E582773050637B5000A37FA050A2735050C2735050E273504F499
S1234520273504F6273504F8273504FA273504FC273504FE27350500273504E6273504E8C6
S1234540273504EA273504EC273504EE273504F0273504F2351827F734053FF8274F270554
S1234560000427050006F50037BD4494379DC50B370527F427F437DD3755000095028A0267
S1234580374A00008500CD02379D9508B7423440373B00E03755000095028A06374A0004DA
S12345A08504CD06379D37550000950234018500CD02379D35409A02375A000095082711D0
S12345C00008FCFFB606850027150004271500063501B010C50BB60C8500CD02379D271327
S12345E0000CB6002713000A374500048506CC083F0C27F734043FF8274F27050004270528
S12346000006F50027FA2771449437DC37AC27FA37DC8A02374A00008500CD02379D95080E
S123462037B80005B30827F5FA0045588A06374A0004374500048506CC083F0A27F734077E
S12346403FFC274FF50037BD4494379DC50F370527F427F437DD3755000095028A02374A86
S12346600000C511B6463440373B00E08500CD02379D37550000950234018506CD08379DEA
S123468035409A02375A0000374500068500CD02379D85089A02375A000095082713000831
S12346A027F6B60485089A06375A00043501B05A3440373B00E08500CD02379D9508271358
S12346C0000827F6B710374500069504DD06379D85089A02375A0000B00E37450006850099
S12346E0CD02379D85089A02375A0000374500068500CD02379D85089A06375A0004850662
S1234700CD08379D27150000271500023501CC043F0A27F734043FFA274FF50A27FA3801C5
S123472010041735100137AC27FA27F58A00FC068A02F50A27FAF58017FA1003C50317FA3A
S12347401000C502370517FA1001F50317FA100317F51002277A37AC27FA277ACA04F50AD3
S123476027FA17F51005277A37AC27FA277ACA04F50A27FA17F51000277A37AC27FA277A5D
S1234780CA04F50A27FA17F51004277A37AC27FA277ACA040505C505F820B414F50F37BD47
S12347A00498379DC505370527F437DD271500000305B0DECC063F0827F717F5317EF80292
S12347C0B64037F5019AB73A273504E4273504E2273504E0273504DE273504DC273504DAAD
S12347E0273504D8FA0044A0FA01B99A27350F7227350F74F50A27FAF50817FA100437AC70
S123480027FAFA00480827F717350F7A37B50B73340137B500FFFA00485A3F0237F50F7420
S123482037F70F72B71837B50001340127F5340127710F72FA00463E3F0427350F72273570
S12348400F74F50117FA0F7D277AF50A27FA277A17FA100137AC27FA27F73405274FF8FFF2
S1234860B61037F5F90A810837FAF9163810F9223910F920B0003810F920CC003F0427F773
S123488034053FFA274F05050501F801B60ECB400F02F5FFCA01C50F3705F61F8A02B01A09
S12348A03A400F7B0004F5FFCA0117F50F7B3705F61F373500203726C10F73008A02C501C8
S12348C0B70C8502B70237F8019CB62CF5FFCA05B026F50F37BD0498379D850227F427FF5A
S12348E037DD37DDB4FE3D0127130000850237F8019AB604F5FF17FA0F7ACA05C505B70475
S1234900FA01C63027330F60C5053705CC063F0A27F7340C274FF50A27FA17F51005277A02
S123492037AC27FA277ACA0117F50F7DF001B514F808B410FA02E800494E497A4A0C4AAE61
S12349404B544BEA4D604CEA37800410F50A27FA17F5100217F5100517F5100017F5100436
S123496037AC27FA37B50B73340137B500FFFA00485A3F02378003FC0A01000103F8F50A0C
S123498027FA17F51000277A37AC27FA277ACA0037B53941340137B500FFFA00485A3F0263
S12349A0C501F90EB64CCB80000CC50017FA0F7CF50317FA0F7DB012C500F804B52837053B
S12349C037FA0F6637FA0F64F50417FA0F7D37F50F6A17FD0F6C379DC50027330F6CB6009B
S12349E027330F6ADA003780038A273304E4FA0048083780037E273304E03801FA1939013A
S1234A00FA19FA0048083780036A0A0100010366F50A27FA17F51000277A37AC27FA277A1A
S1234A20CA0037B53941340137B500FFFA00485A3F02C501F90EB65CC500F980B70827330F
S1234A4004DEFA0048083780032A17F50F7C3705F67F373500803726C100730037FA0F66D7
S1234A6037FA0F6437B80100B308273304DCFA004808378002FEF50417FA0F7D37F50F6A6D
S1234A8017FD0F6C379DC50027330F6CB60027330F6ADA00378002DC273304E03801FA1993
S1234AA03901FA19FA004808378002C80A01000102C4F50A27FA17F51000277A37AC27FA27
S1234AC0277ACA0037B53941340137B500FFFA00485A3F02C501F90EB660CB80000CC50005
S1234AE017FA0F7BF50517FA0F7DB01A8B200040C5003705340137B50001FA0048803F02A5
S1234B0027F6B722F50617FA0F7D37F50F6A17FD0F6C379DC50027330F6CB60027330F6AD8
S1234B20DA0027310F663780024AFA00480837800242273304DAFA004808378002362733B7
S1234B4004E03801FA193901FA19FA004808378002220A010001021EF50A27FA17F5100047
S1234B60277A37AC27FA277ACA0037B53941340137B500FFFA00485A3F02C501F90EB650EB
S1234B80C500F980B708273304D8FA004808378001E2C5003705340137B50002FA00488014
S1234BA03F0227F6B722F50617FA0F7D37F50F6A17FD0F6C379DC50027330F6CB600273370
S1234BC00F6ADA0027310F66378001A8FA004808378001A0273304E03801FA193901FA19D8
S1234BE0FA0048083780018C0A0100010188F50A27FA17F51000277A37AC27FA277ACA0042
S1234C0037B53941340137B500FFFA00485A3F02C501F90E378600BA37F50F6A17FD0F6CB5
S1234C20379DC50027330F6CB60027330F6ADA0027310F663786013CF50A27FA173510015B
S1234C4037AC27FA37F50F6437B80004B70237B80005B63837B50001340127F53401277114
S1234C600F72FA00463E3F0427350F7227350F7417F50F7AB752F50717FA0F7D37B51315E7
S1234C80340137B500FFFA00485A3F02378000E437F50F6437B8007FB30627330F6427338B
S1234CA00F64B00027330F6437F50F7217FD0F74379D37F50F649A0437B500013401340154
S1234CC027710F72FA00463E3F04B098FA004808378000A0273304E03801FA193901FA1936
S1234CE0FA0048083780008C0A200001008837F50F68B63EF50A27FA1735100137AC27FA58
S1234D0037F50F7837F70F76B71037B50001340127F5340127710F76FA00463E3F04F50913
S1234D2017FA0F7D37B505B7340137B500FFFA00485A3F02B03C27710F6E27330F70B6009D
S1234D4027330F6E37DC277A379DF50A27FAD50017FA100037AC27FA27310F68B014F50A44
S1234D6027FA17F5100217F5100017F5100437AC27FAFA004808351827F7343F37AF379CCF
S1234D8027FA373B00A0373AFFBF3810F9223810F92017F50F7DF801B70AF807B70CF809D4
S1234DA0B70EFA004808B018FA004DC8B012FA004E34B00CF50A27FA3801100437AC27FA9E
S1234DC0FA004DC8357E277727F5FA00455827730F722776B6FE27F6B73427710F72FC062D
S1234DE03733000027730F6A27350F66F50217FA0F7DF50A27FA17F5100217F5100517F562
S1234E00100017F51004F50117FA100137AC27FAB01C17350F7D37B54C57340137B500FFEF
S1234E20FA00485A3F02F50A27FA1735100137AC27FA27F7F50A27FA3901100437AC27FA80
S1234E4027330F6237B50002FA00455827730F762776B6FE27F6B71C27710F76FC06373315
S1234E60000027730F6E37F50F7617FD0F78379D950437FA0F68B046FA01C2BE27730F7626
S1234E802776B6FE27F6B72427710F76FC063733000027730F6E37F50F7617FD0F78379D05
S1234EA0950437FA0F6827350F7627350F78B00E3735000F37B5534E27730F6E37FF534C37
S1234EC00F68F50817FA0F7DF50A27FAF50217FA100137AC27FA27F73716B60237F50F60C2
S1234EE0B00037F50F6227F70C00B6FE150D0040FE270D0100FE030D0119FE030D00E1FED9
S1234F0015084F3108CF33FE12084F31084F33FE3C084F3321E40B0EA0B10110D821F30094
S1234F202097000AE3800867F300000408443306C420085FF300000408443306C420085F4C
S1234F40B300000408E7B300000408E7B320001B576700000004084433077084000250087D
S1234F60443307708400025000000408F4A5FE0308F4A6FE030AB1910000620846330AB136
S1234F8091000065084F3321F7000AB3B300009E0AB3B40000A40AB3B50000930AB3B600DA
S1234FA0007B08CF2806C6000000790AB191000074084F330AAB8C00007708CF2A0C0062BD
S1234FC008F4ABFE0308F4AB8000B508CF2806C60000008A08F4A9FE030AAB8D0000840880
S1234FE04F2A08CF330AB191000088084F3308F4ABFE0308F4AB8001350C00A946F40000D8
S1235000020037000006C60000009C0AB191000095084E330AB191000098084433200043BB
S1235020075F8C0C00A906C6000000A20AB1910000A0085FB30C00A906C6000000A80AB16D
S1235040910000A6085FF3084E2408F4A5FE0308F4A6FE03084E21084E220000040AB191BD
S12350600000B50844330C00B100000408F4BD0403930AFA6600ACB808F4BF00200660F4E1
S1235080000002003802000565A03130003902000509A1322A003A02003C020008F4B703EF
S12350A00C0008F4AFC400A008F4AB84013508F4B6FE0308F4A8FE0308F4B000200108F44F
S12350C0B10032A908F4A5FE0308F4A6FE0308F4A40000A308F4A10008A30AA18F0000DC5A
S12350E0084E22084E230C00E0084E21084E22084E23000004FE513130003400000859A27C
S12351000859A308D9A508D9A651800000000B56F4007FFFFF0AB78000010E59E4005602F2
S12351200051000051810000000B0AB78100011559E4005603005101000AB7220AB7020057
S12351400004313500322A00341F000859A20859A308C1A557800056B000F0910B0A3F22E9
S12351600E31310A3F0245821B5700D84EF00000001E21C6E05602E021E40057F4007FFF36
S1235180FF21C66C21E5002000A256490044A02620004702904056200056B00044A6262063
S12351A0004702904056260056B50044A72620004702904056270057810056B100F0890B21
S12351C008D9A60A3F230E31530A3F0345831B5701D84EF00000001E21C6E05603E021E486
S12351E00057F4007FFFFF21C66C21E5002000A25661000A3F820001570AB7230A3F83003E
S1235200015A0AB7230A3FA200015F0A3FA300015F0AB70344A12620004702904056210035
S123522056B10044A82620004702904056280056B60044A92620004702904056290034018E
S12352400057B40020002A20002A0AF9460D02500AF9060001770AF9460A3F2408E2A80832
S1235260CF2A571000FE03085AA834210057B90020002A20002A0D02500AF9060001850ACE
S1235280F9460A3F2508E2AC08CF2E571100569000200010FE03085AAC0AABAF00018C083C
S12352A0E2AC08CE2EFE06085AAC08DCE90AAB8D000194084F2A08DCE90D01F321E4000A44
S12352C0F90600019E0AF9460A3F26313400FE03F499004EDCE0F081D23130002000D2F0F1
S12352E089002000D221C40056610044A226200047029040562200084F2A08DCE90D01F387
S123530021E4000AF9060001B50AF9460A3F27313400FE03F499004EDCE0F081D23130006B
S12353202000D2F089002000D221C40056370044A326200047029040562300084F2A08DC76
S1235340E90D01F321E4000AF9060001CC0AF9460A3F28313900FE03F489004EDCE0F08167
S1235360D23136002000D2F089002000D221C40056330044A426200047029040562400085C
S12353804F2A0D01F321E4000AF9060001E20AF9460A3F29313900FE03F489004EDCE0F001
S12353A081D23136002000D2F089002000D221C40056380044A5262000470290405625009C
S12353C0205800000004F18800F4800048D8002000C221E4C249D0E2F110E22000CAF08857
S12353E0CA2000DAF098DA4FDCDAF080DA48E01E4958F22000F21DDCD249C0D22000FAF495
S123540088FA2000EAF498EA4FDCEAF480EA48E01E4958C22000C219DCE249C0E22000CADC
S1235420F088CA2000DAF098DA4FDCDAF080DA48E01E4958F22000F21DDCD249C0D22000CA
S1235440FAF488FA2000EAF498EA4FDCEAF480EA48E01E4958C22000C219DCE249C0E22078
S123546000CAF088CA2000DAF098DA4FDCDAF080DA48E01E4958F22000F21DDCD249C0D2E0
S12354802000FAF488FA2000EAF498EA4FDCEAF480EA48E01E4958C22000C219DCE249C01A
S12354A0E22000CAF088CA2000DAF098DA4FDCDAF080DA48E01E4958F22000F21DDCD24930
S12354C0C0D22000FAF488FA2000EAF498EA2000EA2000EA20001E49580000000CF18800AE
S12354E0F4800048D8002000C221E4C249D0E2F110E22000CAF088CA2000DAF098DA4FDCDA
S1235500DAF080DA48E01E4958F22000F21DDCD249C0D22000FAF488FA2000EAF498EA4F73
S1235520DCEAF480EA48E01E4958C22000C219DCE249C0E22000CAF088CA2000DAF098DA6E
S12355404FDCDAF080DA48E01E4958F22000F21DDCD249C0D22000FAF488FA2000EAF49841
S1235560EA4FDCEAF480EA48E01E4958C22000C219DCE249C0E22000CAF088CA2000DAF067
S123558098DA2000DA2000DA20001E49580000000CFEF0FEF0FEF0FEF0FE9CFE60FE1EFEEC
S12355A00301555502AAAA0012C0FE03C00000200000FE03C00000FE03C00000200000FE90
S12355C003C00000FE03C00000200000FE03C00000FE03C00000200000FE03C00000FE03BF
S12355E0C00000200000FE03C00000FE0C7EB85210624E10624EFE03C00000200000FE0312
S1235600C00000FE03C00000200000FE03C00000FE03C00000200000FE03C00000FE03C0C1
S12356200000200000FE03C00000FE03C00000200000FE03C00000000001000001FE03C020
S12356400000200000FE03C00000FE03C00000200000FE03C00000FE03C00000200000FEE4
S123566003C00000FE03C00000200000FE03C00000FE03C00000200000FE03C00000FE031E
S1235680C00000200000FE03C00000FE03C00000200000FE03C00000FE03C00000200000E2
S12356A0FE03C00000FE037FFFFFFE0602AAACFE03C00000200000FE03C00000FE03C000E8
S12356C000200000FE03C00000FE03C00000200000FE03C00000FE03C00000200000FE0361
S12356E0C00000FE03C00000200000FE03C00000FE03C00000200000FE03C00000FE03C0E1
S12357000000200000FE03C00000FE03C00000200000FE03C00000FE037FFFFFFE0602AAD4
S1235720ACFE03C00000200000FE03C00000FE03C00000200000FE03C00000FE03C00000B4
S1235740200000FE03C00000FE03C00000200000FE03C00000FE03C00000200000FE03C020
S12357600000FE03C00000200000FE03C00000FE03C00000200000FE03C00000FE03C00020
S123578000200000FE03C00000FE037FFFFFFE09C00000200000FE03C00000FE03C000003D
S12357A0200000FE03C00000FE03C00000200000FE03C00000FE03C00000200000FE03C0C0
S12357C00000FE03C00000200000FE03C00000FE03C00000200000FE03C00000FE03C000C0
S12357E000200000FE03C00000FE03C00000200000FE03C00000FE037FFFFF0C00B6FE15CF
S12358000D0040FE270D00E6FE030D0123FE030D00E2FE15084F3108CF33FE12084F3108B8
S12358204F33FE3C084F3321E40B0EA0B10110D821F3002097000AE3800867F30000040820
S1235840443306C420085FF300000408443306C420085FB300000408E7B300000408E7B3B6
S123586020001B5767000000040844330770840001DF0844330770840001DF00000408F473
S1235880A5FE0308F4A6FE030AB1910000620846330AB191000065084F3321F7000AB3B3C9
S12358A000009E0AB3B40000A40AB3B50000930AB3B600007B08CF2806C6000000790AB13F
S12358C091000074084F330AAB8C00007708CF2A0C006208F4ABFE0308F4AB8000B508CFB3
S12358E02806C60000008A08F4A9FE030AAB8D000084084F2A08CF330AB191000088084F04
S12359003308F4ABFE0308F4AB8001350C00A946F40000020037000006C60000009C0AB100
S123592091000095084E330AB191000098084433200043075F8C0C00A906C6000000A20ACF
S1235940B1910000A0085FB30C00A906C6000000A80AB1910000A6085FF3084E2408F4A5B7
S1235960FE0308F4A6FE03084E21084E220000040AB1910000B50844330C00B10000040843
S1235980F4BD1D02070AFA6600ACB808F4BF0020063802003902000503A162F40000008089
S12359A03A1000057FA23B02003C0300235D000465A208F4B7030C0008F4AFC4005A08F4E5
S12359C0AB80013508F4B6FE0308F4A8FE0308F4B000200108F4B10032A908F4A5FE03080B
S12359E0F4A6FE0308F4A40000A308F4A10008A30AA18F0000DD084E22084E230C00E10880
S1235A004E21084E22084E23000004300A00313000044215340000205D00205D000859A2F7
S1235A200859A30A20C00000F456F400CCCCCC56590056510008D9A508D9A60D019CF2983B
S1235A400044D8450EA0FB0A26202000450EA0FE000A2621331B0034260021E500F09B004D
S1235A60F08BD0F09BD2F089D24EDCD244A2E22000325651262000470290405622000D018D
S1235A809CF2980044D8450EA1110A26242000450EA1140A2625331B0034510021E500F021
S1235AA09B00F08BD0F09BD2F089D24EDCD244A4E2200032566126200047029040562400AC
S1235AC00000043134003456000859A20859A30A20C000012D56F400555555565900565111
S1235AE00008D9A508D9A60D019CF2980044D8450EA1340A26222000450EA1370A262333FA
S1235B001B0034CA0021E500F09B00F08BD0F09BD2F089D24EDCD244A3E220003256512600
S1235B202000470290405623000D019CF2980044D8450EA14A0A26262000450EA14D0A263A
S1235B4027331B0034F50021E500F09B00F08BD0F093D2F089D24EDCD244A5E220003256B8
S1235B606126200047029040562500F68300200060545B0021863327805320CF760EA164F2
S1235B80200054218F0020003A21A4004FDC891EDC005FDCF321C7005EDCFB21E7005FDC82
S1235BA0F321C7002000FB21E7002000C820003A20CE002440002000450E217857F4007F79
S1235BC0FFFF20001957630034400044F00000001A4EDC1B59DC0060F0D00000052000024D
S1235BE0210E0056703200001A0504A056700000001BF09800F480D044F0E200001BF018D1
S1235C0000F080D2F818E2F480D2F818D2F080E2D818E22000D256580056700000001C601E
S1235C2070000000050460A7205A0000000457E10020003AF8983A19DC00F30A860E71A867
S1235C40205400B0900010DC00FC80006BDCDE0C01AEE0907C02204002F078134C0057E0F6
S1235C60006BDCDE574801F3930047D3450EF1BD060AA001DB15E0930057E31420003216F0
S1235C80DC4C21E6F620007421C5ED21E6492000EB56F000000006128D0302A0501C180005
S1235CA02000D1190A00F48000FD80F02000264EDC542000550290504EDC7502707012E459
S1235CC0030E71D747F4000000012000740E21D520EE0021C6000C01D721C61321C4004E8D
S1235CE05C0056F0AE0000071F100302A070108D002000D900000CFE63FE0FFE0FFE0300E7
S1235D0000AEFE037FFFFFFE030000AEFE037FFFFFFE030000AEFE037FFFFFFE030000AE4A
S1235D20FE037FFFFFFE18FE427FFFFF7FFFFF7FFFFF7FFFFF7FFFFF7FFFFF7FFFFF7FFFA2
S1235D40FF7FFFFF7FFFFF7FFFFF37837A4000007FFFFF7FFFFF7FFFFF7FFFFF7FFFFF7F65
S1235D60FFFF7FFFFF7FFFFF7FFFFF7FFFFF7FFFFF37837A4000007FFFFF7FFFFF7FFFFFC5
S1235D807FFFFF7FFFFF7FFFFF7FFFFF7FFFFF7FFFFF7FFFFF7FFFFF37837A4000007FFF25
S1235DA0FF7FFFFF7FFFFF7FFFFF7FFFFF7FFFFF7FFFFF7FFFFF7FFFFF7FFFFF7FFFFF37C7
S1235DC0837A40000000095F0000010000010006D100883F0000447FFFFF7FFFFF7FFFFFBF
S1235DE0FFF92F00095F0000017FFFFFFE4BFE0C40000000095F0000010000010006D100BE
S1235E00883F0000517FFFFF7FFFFF7FFFFFFFF92F00095F0000017FFFFFFE180B2D9D36C1
S1235E2019630173D633126F1029A89F3C5F74FDF483509C7F03B08059C57FDF3CFE12FE7D
S1235E400C40000000095F0000010000010006D100883F00005E7FFFFF7FFFFF7FFFFFFF16
S1235E60F92F00095F0000017FFFFFFEF0FE45FE0C40000000095F0000010000010006D154
S1235E8000883F00006B7FFFFF7FFFFF7FFFFFFFF92F00095F0000017FFFFFFE4BFE0C40B5
S1235EA0000005555500027BFFB36D0519A3D6A8886487ED0C00B6FE150D0040FE270D019F
S1235EC000FE030D0119FE030D00E1FE15084F3108CF33FE12084F31084F33FE3C084F331C
S1235EE021E40B0EA0B10110D821F3002097000AE3800867F300000408443306C420085FD8
S1235F00F300000408443306C420085FB300000408E7B300000408E7B320001B57670000BE
S1235F20000408443307708400022D08443307708400022D00000408F4A5FE0308F4A6FEC1
S1235F40030AB1910000620846330AB191000065084F3321F7000AB3B300009E0AB3B40039
S1235F6000A40AB3B50000930AB3B600007B08CF2806C6000000790AB191000074084F33F8
S1235F800AAB8C00007708CF2A0C006208F4ABFE0308F4AB8000B508CF2806C60000008AFD
S1235FA008F4A9FE030AAB8D000084084F2A08CF330AB191000088084F3308F4ABFE0308D8
S1235FC0F4AB8001350C00A946F40000020037000006C60000009C0AB191000095084E336E
S1235FE00AB191000098084433200043075F8C0C00A906C6000000A20AB1910000A0085F6F
S1236000B30C00A906C6000000A80AB1910000A6085FF3084E2408F4A5FE0308F4A6FE0395
S1236020084E21084E220000040AB1910000B50844330C00B100000408F4BD0402AE0AFAB7
S12360406600ACB808F4BF00200660F4000002003802000552A03130003902000509A1328D
S12360602A003A02003C020008F4B7030C0008F4AFC4007308F4AB84013508F4B6FE0308B8
S1236080F4A8FE0308F4B000200108F4B10032A908F4A5FE0308F4A6FE0308F4A40000A382
S12360A008F4A10008A30AA18F0000DC084E22084E230C00E0084E21084E22084E23000039
S12360C004FE513130003400000859A20859A308D9A508D9A651800000000B56F4007FFF1C
S12360E0FF0AB78000010E59E40056020051000051810000000B0AB78100011559E400569F
S123610003005101000AB7220AB702000004313500322A00341F000859A20859A308C1A5F2
S123612057800056B000F0910B0A3F220E31310A3F0245821B5700D84EF00000001E21C678
S1236140E05602E021E40057F4007FFFFF21C66C21E5002000A256490044A0262000470229
S1236160904056200056B00044A62620004702904056260056B50044A726200047029040B5
S123618056270057810056B100F0890B08D9A60A3F230E31530A3F0345831B5701D84EF0F9
S12361A00000001E21C6E05603E021E40057F4007FFFFF21C66C21E5002000A25661000A14
S12361C03F820001570AB7230A3F8300015A0AB7230A3FA200015F0A3FA300015F0AB70358
S12361E044A12620004702904056210056B10044A82620004702904056280056B60044A917
S12362002620004702904056290034010057B40020002A20002A0AF9460D022D0AF906003A
S123622001770AF9460A3F2408E2A808CF2A571000FE03085AA834210057B90020002A2058
S1236240002A0D022D0AF9060001850AF9460A3F2508E2AC08CF2E57110056900020001075
S1236260FE03085AAC0AABAF00018C08E2AC08CE2EFE03313400085AAC08DCE90AAB8D00FD
S12362800194084F2A08DCE90D01D00AF90600019D0AF9460A3F26F4990018DCE0F081D236
S12362A03130002000D2F089002000D2564900084F2A08DCE90D01D00AF9060001AC0AF998
S12362C0460A3F27F4990018DCE0F081D23130002000D2F091002000D2563700084F2A0884
S12362E0DCE90D01D00AF9060001BB0AF9460A3F28F4890018DCE0F081D23136002000D28B
S1236300F0890044D9D256330064F4000000EA084F2AF4890018DCE0F081D23136002000AA
S1236320D2F089002000D2563800205800000004F18800F4800048D8002000C221E4C24913
S1236340D0E2F110E22000CAF088CA2000DAF098DA4FDCDAF080DA48E01E4958F22000F2E2
S12363601DDCD249C0D22000FAF488FA2000EAF498EA4FDCEAF480EA48E01E4958C2200027
S1236380C219DCE249C0E22000CAF088CA2000DAF098DA4FDCDAF080DA48E01E4958F220A5
S12363A000F21DDCD249C0D22000FAF488FA2000EAF498EA4FDCEAF480EA48E01E4958C215
S12363C02000C219DCE249C0E22000CAF088CA2000DAF098DA4FDCDAF080DA48E01E495857
S12363E0F22000F21DDCD249C0D22000FAF488FA2000EAF498EA4FDCEAF480EA48E01E49DD
S123640058C22000C219DCE249C0E22000CAF088CA2000DAF098DA4FDCDAF080DA48E01E9D
S12364204958F22000F21DDCD249C0D22000FAF488FA2000EAF498EA2000EA2000EA2000C9
S12364401E49580000000CF18800F4800048D8002000C221E4C249D0E2F110E22000CAF0FF
S123646088CA2000DAF098DA4FDCDAF080DA48E01E4958F22000F21DDCD249C0D22000FA70
S1236480F488FA2000EAF498EA4FDCEAF480EA48E01E4958C22000C219DCE249C0E2200022
S12364A0CAF088CA2000DAF098DA4FDCDAF080DA48E01E4958F22000F21DDCD249C0D22070
S12364C000FAF488FA2000EAF498EA4FDCEAF480EA48E01E4958C22000C219DCE249C0E208
S12364E02000CAF088CA2000DAF098DA2000DA2000DA20001E49580000000CFEF0FEF0FE57
S1236500F0FEF0FEF0FE15FE60FE1EFE0301555502AAAA0012C0FE03C00000200000FE0368
S1236520C00000FE03C00000200000FE03C00000FE03C00000200000FE03C00000FE03C092
S12365400000200000FE03C00000FE03C00000200000FE03C00000FE0C7EB85210624E1052
S1236560624EFE03C00000200000FE03C00000FE03C00000200000FE03C00000FE03C00062
S123658000200000FE03C00000FE03C00000200000FE03C00000FE03C00000200000FE0392
S12365A0C00000000001000001FE03C00000200000FE03C00000FE03C00000200000FE0391
S12365C0C00000FE03C00000200000FE03C00000FE03C00000200000FE03C00000FE03C0F2
S12365E00000200000FE03C00000FE03C00000200000FE03C00000FE03C00000200000FE35
S123660003C00000FE03C00000200000FE03C00000FE037FFFFFFE0602AAACFE03C0000076
S1236620200000FE03C00000FE03C00000200000FE03C00000FE03C00000200000FE03C031
S12366400000FE03C00000200000FE03C00000FE03C00000200000FE03C00000FE03C00031
S123666000200000FE03C00000FE03C00000200000FE03C00000FE03C00000200000FE03B1
S1236680C00000FE037FFFFFFE0602AAACFE03C00000200000FE03C00000FE03C0000020D9
S12366A00000FE03C00000FE03C00000200000FE03C00000FE03C00000200000FE03C000D1
S12366C000FE03C00000200000FE03C00000FE03C00000200000FE03C00000FE03C00000B1
S12366E0200000FE03C00000FE03C00000200000FE03C00000FE037FFFFFFE09C0000020AE
S12367000000FE03C00000FE03C00000200000FE03C00000FE03C00000200000FE03C00070
S123672000FE03C00000200000FE03C00000FE03C00000200000FE03C00000FE03C0000050
S1236740200000FE03C00000FE03C00000200000FE03C00000FE03C00000200000FE03C010
S12367600000FE037FFFFF0C00B6FE150D0040FE270D00E6FE030D0125FE030D00E2FE1526
S1236780084F3108CF33FE12084F31084F33FE3C084F3321E40B0EA0B10110D821F30020F1
S12367A097000AE3800867F300000408443306C420085FF300000408443306C420085FB321
S12367C000000408E7B300000408E7B320001B57670000000408443307708400025708444D
S12367E03307708400025700000408F4A5FE0308F4A6FE030AB1910000620846330AB1914A
S1236800000065084F3321F7000AB3B300009E0AB3B40000A40AB3B50000930AB3B60000D2
S12368207B08CF2806C6000000790AB191000074084F330AAB8C00007708CF2A0C0062081C
S1236840F4ABFE0308F4AB8000B508CF2806C60000008A08F4A9FE030AAB8D000084084FA0
S12368602A08CF330AB191000088084F3308F4ABFE0308F4AB8001350C00A946F40000028C
S12368800037000006C60000009C0AB191000095084E330AB191000098084433200043071E
S12368A05F8C0C00A906C6000000A20AB1910000A0085FB30C00A906C6000000A80AB1914B
S12368C00000A6085FF3084E2408F4A5FE0308F4A6FE03084E21084E220000040AB19100B6
S12368E000B50844330C00B100000408F4BD0402AE0AFA6600ACB808F4BF00200638020049
S12369003902000503A162F4000000803A1000057FA23B02003C0300235D000465A208F446
S1236920B7030C0008F4AFC4007308F4AB84013508F4B6FE0308F4A8FE0308F4B000200125
S123694008F4B10032A908F4A5FE0308F4A6FE0308F4A40000A308F4A10008A30AA18F00A1
S123696000DD084E22084E230C00E1084E21084E22084E230000040AB723300A003130006D
S1236980044215340000205D00205D000859A20859A30A20C00000F556F400CCCCCC565927
S12369A00056510008D9A508D9A60D01B7F2980044D8450EA0FC0A26202000450EA0FF0A59
S12369C02621331B0034260021E500F09B00F08BD0F09BD2F089D24EDCD244A2E22000322A
S12369E05651262000470290405622000D01B7F2980044D8450EA1120A26242000450EA13C
S1236A00150A2625331B0034510021E500F09B00F08BD0F09BD2F089D24EDCD244A4E220CB
S1236A2000325661262000470290405624000AB7030000040AB7233134003456000859A2F2
S1236A400859A30A20C000013056F40055555556590056510008D9A508D9A60D01B7F29818
S1236A600044D8450EA1370A26222000450EA13A0A2623331B0034CA0021E500F09B00F00B
S1236A808BD0F09BD2F089D24EDCD244A3E220003256512620004702904056230060F00009
S1236AA000001F0512A064F40000008057E1003128000AF9460D01FA20580005F42000FFB2
S1236AC0FF60700000001F1E21000AF90600015B0AF9460A2F2930160064F4000000CF0DFB
S1236AE001B7313500F2980044D8450EA1640A26262000450EA1670A2627331B0034F500D7
S1236B0021E500F09B00F08BD0F093D2F089D24EDCD244A5E2200032566126200047029006
S1236B2040562500F68300200060545B0021863327805320CF760EA17E200054218F002044
S1236B40003A21A4004FDC891EDC005FDCF321C7005EDCFB21E7005FDCF321C7002000FB00
S1236B6021E7002000C820003A20CE002440002000450E219257F4007FFFFF200019576394
S1236B800034400044F00000001A4EDC1B59DC0060F0D0000005200002210E005670320047
S1236BA0001A0504A056700000001BF09800F480D044F0E200001BF01800F080D2F818E2F4
S1236BC0F480D2F818D2F080E2D818E22000D256580056700000001C6070000000050460AA
S1236BE0A7205A000AB70300000457E10020003AF8983A19DC00F30A860E71C3205400B06E
S1236C00900010DC00FC80006BDCDE0C01C9E0907C02204002F078134C0057E0006BDCDE0A
S1236C20574801F3930047D3450EF1D8060AA001DB15E0930057E31420003216DC4C21E6FB
S1236C40F620007421C5ED21E6492000EB56F000000006128D0302A0501C18002000D1195A
S1236C600A00F48000FD80F02000264EDC542000550290504EDC7502707012E4030E71F21F
S1236C8047F4000000012000740E21F020EE0021C6000C01F221C61321C4004E5C0056F03E
S1236CA0AE0000071F100302A070108D002000D900000CF18800F4800048D8002000C22125
S1236CC0E4C249D0E2F110E22000CAF088CA2000DAF098DA4FDCDAF080DA48E01E4958F27C
S1236CE02000F21DDCD249C0D22000FAF488FA2000EAF498EA4FDCEAF480EA48E01E49586E
S1236D00C22000C219DCE249C0E22000CAF088CA2000DAF098DA4FDCDAF080DA48E01E49A3
S1236D2058F22000F21DDCD249C0D22000FAF488FA2000EAF498EA4FDCEAF480EA48E01E84
S1236D404958C22000C219DCE249C0E22000CAF088CA2000DAF098DA4FDCDAF080DA48E029
S1236D601E4958F22000F21DDCD249C0D22000FAF488FA2000EAF498EA4FDCEAF480EA48DB
S1236D80E01E4958C22000C219DCE249C0E22000CAF088CA2000DAF098DA4FDCDAF080DA13
S1236DA048E01E4958F22000F21DDCD249C0D22000FAF488FA2000EAF498EA2000EA200004
S1236DC0EA20001E49580000000CFEF0FEF0FEF0FEF0FEF0FE4BFE0FFE0FFE030000AEFE24
S1236DE0037FFFFFFE030000AEFE037FFFFFFE030000AEFE037FFFFFFE030000AEFE037F86
S1236E00FFFFFE0F000200FE06FE427FFFFF7FFFFF7FFFFF7FFFFF7FFFFF7FFFFF7FFFFFB2
S1236E207FFFFF7FFFFF7FFFFF7FFFFF37837A4000007FFFFF7FFFFF7FFFFF7FFFFF7FFF74
S1236E40FF7FFFFF7FFFFF7FFFFF7FFFFF7FFFFF7FFFFF37837A4000007FFFFF7FFFFF7F54
S1236E60FFFF7FFFFF7FFFFF7FFFFF7FFFFF7FFFFF7FFFFF7FFFFF7FFFFF37837A400000B4
S1236E807FFFFF7FFFFF7FFFFF7FFFFF7FFFFF7FFFFF7FFFFF7FFFFF7FFFFF7FFFFF7FFF8E
S1236EA0FF37837A40000000095F0000010000010006D100883F0000447FFFFF7FFFFF7F96
S1236EC0FFFFFFF92F00095F0000017FFFFFFE4BFE0C40000000095F0000010000010006A0
S1236EE0D100883F0000517FFFFF7FFFFF7FFFFFFFF92F00095F0000017FFFFFFE180B2DD3
S1236F009D3619630173D633126F1029A89F3C5F74FDF483509C7F03B08059C57FDF3CFEC9
S1236F2012FE0C40000000095F0000010000010006D100883F00005E7FFFFF7FFFFF7FFF13
S1236F40FFFFF92F00095F0000017FFFFFFE57FE03C00000200000FE03C00000FE03C00069
S1236F6000200000FE03C00000FE03C00000200000FE03C00000FE03C00000200000FE03A8
S1236F80C00000FE03C00000200000FE03C00000FE03C00000200000FE03C00000FE03C028
S1236FA00000200000FE03C00000FE03C00000200000FE03C00000FE66FE0C400000000993
S1236FC05F0000010000010006D100883F00006B7FFFFF7FFFFF7FFFFFFFF92F00095F003D
S1236FE000017FFFFFFE4BFE0C40000005555500027BFFB36D0519A3D6A8886487ED173546
S12370000F8AFA00707CFA0071E4FA0074F227F6B60AF50117FA0F8AFA00707CFA0071E48C
S1237020FA00738027710018340327F5FA0077FC3F04F50F27FA2771001037DC37AC27FAC8
S123704037DC340337B5001FFA0077FC3F04F50F27FA2771001437DC37AC27FA37DC3403F5
S123706037B50020FA0077FC3F042771001C340337B5001EFA0077FC3F0427F73920F90734
S12370803910F9073940F90737B500C8FA009FBE3840F907FA02000037B5000AFA009FBE5E
S12370A027F717F50F89B6063820F9073920F907B0043810F9073910F90727F7343F37AFE1
S12370C0379C27FA3880FC1F3A010F88001817F50F89B6063820F9073920F907B0043810EE
S12370E0F9073910F90717350F88357E27773716B60EF5CE17FA0F87F58E17FA0F8617351F
S12371000F89B00EF5CD17FA0F87F58D17FA0F86F50117FA0F8927F734073FFA274F851444
S1237120B60017350F7E85088A00850A8A0285148A048504378F009E17F50F7EB71A374590
S12371400000850227030002B6002703000037DC277A379D150017310F7EB0708510CD1292
S1237160379DD500F8FEB63627030012B60027030010CD12D50017FA0F7EB6128500CD02E6
S1237180379DF5FE27030002B60027030000DA00B0002703000427030012B6302703001004
S12371A0B02A37450010851227030012B6002703001037DC277A379DD500277A8500CD0250
S12371C0379D277A27030002B60027030000DA00270100043780FF58374500108512CC0621
S12371E03F0C27F734043FF6274F17F50FA3B6F6F50117FA0FA317350F8827050002850284
S123720037B80002378C0170FA0200008502B62817F50F8AB70C3735000037B55EB48A0880
S1237220374A0006B00A3735000037B54EE88A08374A000637B504008A00B02C17F50F8A67
S1237240B7123735000037B567678A08374A000637B504008A00B0103735000037B557FB3E
S12372608A08374A000637B502008A008502FA0070EE37B58E0037FAFC1C2705000437452B
S123728000043738000EBE10F50F37BDFD40379D17F50F8727DA27030004B0DE27F53401E2
S12372A037450006850834033735000F37B5FD20FA0071183F062705000485003735000A0D
S12372C0FA02E7B48804BF3417F50F88B6F637B5001E340137450006850834033735000F45
S12372E037B5FD20FA0071183F068A08374A0006F50217FA0F883980FC1A27030004B0B69E
S123730017F50F88B6F685003735000AFA02E7C83735000337268A0437350002FA02E7B415
S12373203707371537B17F0037FAFC1C8504340137450006850834033735000F37B5FD2087
S1237340FA0071183F068A08374A0006F50217FA0F883980FC1A17F50F88B6F617350FA38D
S1237360F50217FA0F8837B500C8FA009FBE17350F88270300023780FE82CC0A3F0C27F7DA
S123738034043FFA274F27050000850037B80002378C0150FA0070EE8500378600A017F506
S12373A00F8AB73637B50100340127F53735000834033735000037B56507FA0079FA3F06E4
S12373C037B50100340127F53735001034033735000037B56513FA0079FA3F06B03437B566
S12373E00100340127F53735000834033735000037B5559BFA0079FA3F0637B50100340170
S123740027F53735001034033735000037B555A7FA0079FA3F0627F58A0237B128068A0447
S123742037B50001275C3D02340937AD37BD00FF340937B500FFFA0078A83F083780009CA9
S123744017F50F8AB73637B50100340127F53735000834033735000037B56DD6FA0079FAA5
S12374603F0637B50100340127F53735001034033735000037B56EA7FA0079FA3F06B034CF
S123748037B50100340127F53735000834033735000037B55CF9FA0079FA3F0637B50100B3
S12374A0340127F53735001034033735000037B55DC5FA0079FA3F0627F58A0237B12806DA
S12374C08A0437B50001275C3D02340937AD37BD01FF340937B500FFFA0078A83F082703A3
S12374E000003780FEA227F5FA0070EECC063F0827F734043FF8274F37B500128A0037B52D
S123750034568A0237B50001275C340937AD37BD012E340937B50001FA0078A83F0837B526
S1237520012EFA00760A8A06374A000485048800B60885068802B60237B50001B0FE27F536
S1237540CC083F0A27F734043FFA274F17F50F88B6F617F50FA3B6F0F50117FA0FA327056D
S123756000043745000437380002BE1EF50F37BDFD40379D17F50F8627DA37BD800085048E
S123758027F437DD27157D2027030004B0D037B5820037FAFC1CF50217FA0F883980FC1A0C
S12375A017F50F88B6F6F50F27FA37F5FD04277A37AC27FA277A27758A02374A0000F50F33
S12375C027FA37F5FD02277A37AC27FA277A3707371527758102374300008A02374A0000E5
S12375E0F50F27FA37F5FD00277A37AC27FA277A277B27F58102374300008A02374A00002B
S123760017350FA3CC063F0827F734053FFA274F17F50F88B6F617F50FA3B6F0F50117FA8F
S12376200FA317FA0F88C5083705FA0070EE270500043745000437380002BE10F50F37BDA4
S1237640FD40379D17F50F8627DA27030004B0DEF50F27FA37B5005137FAFD202735FD228C
S1237660C509370537FAFD2437AC27FA37B5820037FAFC1CF50117FA0F883980FC1A17F576
S12376800F88B6F627050004850437B80002BE14F50F37BD8000379D850427F437DD2715E7
S12376A07D2027030004B0DC37B5820037FAFC1CF50117FA0F883980FC1A17F50F88B6F6FC
S12376C0F50F27FA37F5FD04277A37AC27FA277A27758A02374A0000F50F27FA37F5FD0215
S12376E0277A37AC27FA277A3707371527758102374300008A02374A0000F50F27FA37F5BF
S1237700FD00277A37AC27FA277A277B27F58102374300008A02374A000017350FA3CC068A
S12377203F0A27F7340F274F17F50F88B6F617F50FA3B6F0F50117FA0FA327050000374511
S1237740000037380002BE22F50F37BDFD40379D17F50F8627DA7C0527C5370537BDFD206F
S1237760374500002774279A27030000B0CC37B5820037FAFC1CF50217FA0F883980FC1A62
S123778017F50F88B6F617350FA3CC023F0827F7340F274F17F50F88B6F617F50FA3B6F0F9
S12377A0F50117FA0FA3270500003745000037380002BE22F50F37BDFD40379D17F50F8669
S12377C027DA7C0527C5370537BDFD20374500002774279A27030000B0CC37B5820037FACD
S12377E0FC1CF50117FA0F883980FC1A17F50F88B6F617350FA3CC023F0827F7340D274FC9
S123780017F50F88B6F617F50FA3B6F0F50117FA0FA317FA0F88C5043705FA0070EE2705C7
S123782000003745000037380005BE10F50F37BDFD40379D17F50F8627DA27030000B0DE23
S1237840F50F27FA37B5004737FAFD202735FD22C505370537FAFD2437AC27FA37B50001BA
S12378608A003745000037380003BE1C7C0A27C53705277AF50F37BDFD24379D277A374559
S123788000002774279A27030000B0D237B5850037FAFC1C3980FC1A17F50F88B6F61735B8
S12378A00FA3CC023F0627F734053FF8274F17F50F88B6F617F50FA3B6F0F50117FA0FA38F
S12378C0F50217FA0F88C5103705FA0070EE270500063745000637380005BE10F50F37BDAE
S12378E0FD40379D17F50F8627DA27030006B0DEC50BB70EF50F27FA37B5004D37FAFD20D2
S123790037AC27FAB00CF50F27FA37B5004937FAFD2037AC27FAC50BF8FFB6103705277A8D
S1237920F50F27FA277A37FAFD2237AC27FAB008F50F27FA2735FD2237AC27FAC5113705BB
S1237940277AF50F27FA277A37FAFD242735FD262735FD28851637FAFD2A37AC27FA37B587
S1237960850037FAFC1C3980FC1A2705000485048816BC728512CD14379D850427F427F4D6
S123798037DD3755000095028A02374A000017F50F88B6F637B500018A06374500063738E2
S12379A00003BE1A27C53705277AF50F37BDFD20379D277A374500062774279A2703000687
S12379C0B0D437B5830137FAFC1C8516FCFF8804B604F50117FA0F88B002F50217FA0F889B
S12379E03980FC1A27030004B08017F50F88B6F617350FA3CC083F0C27F7340F274F17F507
S1237A000F88B6F617F50FA3B6F0F50117FA0FA3270500003745000037380008BE10F50F11
S1237A2037BDFD40379D17F50F8627DA27030000B0DEF50F27FA37B5005E37FAFD202735CA
S1237A40FD22C50F370537FAFD242735FD26C51037FAFD28C51137FAFD2A37AC27FA37B5D9
S1237A6000018A003745000037380003BE1C7C0C27C53705277AF50F37BDFD2A379D277ACA
S1237A80374500002774279A27030000B0D237B5880037FAFC1CF50117FA0F883980FC1A34
S1237AA017F50F88B6F627050000374500003738000EBE10F50F37BDFD40379D17F50F87D5
S1237AC027DA27030000B0DE37B58E0037FAFC1C27F5340137450004850634033735000F18
S1237AE037B5FD20FA0071183F0685103735000337268A102705000085103735001EFA026F
S1237B00E7B48800BF3417F50F88B6F637B5001E340137450004850634033735000F37B514
S1237B20FD20FA0071183F068A06374A0004F50217FA0F883980FC1A27030000B0B68510B4
S1237B403735001EFA02E7C88A10B75C17F50F88B6F68510FCFF37350002FA02E7B48A00D1
S1237B608510F901B70EF50F37BDFD40379D17F50F863745000027DA45013715778037FACC
S1237B80FC1C8510340137450004850634033735000F37B5FD20FA0071183F068A06374A60
S1237BA00004F50217FA0F883980FC1A17F50F88B6F617350FA3CC023F0827F717F50F882C
S1237BC0B60217F50FA3B71E17F50F7F17330F7F370537B80040BD0817350F8817350FA3D3
S1237BE017350F7F37B5FFFFB00217350F7F27F527F734053FFA274FFA007BBC27F6B7000A
S1237C0027F5B028C509F806B40CFA02E8007C507C587C607C687C707C78F8FDB706F8FE14
S1237C20B718F8FFB71CB01A17F50F8AB60427F5CC063F0A27F737B5012F8A00B03A37B5AD
S1237C4001268A00B03237B5003F8A00B02A37B500208A00B02237B500218A00B01A37B549
S1237C6001228A00B01237B501238A00B00A37B501248A00B00237B501258A00F50117FA4D
S1237C800FA317FA0F88C5003705FA0070EE270500043745000437380002BE10F50F37BD46
S1237CA0FD40379D17F50F8627DA27030004B0DEF50F27FA37B5005337FAFD202735FD2224
S1237CC0850037FAFD2437AC27FA37B5820037FAFC1C3980FC1A17F50F88B6F627050004C0
S1237CE0850437B80002BE14F50F37BD8000379D850427F437DD27157D2027030004B0DC9D
S1237D0037B5820037FAFC1CF50117FA0F883980FC1A17F50F88B6F6F50F27FA37F5FD029C
S1237D20277A37AC27FA277A27FF8A02F50F27FA37F5FD00277A37AC27FA277A27FF370E48
S1237D40371AF68081028A02C509F806B40CFA02E8007DD47DE27DF07E0A7E247E3EF8FDE1
S1237D60B706F8FEB722F8FFB73EB03CF50F27FA1775FD03371537F1FD04277A37AC27FAD0
S1237D80277A37FA0F828A02378000C6F50F27FA1775FD03371537F1FD04277A37AC27FAA8
S1237DA0277A37FA0F848A02378000A6F50F27FA1775FD03371537F1FD04277A37AC27FAA6
S1237DC0277A37F70F8237FA0F8027350F828A02B07E37F50F80F910B77617098002B07025
S1237DE037F50F80F920B76817098002B06237F50F80F940B7001709800237F50F84F903D0
S1237E00B74E17094002B04837F50F80F980B7001709800237F50F84F90CB7341709400261
S1237E20B02E37F50F807901B7001709800237F50F84F930B71A17094002B01437F50F8038
S1237E407902B7001709800237F50F84F9C0B7001709400217350FA38502B60237B500018F
S1237E608A028502CC063F0A27F734053FF8274FFA007BBC27F6B706277527F5CC083F0CEA
S1237E8027F7C50BF801B710F802B714F80BB718F80CB71CF815B720F816B72437B50020E9
S1237EA08A00B02237B500218A00B01A37B500268A00B01237B500278A00B00A37B5002838
S1237EC08A00B00237B500298A00F50117FA0FA317FA0F8827F5FA0070EE27050006374540
S1237EE0000637380002BE10F50F37BDFD40379D17F50F8627DA27030006B0DEF50F27FAAB
S1237F0037B5005337FAFD202735FD22850037FAFD2437AC27FA37B5820037FAFC1C39800A
S1237F20FC1A17F50F88B6F627050006850637B80002BE14F50F37BD8000379D850627F466
S1237F4037DD27157D2027030006B0DC37B5820037FAFC1CF50117FA0F883980FC1A17F544
S1237F600F88B6F6F50F27FA37F5FD04277A37AC27FA277A27758A04374A0002F50F27FA50
S1237F8037F5FD02277A37AC27FA277A3707371527758104374300028A04374A0002F50F30
S1237FA027FA37F5FD00277A37AC27FA277A277B27F58104374300028A04374A0002173511
S1237FC00FA3CC083F0C27F737F50F8427F73735000037B57FCE27730F9227FB17FD0F9418
S1237FE0379DD50017FA0F9027F73B40F920000637B50001B0FE27F527F73B40F920FFFA0A
S123800027F73405274F17FA0F8C37B5000134013735000F37B50F8C340337450008850A75
S1238020FA00807ACC003F0A27F73405274F37FA0F8C37B5000234013735000F37B50F8C75
S1238040340337450008850AFA00807ACC003F0A27F73407274F27730F8C37B500043401A0
S12380603735000F37B50F8C34033745000A850CFA00807ACC003F0C27F73407274F850E3F
S1238080B73C37F50F96B7023940F920B0F0FA007FFA3840F92037F5F90AFC0337FAF91AB7
S12380A0850E37FA0F96850A37FA0F9C850C37FA0F9E850237FA0F98850437FA0F9A39403E
S12380C0F920CC003F0627F7343F37AF379C27FA3FFE274F37F50F9217FD0F94379DD50027
S12380E017F80F90B70039010FA137F50F96B77A8A0037B80032B30237B500328A002731CB
S12381000F9627710F9827330F9AB60027330F9827730F9227710F9C27330F9EB600273328
S12381200F9C37DC277A379DD50017FA0F9037F50F9217FD0F94379DD50017F80F90B704ED
S123814017F50F90DA00B00227010000B6AC8500B70A37F5F90A37B1924037FAF91AB00E29
S123816037F5F90A37B102EC37FAF91AB0003840F9203840F9223F02357E2777204080006C
S1238180010204081000FA0081BC3860FA41FA008198FA0089F427F717F50020F801B70826
S12381A03901F91F2738F91E0002B0003903F91F2738F92201003901F92027F7340C274F4B
S12381C037B500018A008500FCFBBE1437B500FF340127F534018500FA0083EA3F0427030C
S12381E00000B0DE37B500018A008500FCFEBE1837B500FF340127F53401850037B10080C3
S1238200FA0083EA3F0427030000B0DA351827F734043FFA274FF50117FA1002FA0081BC5A
S1238220F507CA04C504F8013783013A0505C505F80A3784010EC504F805B34237B500FF73
S1238240340137350001C505B70227743711B6F63402C5043705FC7BFA0083EA3F04C50540
S1238260F8063785009CC504F806378600D637B5006EFA009FBE378000CA0104B0A20305B9
S1238280B0A8F50037BD817C379DC5053705277B27D5B71637B500FF3401C5053705277B8F
S12382A027D53401C504FA0083EA3F04B052C504F801B34CF806B448C505F803B62037B5D2
S12382C000FF340137350008C504F1FEB702277D3711B6F6340237B50001FA0083EA3F041C
S12382E0B01E37B500FF340137350080C504F1FEB702277D3711B6F6340237B50001FA007A
S123830083EA3F0437B50122FA009FBEFA02000037B500FF340127F53401FC01FA0083EA72
S12383203F0437B500FF340127F53401C5043705FA0083EA3F04FA008B7427F63787FF3CC7
S1238340050537800090C504F8053783FF2A37B500FF340127F53401C5043705FC7BFA0038
S123836083EA3F043780FF1037B500FF37BD00FF340937B50081FA0083EA3F0437B500FF66
S123838037BD00FF340937B50082FA0083EA3F04F501CA04C504F805B21237B500FF340123
S12383A03401C5043705FA0083EA3F040304B0E037B503E8FA009FBEFA02000037B503E83D
S12383C0FA009FBEFA02000037B503E8FA009FBEFA020000F501CA05FA0081BC17351002C2
S12383E0C5053705CC063F0827F734053FFC274FF980378700A217088007C5073705FCFFD0
S12384008A02C50FC60DCA0DC50F3710277AF50F37BD0FA4379D277A3745000227D6C70D23
S1238420CA0D27DAFA00899627F63787010437B5800437FAFC1837B5010037FAFC1C173530
S1238440FC1E270500023745000237380002BC2EF50F37BDFD40379DF58B27DAF50F37BD75
S12384600FA4379D27D53705277AF50F37BDFD20379D277A374500022774279A2703000208
S1238480B0C037B5800037FAFC1A17F5FC1FF980B7F4FA0089D237800098C5073705FCFFC3
S12384A08A02C50FC60DCA0DC50F3710277AF50F37BD0FA6379D277A3745000227D6C70D81
S12384C0CA0D27DAFA00899627F6B76437B5800437FAFC1837B5040037FAFC1C1735FC1E1B
S12384E0270500023745000237380005BC2EF50F37BDFD40379DF58727DAF50F37BD0FA63B
S1238500379D27D53705277AF50F37BDFD20379D277A374500022774279A27030002B0C0AA
S123852037B5800037FAFC1A17F5FC1FF980B7F4FA0089D2CC043F0827F734053FFC274FC5
S12385403711CA00F5104500B70237143701B6F6CA02C50DB702C502CA03B0FE0503C5026B
S123856037053401C503340137B50001FA0083EACC043F0C27F73405274FF800B714F80191
S1238580B728F802B73CF803B750F804B764F805B7783780008C37B5003F3401C509370519
S12385A0340137B50082FA0083EA3F04B07237B5003F3401C5093705340137B50081FA0042
S12385C083EA3F04B05A37B5001F3401C5093705340137B50005FA0083EA3F04B04237B5E5
S12385E0001F3401C5093705340137B50004FA0083EA3F04B02A37B5001F3401C509370526
S1238600340137B50003FA0083EA3F04B01237B5001F3401C5093705340137B50002FA005F
S123862083EA3F04CC003F0427F7000810204080FF00081950FF34043FF0274F17F51002F7
S1238640B702CC103F1227F73A010FA2000837B500328A00B0002705000017F50FABB70E0F
S123866017350FAB37B5FFFD8A0637B500018A04B00EF50117FA0FAB37B500028A0637B514
S123868000058A0485068A0885088804378E02C4FA007BF28A0C8508BC0227030008B0E474
S12386A0850CB7F2277AF50F37BD0FB6379D277A374500082774279A850C7980B71637B586
S12386C03FFF37BD0FD6279A2708000CC0008500FC0137BD0FCA279A850837B80001BF4037
S12386E0FCFE8A0AF50F37BD0FC2379D3745000A27742795B706850A27F437DD27110000BB
S1238700850C7940B71A8500FC01277AF50F37BD0FC2379D277A3745000A2774279A2708C8
S1238720000CC000F50F37BD0FE2379D3745000827742795880CB400850C279AF50F37BD3F
S12387400FD6379D3745000827742795880CB208850C279A850037BD0FCA279AF50F37BDD6
S12387600FE2379D37450008277427958A0C37BD0FCA2795B708850827F437DD2711000083
S1238780B00EF50F37BD0FD6379D850C374500082774279A850C27FD8A02277AF50F37BD1B
S12387A00FE2379D277A374500082774279A3A020FA20014270D000285022791279A270D04
S12387C0000285022791279A850C27FD27FD27FD27FD27FD8A0237B801FFBC0027030002EB
S12387E0850227FDCA0F8508FCFFBE3837B500068A0A3745000ABD10F50037BD862A379D2D
S123880027D5C80FB3022701000AB0E23735003FF506C00BB70227743711B6F6374A0002CC
S1238820C503F63FCA0FB03637B500048A0A3745000ABD10F50037BD8631379D27D5C80F5A
S1238840B3022701000AB0E23735000FF504C00BB70227743711B6F6374A0002C503F60FC4
S1238860CA0FF50F37BD0FD6379D3745000827742795880C3783009C27FF27FF27FF27FF0D
S123888027FF8A0237B801FFBC0027030002850227FDCA0E8508FCFFBE3837B500068A0AC4
S12388A03745000ABD10F50037BD862A379D27D5C80EB3022701000AB0E237350001F50641
S12388C0C00BB70227743711B6F6374A0002C503F63FCA0EB03637B500048A0A3745000A39
S12388E0BD10F50037BD8631379D27D5C80EB3022701000AB0E237350001F504C00BB702FE
S123890027743711B6F6374A0002C503F60FCA0EC50EC70FCA0F850837B80001BF22040FA9
S1238920CB020F021709010F1708020FF50F37BD0FC2379D3DFC3745000827742795B7008D
S12389401709020FC50F370534018508FA0085763F023780FD422733002237F50022F90120
S1238960B710FA007FC834013735000F37B50FB6FA01C2FE3F02CC103F1227F73405274F94
S1238980F50F37BD0FB6379D3745000227742795CC003F0427F7340C274F17F50FA3B70015
S12389A00501B022F50117FA0FA337FFFC180FF837FFFC1A0FFA37FFFC1C0FFC37FEFC1ED4
S12389C00FFE3880FC1FF501CA01C5013705351827F73880FC1F37FF0FF8FC1837FF0FFA22
S12389E0FC1A37FF0FFCFC1C37FE0FFEFC1E17350FA327F734043FF6274F05050504381E40
S1238A00FA1937F5F7063705F60F37B8000FB76427050008F502CA03850837B80004BC5434
S1238A20C503371017FAFA1937F5F7063705F60F37B8000FB72027050006F501CA02850641
S1238A40FCFCBC12C50237058A0037F5F7068600B60CC505B710CA04B00C270300080403FA
S1238A60B0B2270300060402B0D0C50737143714C1093713CA05B0E645043715C105730031
S1238A8037FA0FF437F80FAC3787009A37F50FF43787008637F50FAC79FFB67C17331000FE
S1238AA017F51000F804B302F50417FA1000F50F37BD0FEE379D17F510003705277BC5053E
S1238AC027DAC504B73A17F50FAEC805B60617F51000277BC50427DA17F50FAEB622173312
S1238AE0100017F51000F804B302F50417FA1000F50F37BD0FEE379D17F510003705277BB8
S1238B00C50427DA37F50FF437B80002B70237B80003B60437B5001037FA0FB0C50517FA3B
S1238B200FAE37FF0FF40FAC37F50FF437B80002B70237B80003B63237F50FB027310FB0CB
S1238B4027F6BE2637B5000337FA0FB017F51000B618F50117FA1000F50F37BD0FEE379D67
S1238B6017F510003705277B17F50FF527DACC0A3F0C27F7340C274F17F51000B716F50F04
S1238B8037BD0FEE379D17F510003705277B27D5CA0117311000B0FE0501C50137053518F0
S1238BA027F737F50FF427F7343F37AF379C27FA3FFC274F17F5F907F603CA032738F922FC
S1238BC00100CB010314C503F803B60437B5FFFF8A00B01637B500018A00B00EC503B6043F
S1238BE037B5FFFF8A00B00237B500018A002738F922010037B5000234013735000F37B5CF
S1238C000FB4FA009E203F0227F6B6002704000017F5319B17FA0FB437F50FF4FCFCB60607
S1238C2085003735000A37268A00850037F10FF637FA0FF6850037FA0FB2F50117FA1001D7
S1238C403F04357E2777340C274F2705000017F51001B70C37F50FF68A00800037FA0FF649
S1238C60173510018500351827F7340D274FF50117FA1002C505F8FFB64837B500FF37BD35
S1238C8000FF340937B50081FA0083EA3F0437B500FF37BD00FF340937B50082FA0083EA8D
S1238CA03F0437B500018A008500FCFBBE1837B500FF37BD00FF34098500FA0083EA3F045A
S1238CC027030000B0DEFA0081BCCC023F0627F7FA0081BCFA020356FA020B12173510026D
S1238CE027F7343F37AF379C27FA3FFC274F37F5FC0C8A0217F5FC0FCA01277AF50F37BD19
S1238D001008379D277A3775180827DA37F518082733180837B807FFB500273518082733AF
S1238D20180A37F5180A37B80400B30C37B80800B506F50117FA10072731180A3F04357ECD
S1238D4027772735180A273518081735100727F737F518082731180827F6BC0437B507FF63
S1238D6037FA18082733180A27F7FA008D423904FC0437B5000F37FAFC0837B5000C37FAA5
S1238D80FC0A3920FC0B27F734043FFC274F37B540008A0237F5180AB60C850227010002E9
S1238DA027F6B6EC37B500F1B000FA008DB4CC043F0627F734043FFC274F37F5180A378700
S1238DC0009817F50025F8FFB70C2731180ACA01F5FF17FA002537800084373B00E037F5E4
S1238DE0180837F0180A8A022731180A373AFF1F8502BC0237B108008A02F50F37BD1008A0
S1238E00379D3745000227D5CA013713F8F8B24CCB80011AC50117FA1005F60CF80CB604EB
S1238E20F50117FA1006B034F50217FA1006B02C17F51005F8F0B72417F51005B71E17F54D
S1238E401006B70217311006B012C50117FA002517F51005CA012733180AB000F5FECA014D
S1238E60C5013705CC043F0627F7340D274F37B503E88A0037F5FC0C7901B6042701000011
S1238E808500B6EC8500BF04C505370537FAFC0ECC023F0627F7204572726F723A20002049
S1238EA04D494449204F766572666C6F77200000340C274FFA008DB4CA01F980B7F2F8F031
S1238EC0B71CF8F7B748F8FEB744F8FFB74017F50024F8FFB70EC501F60F17F80024B62E20
S1238EE0B002FA008F6CB02617080F01C501F8C0B61CFA008D88CA01F850B212370537FA1F
S1238F000048FA00EC72FA02000037F50048FA01B7CA17F51007B74C37F5319837B80400B3
S1238F20BC42FA00AE7027F5FA00C25C37B5000D3735000234033735000037B58E96FA00CF
S1238F40C1043F0437B500173735000234033735000037B58E9FFA00C1043F0437B507D013
S1238F6037FA319817351007351827F734043FA4274F055AFA008D88CA5BF830B700F87EAC
S1238F80B624F518CA5AC55A37870126FA008D88CA5B17F80024B73217F50024F8FFB72A66
S1238FA0C55BF87F3786010AB020C55BB602FA008D88CA5BC55BB602FA008D88CA5BC55B46
S1238FC0F876B700F87EB6BAF526CA5AB0B4FA008D88CA5BF806B614FA008D8837B80001E4
S1238FE0B60AFA008D8837B800F7B600FA009184C55BC85A378600BA0559275C3D093705D7
S123900037AD8A048D06FA008D88CA5B277A8504CD06379D277A27030006B600270300048D
S1239020DA00C55BF980B702FA008D50B020C55BC159CA59275C3D59370537AD8A008D02AA
S123904085048800B60085068802B702C55BF80AB6B08504CD06379D1500FA008D88CA5B76
S1239060C159CA5917088059FA008D88CA5BF8F7B63EC559B63A37B50040FA009A48275C07
S12390803D09370537AD8A048D068504CD06379DD500B71C37450004850627030006B6007C
S12390A02703000437DC277A379DD5003705FA009A48B0D2CC5C3F5E27F73405274F17F5E9
S12390C01004F810B40E370537B100C0FA008E6AC5033705FA008E6ACC003F0427F734077A
S12390E03FFA274F050117F51004F810B302CC063F0C27F737B500F0FA008E6A27F5FA00BB
S12391008E6A27F5FA008E6A37B50076FA008E6A17F510043705FA008E6A37B50026FA0097
S12391208E6A85088A02850A8A048502CD04379DD5003705FA008E6A8502CD04379DD500CD
S1239140C101CA0127030004B60027030002CD04D500B6D237B5000DFA008E6A37B5000A5F
S1239160FA008E6AF517C101CA013712CA013705F67FFA008E6A37B500F7FA008E6ACC0602
S12391803F0C27F737B500F0FA008E6A37B5007EFA008E6A17F51004F810B4043705FA0022
S12391A08E6AB00227F5FA008E6A37B50006FA008E6A37B50002FA008E6A27F5FA008E6A21
S12391C027F5FA008E6A37B50076FA008E6A37B50026FA008E6A27F5FA008E6A27F5FA0001
S12391E08E6A27F5FA008E6AF50027FA17F54476277A37AC27FA277A3705FA008E6AF50020
S123920027FA17F54477277A37AC27FA277A3705FA008E6AF50027FA17F54478277A37AC8C
S123922027FA277A3705FA008E6AF50027FA17F54479277A37AC27FA277A3705FA008E6AE7
S123924037B500F7FA008E6A27F734043FD6274FFA008D88CA25F808B300F508CA25FA00BD
S12392608D88371E371EF680CA24FA008D88C124CA2405210529C529C825378400B0FA0051
S12392808D88CA23C121CA21FA008D88CA28C523F601371E371EF680C128CA28FA008D8811
S12392A0CA27C523F602371E371E371EF6C0C127CA27FA008D88CA26C523F60437143714D4
S12392C0371437143714C126CA26C529370527F427F4275C37DDC526370527759A02375AEB
S12392E00000C52737BE000827F4277C3EFFB6F49102375300009A02375A0000C529370568
S123930027F427F4275C37DDC5283705277B27F59102375300009A02375A0000C528C1217C
S1239320CA21C127CA21C126CA2103293780FF4417088021FA008D88CA22F8F7B602C5212B
S1239340CA22B008FA008D8837B800F7B7FE0522C522C821B624C5253705275C340937AD20
S12393603401C524340127F5FA0078A83F0837B500F0FA008E6A37B500F7FA008E6ACC2A80
S12393803F2C27F7F50F27FA1735317EF50A27FA3902100417F51006277A37AC27FA277A49
S12393A0F910B770F50A27FA3802100417F51006277A37AC27FA277AF901B758F50A27FA7A
S12393C017F51006277A37AC27FA277AF910B644F50A27FA17F51006277A37AC27FA277A96
S12393E0F6E0F820B60AF50F27FAF50117FA317E37AC27FAF50A27FA17F51006277A37AC16
S123940027FA277AF6E0F840B60AF50F27FAF50217FA317E37AC27FAF50F27FA17F5317EF8
S1239420277A37AC27FA277A370527F7340C274F0501F50F27FA17F5317E277A37AC27FA47
S1239440277ACA00F50F27FAF50117FA317EF50A27FA3910100437AC27FA37B500AAFA00B1
S12394609B2E37B5000AFA009FBEFA009D6437B800AAB600F501CA0137B50055FA009B2EC3
S123948037B5000AFA009FBEFA009D6437B80055B6FE0301C501F802B7000501B000F50161
S12394A0CA01F50A27FA38101004F50F27FAC50017FA317E37AC27FAC5013705351827F746
S12394C0340C274F050137B500AAFA009B2E37B5000AFA009FBEFA009D6437B800AAB600DC
S12394E0F501CA0137B50055FA009B2E37B5000AFA009FBEFA009D6437B80055B6FE03015F
S1239500C501F802B7000501B000F501CA01C5013705351827F7340C274F0501F50F27FA0B
S123952017F5317E277A37AC27FA277ACA00F50F27FAF50117FA317EF50A27FA3901100413
S123954037AC27FAFA0094C0CA01F50A27FA38011004F50F27FAC50017FA317E37AC27FACF
S1239560C5013705351827F7FA00938427F6B77AF50F27FA17F5317E277A37AC27FA277AF5
S1239580F801B640F50A27FAF58317FA100337B50C0037FA1000F50317FA100317F51005A6
S12395A017F6100017F610063716F50117FA1001F50817FA100437AC27FA3735000137B583
S12395C0623427735322B036F50F27FA17F5317E277A37AC27FA277AF802B622FA004714AF
S12395E03735000137B5623427735322B010173501941735533D3735000137B56234277363
S123960053222735317C2735317A27353178273531761735317F1735317127F70000035856
S1239620204572726F723A200020427566666572204F766572666C6F77200000340C274FDE
S1239640F50F27FA17F5317E277A37AC27FA277AF802B604FA01BD1CFA01C648F50F27FA2A
S123966017F5317E277A37AC27FA277AF8013786012AF50A27FA37AC27FA3B40002600043B
S12396803820317F17F50026F980378700DC3801180CFA009AE88A0037B80960B33A3B8016
S12396A0317F001637B50013FA009C5E17F5319B17FA31723980317FB07237B500133401A2
S12396C03735000F37B53172FA009E203F0227F6B75A37B50013FA009C5EB050850037B8EE
S12396E004B0B4483A80317F001C37B50011FA009C5E17F5319B17FA3172F50517FA317106
S12397003880317FB02617F53171B72037B500AB34013735000F37B53172FA009E203F02B3
S123972027F6B7081731317137B50011FA009C5E3A40317F006837F5319A37F0317427757D
S123974037ECF500379E37EC37BE961CFA02E85CBF483840317FFA009AA427F6B73CF50A98
S123976027FA3902100137AC27FAB02E37B5001334013735000F37B53172FA009E603F021F
S1239780F50517FA31713840317FFA009AA427F6B708F50A27FA3902100137AC27FAFA0072
S12397A09ABC37B80050B30A37F5532217FD5324379DFA02E5323A01317F005837F5319808
S12397C037B80400BC4AFA00AE7027F5FA00C25C37B5000D3735000234033735000037B54A
S12397E09620FA00C1043F0437B500173735000234033735000037B59629FA00C1043F04EC
S123980037B507D037FA31983801317F2735317C2735317A351827F70000000198C60003C1
S123982098CE0000000298FA001198DE0013990C343F37AF379C3FFC274FF50F27FA17F5DD
S1239840317E277A37AC27FA277AF802B604FA004912378001EAF50A27FA17F51002277A85
S123986037AC27FA277AF607CA03F50A27FA17F51005277A37AC27FA277ACA02C503F8045E
S1239880378600DE0A0100020090F50A27FA17F51005277A37AC27FA277AF60E17F7317F43
S12398A017FA317FF50A27FA17F51000277A37AC27FA277A37058A003A400026001037BDF7
S12398C09818FA02E8183920317F378000943A8000260046850037BD9822FA02E8183940B6
S12398E0317FF50A27FA3802100137AC27FA37FF319A31743F04357E27773840317FF50AE4
S123990027FA3902100137AC27FAB054FA009AE837B80E10B3003901180C37F5317C2775BF
S123992037B11A013733000F37DC277A379DC501DA0037F5317CFC0137351770374C372AD2
S1239940374C37FA317C37F8317AB61437F5317AFC0137351770374C372A374C37FA317AF4
S12399603901317F3A01180C004AF50A27FA17F5100617F51005277A37AC27FA277AF9208E
S1239980B71CF50A27FAF51317FA100037AC27FA17F5319B17FA31723980317F3801180C51
S12399A0B008F50A27FA3902100137AC27FA3F04357E277737F5317837F83176B7743B4096
S12399C0317F007EF50A27FA17F51001277A37AC27FA277AF902B766F50A27FA17F5100579
S12399E0277A37AC27FA277AF920B75237F53176277537B1180D3733000F37DC277A379D7E
S1239A00F50A27FAD50017FA100037AC27FA37F53176FC01373501F4374C372A374C37FA5F
S1239A20317637F83178B616F50A27FA3802100137AC27FAB008F50A27FA3802100137AC62
S1239A4027FA3F04357E27773405274F37F5317C277537B11A013733000F37DC277A379D25
S1239A60C503DA0037F5317CFC0137351770374C372A374C37FA317C37F8317AB61A37F55C
S1239A80317AFC0137351770374C372A374C37FA317A3901317F37B5FFFFB0FE27F5CC007A
S1239AA03F0427F737F5317837F0317637B101F4373501F4374C372A374C27F737F5317608
S1239AC037F0317837B101F3373501F4374C372A374C27F7F50A27FA3802100137AC27FA81
S1239AE037FF3178317627F737F5317C37F0317A37B1177037351770374C372A374C27F72C
S1239B0037F5317A37F0317C37B1176F37351770374C372A374C27F737FF317C317A27F704
S1239B20000000029B9000009B6201F49C063405274FF50F27FA17F5317E277A37AC27FA2C
S1239B40277AF802B60C17F551E7B73AC5033705FA01C22EB030FA009ABC37BD9B20FA02A5
S1239B60E8183B40317F0028F50A27FA17F51005277A37AC27FA277AF920B710F50A27FA07
S1239B80C50317FA100037AC27FACC003F0427F7FA009ABC27F6B66A3A40317F004637F57E
S1239BA03176FC01373501F4374C372A374C37FA31763910317F37F53178277537B1180DE6
S1239BC03733000F37DC277A379DC503DA0037F53178FC01373501F4374C372A374C37FA13
S1239BE03178B0A2F50A27FA17F51001277A37AC27FA277AF902B694F50A27FA3902100132
S1239C0037AC27FAB08637F53178277537B1180D3733000F37DC277A379DC503DA0037F5B9
S1239C203178FC01373501F4374C372A374C37FA31783B40317F0020F50A27FA17F5100150
S1239C40277A37AC27FA277AF902B608F50A27FA3902100137AC27FACC003F0427F7340D23
S1239C60274FF50A27FA17F51001277A37AC27FA277ACA01F50A27FA3802100137AC27FAAD
S1239C80F50A27FA17F51005277A37AC27FA277AF920B7E8F50A27FAC50517FA1000C501B0
S1239CA017FA100137AC27FACC023F0627F7340F274F37450004850627030006B600270375
S1239CC0000437DC277A379DD500CA01B7043705FA009B2EB0D8CC023F0827F7340F274F26
S1239CE037450004850627030006B6002703000437DC277A379DD500CA01B71C3705FA0010
S1239D009B2EC501F80DB600F501B0FE37153716B7CA37B5000AFA009B2EB0C0CC023F08F9
S1239D2027F7340F274F0500C50D010D370527F6B72437450004850627030006B600270314
S1239D40000437DC277A379DD500CA013705FA009B2EC501C100CA00B0CAC5003705CC023A
S1239D603F0827F7340C274F050137F5317C37F8317AB72837F5317A277537B11A0137334C
S1239D80000F37DC277A379DD500CA0137F5317AFC0137351770374C372A374C37FA317A7E
S1239DA0C5013705351827F737F5317837F83176B612F50A27FA17F51005277A37AC27FAD9
S1239DC0277AF660F860B70027F5B00037B5000127F727353196273331882735319837B55B
S1239DE0006437FA319437FA318E37B5000337FA319237B5000137FA319037B5013837FAFD
S1239E00FA2237B5007837FAFA2427F7343F37AF379C27FA2733319A3880F923357E2777BA
S1239E203407274FFA009E7CC80BB5288502CD04379DC50BD100DA00374500028504FA0001
S1239E409E7CC80BB5088502CD04379D17F5319BDA0037B5FFFFB0FE27F5CC003F0627F793
S1239E603407274F17F5319BC00B277A8502CD04379D277ADA00CC003F0627F73407274F62
S1239E8017F5319B3705277A8502CD04379D277AD0007200CC003F0627F7343F37AF379C9F
S1239EA027FA37F53198BF0CFCF637FA319837B8000ABC00FA009FD837F53194BF0CFCF6FD
S1239EC037FA319437B8000ABC00FA00A06227313192BE0837B5000337FA3192FA0089F49C
S1239EE027313190BE0837B5000137FA3190FA00863637F53196FC0A37FA319637B803E81F
S1239F0037850084273531962733318037F53180FCC4B6722735318037F5318637B005A08E
S1239F2037F5318437B20000B40827333186B65627333184B05037F5318637B0100037F565
S1239F40318437B20000B41E37F5318227333182FCF6B6322735318237F53186FC0A37FA9E
S1239F603186B42227333184B01C37F5318227333182FCC4B6102735318237F53186FC3CD9
S1239F8037FA3186B400273331842731318EB600FA009FE2FA00C9FE357E277737F53196C5
S1239FA027F737F5F90A37B10FA037FAF91437F5F9227908B7F42738F922080027F734052F
S1239FC0274F85022701000227F6B702FA009FA2B0ECCC003F0427F737B5FFFF37FA319898
S1239FE027F717F5318CB70A37B5006437FA318E1735318CB00A37B5006437FA318EF5017C
S123A00017FA318C17F5318C3705FA00A01027F727F6B7023980FA11B0003880FA1127F776
S123A02017F5318A17F8318CB71437FE318C318A17F5318CB70237B50001B00037B5FFFF08
S123A04027F727F5B0F617F5318BB7063840FA111735318BB0063940FA11F50117FA318B0F
S123A06027F7FA01C54037B5006437FA319427F753595354454D204953204C4F434B4544E7
S123A0802021000037B5000D3735000334033735000037B5A070FA00C1043F0437B507D0AF
S123A0A037FA319827F74E4F2045444954204D4F4445202100546F206368616E6765207042
S123A0C06172616D6574657273007573652046554C4C204544495400FA00AE7037B50003CB
S123A0E03735000334033735000037B5A0A6FA00C1043F0437B5000D37350003340337350B
S123A100000037B5A0B5FA00C1043F0437B500173735000334033735000037B5A0CAFA0093
S123A120C1043F0437B50BB837FA319827F74E4F2045444954204D4F4445202100546F2000
S123A140726563616C6C2070726F6772616D73007573652046554C4C204544495400FA001D
S123A160AE7037B500033735000334033735000037B5A12EFA00C1043F0437B5000D37359A
S123A180000334033735000037B5A13DFA00C1043F0437B500173735000334033735000034
S123A1A037B5A150FA00C1043F0437B50BB837FA319827F74E4F2045444954204D4F4445CD
S123A1C0202100546F2073746F72652070726F6772616D73007573652046554C4C20454456
S123A1E049540000FA00AE7037B500033735000334033735000037B5A1B4FA00C1043F0462
S123A20037B5000D3735000334033735000037B5A1C3FA00C1043F0437B50017373500036B
S123A22034033735000037B5A1D5FA00C1043F0437B50BB837FA319827F7464143544F528D
S123A2405920505245534554202100546F206564697420636F707920746F00557365722047
S123A2606D656D6F72792066697273740000FA00AE7037B5000337350003340337350000E0
S123A28037B5A23AFA00C1043F0437B5000D3735000334033735000037B5A24BFA00C1044D
S123A2A03F0437B500173735000334033735000037B5A25BFA00C1043F0437B50BB837FA77
S123A2C0319827F7340C274FFA008BA28A0037B80001B60239800053B00038FE00533518F2
S123A2E027F7FA00AE4427F5FA00C25C3735000037B5A558277333D817F5519EB70E17F556
S123A300319CB708FA00A08417F5319CF804B652273531983735000037B5A492277333DC56
S123A3203735000037B5A544277333E017F5319CB71AF801B71EF802B756F803378700965D
S123A340F804378700CAF805378700F01735319CFA00E98A3780010C17F50053B606FA006B
S123A360A15E1735319C27F73735000037B5ED94277333DC3735000037B5ED48277333E0E7
S123A3803735000037B5EE5A277333D8FA00E9EA378000D017F50053B606FA00A0D8173547
S123A3A0319CB0BE3735000137B5405C277333DC17F50053B7083735000137B52EB42773CD
S123A3C033E03735000137B540CC277333D827F5FA0120203780008C17F50053B606FA00AD
S123A3E0A1E41735319C27F73735000037B5E682277333DC3735000037B5E588277333E0C2
S123A4003735000037B5E770277333D8FA00E26AB0503735000137B560B0277333DC373520
S123A420000137B5605A277333E03735000137B56172277333D827F5FA015FD8B024373565
S123A440000137B5CAFC277333DC3735000137B5CAFA277333E03735000137B5CB162773FE
S123A46033D8FA01C70427F700100001A4ACA4C6A4CAA4CAA4E6A4CCA502A4A0A51AA51ADF
S123A480A51AA51AA51CA526A530A53A00000000A4A027F6378700A837BDA468FA02E81837
S123A4A01735319CFA00A2E23780009417F5319CF802B6021735319CB002F50217FA319C8B
S123A4C0FA00A2E2B078FA00E98AB07217F5319CF803B6021735319CB002F50317FA319C16
S123A4E0FA00A2E2B05817F5319CF804B604F50A17FA319CB002F50417FA319CFA00A2E25F
S123A500B03C17F5319CF801B6021735319CB002F50117FA319CFA00A2E2B02237B50001E5
S123A520FA020C0AB01837B50002FA020C0AB00E37B50003FA020C0AB00437B50004FA02DE
S123A5400C0A27F727F700000003A5A40000A5A60001A5AEFFFFA5B237F5319837B8FFFF83
S123A560BE08273531981735319CFA00A2E217F55172B71A37F53198B61417F551721733DD
S123A5805172370537B80003BD04FA00E98A1735517217F533E4B716FA00A02037BDA54600
S123A5A0FA02E818B00827F5FA0204ACB000FA00E98A27F7596F757220626F6F746C6F6121
S123A5C064657220646F6573006E6F7420737570706F72742052533438352021004544496A
S123A5E0542020203D20757064617465004F5054494F4E203D2061626F72740020202020D5
S123A600596F75206D757374206E6F742020202020002020737769746368206F6666205062
S123A6204F57455220212000506C65617365207761697420756E74696C2020202000757098
S123A640646174652069732072656164792E2E2E202120004E6F20726573657420616674E1
S123A660657220706174636821005570646174696E6720626F6F746C6F6164657200557062
S123A680646174656420746F2056322E3020210034043FEC274FF50027FA37F53FFE277A71
S123A6A037AC27FA277A8A1227F58A0E37B13FFC8A1027F58A0A37B13FFA8A0C270500024F
S123A6C02705000427050000850ACD0C379D950037B1FE003787024E850ECD10379D95007C
S123A6E0FC0137860180851237B1475AB60827F58A0237B106548A04B014851237B85EF924
S123A700B70237B80EE5B60627F58A0237B106768A04850487023787020CFA00AE7027F532
S123A720340134013735000037B5A5B4FA00C1043F0437B50008340127F534013735000012
S123A74037B5A5C9FA00C1043F0437B500103735001434033735000037B5A5DDFA00C1044D
S123A7603F0437B500183735001434033735000037B5A5EDFA00C1043F04FA02194C37B89B
S123A7800001378600D4FA00AE7037B50010FA00C25C27F53735000134033735000037B5DF
S123A7A0A5FCFA00C1043F0437B500083735000234033735000037B5A612FA00C1043F0447
S123A7C037B500103735000234033735000037B5A628FA00C1043F0437B50018373500023A
S123A7E034033735000037B5A63EFA00C1043F0427F5FA00C25CFA02000037B504B0FA0016
S123A8009FBEFA020000373B00E037B50001275C340937AD3401374500028504FA01CE985B
S123A8203F0637B507FF8A0037B50001275C340937AD34013745000E8510FA01CE983F06C8
S123A840373AFF1F37B50BB8FA009FBE3735000037B5A654FA017268378000CAFA020000BB
S123A860FA00B944378000BE37F5FB007908378600B4FA00AE4427F5FA00C25C37B5000A39
S123A8803735000134033735000037B5A66AFA00C1043F04373B00E037B500048A0627F5B8
S123A8A08A0837B1800037FAFB008506277537FAFB04850837FAFB0637B50001FA01D0CCD4
S123A8C037B52000340127F53735000334032775FA01CE983F06270500062705000885063E
S123A8E0277537FAFB04850837FAFB0637B5080037FAFB00373AFF1FFA02000037B500141E
S123A9003735000834033735000037B5A67EFA00C1043F0437B503E8FA009FBEFA020000E0
S123A920FA00B944FA020000CC143F1627F7340C274F27050000FA020000FA007FCEFA00AE
S123A940C37EFA008186FA00ADCEFA009568FA00C28AFA020000FA00B944FA020000F5011A
S123A96017FA1002373AFF1FFA006FFEFA009DD2FA008D6A37B50001FA0200A2FA020000D9
S123A98017F5519EB600FA024744FA00A2C4FA02000017F5317EF802B600FA00A690FA008A
S123A9A0E15AFA01262C27F5FA00EC72FA020AF2FA02038EFA014C9AFA02000037B502BC8B
S123A9C0FA009FBEFA02000037B502BCFA009FBEFA02000037B502BCFA009FBEFA02000026
S123A9E017351002FA00A2E2FA020B12FA008B7427F6B6F437B50064FA009FBE37B500010A
S123AA00FA020024FA00C9A2FA0047BAFA020000FA00CA14270300008500760727F6B6E8F7
S123AA20F50F27FA37B5432137FA000637AC27FAFA00A046B0D2007A002000000000000066
S123AA40000000000000000000007FFFFFFFFFC0000000000000000000007FFFFF07FFC074
S123AA60000000000000000000007FFFFF03FFC0000000000000000000007FFFFF03FFC054
S123AA80000000000000000000007FFFFF01FFC00FFE0780F003E007C0007FFFFF01FFC00A
S123AAA00FFF83C1E00FF81FF00070003F00FFC00FFFC1E1E01FFC3FF80070003F08FFC084
S123AAC00FFFE0F3C01E3E7C7C0070003F087FC00783F07BC03C1E783C0070003F0C7FC0CA
S123AAE00780F83F803C1E783C0070FFFF0C3FC00780781F80001E783C0070FFFF0E3FC0A2
S123AB0007C0780F00001E783C0070FFFF0E1FC007C03C1F80003C3C780070FFFF0F1FC0C8
S123AB2003C03C1FC001F81FF00070FFFF0F0FC003C03C3DE001F00FE00070003C0F8FC0D9
S123AB4003C03C3CF001F81FF00070003C0F87C003C03C787800783C780070003C0FC7C05F
S123AB6003E03C783C003C783C0070003C0FC3C001E07CF01E003C783C0070FFFFFFE3C065
S123AB8001E0F800003C3C783C0070FFFFFFE1C001FFF800003E7C7C7C0070FFFFFFF1C0D6
S123ABA001FFF000001FF83FF80070FFFFFFF0C001FFE000000FF01FF00070FFFFFFFFC01C
S123ABC001FFC0000007E00FE00070003FFFFFC00000000000000000000070003FFFFFC001
S123ABE00000000000000000000070003FFFFFC00000000000000000000070003FFFFFC077
S123AC00000000000000000000007FFFFFFFFFC0000000000000000000007FFFFFFFFFC0BA
S123AC200000000000000000000000000000000000000000000000000000009C0014FFFE63
S123AC4000FFFF803C01FFFF007803FFFE00F007FFF0FFFF01FFFFC07E03FFFF80FC07FF1B
S123AC60FF01F80FFFF0FFFDFF7FFB7FFFFEFFF7FFB7FDFFEDFF7FFBFFF0FFFCFE7FF33F42
S123AC80FFFCFFE7FF33F9FFCCFE7FF3FFF0FFFCFE7FF33FFFFCFFE7FF33F9FFCCFE7FF389
S123ACA0FFF0FFFCFE7FF33FFFFCFFE7FF33F9FFCCFE7FF3F1F0FFFCFE7FF33FFFFCFFE744
S123ACC0FF33F9FFCCFE7FF3F1F0FFFCFE7FF33FFFFCFFE7FF33F9FFCCFE7FF3F1F0FFFD5B
S123ACE0FF7FFB7FFFFEFFF7FFB7FDFFEDFF7FFBFFF0FFFFFFFFFFC07E03F01F80FC07FF91
S123AD00FF01F80FFFF0FFFFFFFFFFE0FF07F83FC1FE0FFFFF83FC1FFFF0FFFDFF7FFBFF54
S123AD20DFFEDFF6FFF7FFFFEDFF6FFBFFF0FFFCFE7FF3FF9FFCCFE67FF3FFFFCCFE67F3D6
S123AD40F1F0FFFCFE7FF3FF9FFCCFE67FF3FFFFCCFE67F3F1F0FFFCFE7FF3FF9FFCCFE625
S123AD607FF3FFFFCCFE67F3F1F0FFFCFE7FF3FF9FFCCFE67FF3FFFFCCFE67F3FFF0FFFC22
S123AD80FE7FF3FF9FFCCFE67FF3FFFFCCFE67F3FFF0FFFDFF7FFBFFDFFEDFF6FFF7FFFF53
S123ADA0EDFF6FFBFFF0FFFF01FFFFC07E03FFFF80FC07E03F01F80FFFF0FFFE00FFFF80FA
S123ADC03C01FFFF007803C01E00F007FFF0F50C27FAF5E217FA0004F5A417FA0004F5AF95
S123ADE017FA0004F5A017FA0004F5A917FA0004F5E217FA0002F5A417FA0002F5AF17FA92
S123AE000002F5A017FA0002F5A917FA000237AC27FAFA00AE4417F5338827F8FA00AE2233
S123AE2027F73405274F75053724F14A17FAF926C50317FA3388CC003F0427F717F5338879
S123AE4027F827F7340C274F27050000850037B801E8BC10F50F37BD31A0379D850037DD70
S123AE60150027030000B0E0FA00AF70351827F7340C274F27050000850037B801E8BC1070
S123AE80F50F37BD31A0379D850037DD150027030000B0E0351827F7340D274F270500005B
S123AEA037450000373801E8BC0EF50F37BD31A0379DC50527DA27030000B0E0FA00AF70B5
S123AEC0CC023F0627F73405274F850827FD27FD27FD3735007A372681028A02C509F60778
S123AEE037058A088502BD2237B1FE18BC1CF5014509B70237143701B6F6277AF50F37BD7F
S123AF0031A0379D277A3745000227D727DACC003F0427F73405274F850827FD27FD27FD95
S123AF203735007A372681028A02C509F60737058A088502BD2437B1FE18BC1EF50145099E
S123AF40B70237143701B6F63710277AF50F37BD31A0379D277A3745000227D627DACC0097
S123AF603F0427F717FA319FB600FA00AF7027F734043FF8274F17F5319FB702CC083F0A07
S123AF8027F72705000427050002850437B80004BC6AC505F1B8277AF50C27FA277A17FAA7
S123AFA00004C505F1B817FA0002173500041735000237AC27FA27050006850637B8003D78
S123AFC0BC2E81028A00F50F37BD31A0379D37450000F50C27FA27D517FA000537BD31DD27
S123AFE03745000027D517FA000337AC27FA27030006B0C2270300048502FC7A8A02B0862E
S123B000CC083F0A27F73405274F850827FD27FD27FD3735007A372681028A0227080008C0
S123B020FFF88502BD4A37B1FE18BC44C50BB71EF5014509B70237143701B6F6277AF50F13
S123B04037BD31A0379D277A3745000227D727DAB01EF5014509B70237143701B6F63710F4
S123B060277AF50F37BD31A0379D277A3745000227D627DACC003F0427F7340D274F37B5A1
S123B08000018A00C50537058800BF3C27F537BD007934098500FCFF340127F5FA00B358FC
S123B0A03F06C501F1C0277AF50C27FA277A17FA0004C501F1C017FA000237AC27FA37B5DD
S123B0C0000AFA009FBE27030000B0B4FA00AE44F5C0277AF50C27FA277A17FA0004F5C0AE
S123B0E017FA000237AC27FACC023F0627F734053FF0274FC5193705F607B66EC51DFC010C
S123B1003705F607B6642705000CC51D3705C0197200FC0137350008FA02E7B4880C378FD5
S123B120022EC51337058A0AC51B3705FC01880ABF32F50F37BD31A0379D850C3735007A83
S123B1403726810A37DDF50F37BE31A0379E850C3735007A3726277B3741000A27E5371005
S123B160DA002703000AB0BC2703000CB098F5FFCA09CA08C51DF806B30EC519F108370586
S123B180F607B73A04093711B6F6B032C51D3705FC0137350008FA02E7B427F427F427F463
S123B1A08A04C51D3705FC0180048A0237B5000880028A00C5094501B702371F3701B6F6CB
S123B1C0CA09C51D3705FC083705F607FC018A0437B5000880048A02C5084503B702371F8A
S123B1E03701B6F6CA08C51337058A0CC51B3705FC01880CBF5AF50F37BD31A0379DC519AA
S123B200370537350008FA02E7B43735007A3726277B3741000C27D5CA06C609CA073710C7
S123B220C609CA07F50F37BD31A0379DC519370537350008FA02E7B43735007A3726277BC3
S123B2403741000CC5093710C606C70727DA2703000CB094C51D370537350008FA02E7B413
S123B2608A04C519370537350008FA02E7B48004B70237B50001B0FE27F5CA02C51D370539
S123B280C019720037B80007BF00F501B0FE3715C702378700BAC51337058A0CC51B3705B3
S123B2A0FC01880CBF5AF50F37BD31A0379DC51D370537350008FA02E7B43735007A3726D7
S123B2C0277B3741000C27D5CA06C608CA073710C608CA07F50F37BD31A0379DC51D370538
S123B2E037350008FA02E7B43735007A3726277B3741000CC5083710C606C70727DA2703FD
S123B300000CB094C5193705F6078A04C519FC0880048A02C51D3705F6078A00C51D80003B
S123B3208802B72AC51D3705F6078A04C51D8004FC013401C51B37053401C519F6078A02A5
S123B340C519FC0880023401C5133705FA00B0EE3F06CC103F1427F734053FFA274F850E97
S123B360FCE0BC5C851080088A04BC0885108A0085088A1085008A08C513B61C85088A0246
S123B38085028810BE36FC86BC08850E34018502FA00AF143F0227030002B0E085088A022E
S123B3A085028810BE16FC86BC08850E34018502FA00AEC63F02C513370581028A02B0DCA3
S123B3C0FA00AF70CC063F0A27F734053FFA274F37B8007ABC5C8510800E8A04BC088510A4
S123B3E08A00850E8A1085008A0EC513B61C850E8A0285028810BE3637B80020BC06340193
S123B4008508FA00AF143F0227030002B0E0850E8A0285028810BE1637B80020BC063401C9
S123B4208508FA00AEC63F02C513370581028A02B0DCFA00AF70CC063F0A27F734053FF261
S123B440274F851A80168A04851880108A068504BAFE27F28A008506BAFE27F28800378D66
S123B46000908506BC1C85188A0885108A1885088A1027020006851A8A0885168A1A85081C
S123B4808A16270200044505371537450006FA02E7B48A08C51DB60437B500018A02B002D3
S123B4A0C51D37058A022705000C850C8806378E00D03745000837268A0ABD0437B1008054
S123B4C08A0AB002850AFC808A0A850A37350100FA02E7B48A0AC51D370534018516810AE3
S123B4E03401850C8110FA00B0063F048502810C8A0CB0B28504BC1C851A8A0885168A1A21
S123B50085088A162702000485188A0885108A1885088A10270200064507371537450004F9
S123B520FA02E7B48A08C51DB60437B500018A02B002C51D37058A022705000A850A88041C
S123B540BE3E3745000837268A0CBD0437B100808A0CB002850CFC808A0C850C3735010062
S123B560FA02E7B48A0CC51D370534018516810A3401850C8110FA00B0063F048502810AC5
S123B5808A0AB0B4FA00AF70CC0E3F1227F7340D274F1733319FC5133705CD0ECE0A341968
S123B5A08504FA00B3CA3F06C5133705CD0CCE0A34198504FA00B3583F06C5133705CD0E6E
S123B5C0CE0A3419850CFA00B3CA3F06C51337053401850CFCFFCD0E34098504FA00B3587A
S123B5E03F06CB021132C51337053401850CFC013401850EFC0134018504FC01FA00B35896
S123B6003F06C5133705CD0E3409850AFC013401850CFC01FA00B3CA3F06CB041126850A15
S123B620FC018A00CD004D0EBC1837B500013401850CFCFF34098504FC01FA00B3583F06C8
S123B64027030000B0DA1731319FFA00AF70CC023F0627F7340D274F1733319F850A8A00E6
S123B6608500880EBE1227F5CD0CCE0034198504FA00B3583F0627030000B0E01731319F26
S123B680FA00AF70CC023F0627F734073FEC274F374A00108A02374A0000FC028A12B40094
S123B6A0270300108500CD02379D95008A0C3745001085128A02374A0000FC028A12B4007B
S123B6C0270300108500CD02379D95008A0A8120FCFF8A0485048820378D009037B58000C0
S123B6E08A08851E8A0E851E810C880EB34A8510CD12379D95008608B71685043401850E2D
S123B700FA00AF143F02B01427010004B0C22703000EB0CE85043401850EFA00AEC63F020F
S123B720270F00088508B6E28512FC028A12B4002703001037B580008A08B0CE850C37350A
S123B7400020374C372A374C8A06B7088512FC028A12B40027030010850637B80010B4A40E
S123B7608512FC028A12B49C27030010B096FA00AF70CC143F1A27F734073FE8274F374AFB
S123B78000148A02374A0000FC028A16B400270300148500CD02379D95008A0E374500140F
S123B7A085168A02374A0000FC028A16B400270300148500CD02379D95008A0C852627F236
S123B7C081228A08852827F281248A06850CFCFF8A048504378D00CA8828BD768528812CC7
S123B7E08804BF6E37B580008A12270500108510880EB4788826B53E8526812A8810B33679
S123B8008514CD16379D95008612B71A85048106340185108108FA00AF143F02B018270185
S123B8200004B0AA27030010B0C085048106340185108108FA00AEC63F02270F001285120B
S123B840B6DE8516FC028A16B4002703001437B580008A12B0CA850E27FF27FF27FF27FF78
S123B86027F427758116374300148A16374A0014850E37350020374C372A374C8A0AB708DA
S123B8808516FC028A16B40027030014850A37B80010B4868516FC028A16B4002703001486
S123B8A03780FF78FA00AF70CC183F1E27F73405274F37B500143735000D340327F534012E
S123B8C0C50337053735000AFA02E7B43735000D3726FC0D3745000ACD08340B373500006E
S123B8E037B5AC3AFA00B7783F0C37B500143735000D340327F53401C50337053735000A83
S123B900FA02E7C83735000D3726FC0D3745000A34038508FC0D34013735000037B5AC3AD3
S123B920FA00B778CC003F1027F7FA00AE4427F5340134013735000037B5AA36FA00B68ABD
S123B9403F0427F7FA00AE44FA02000027F5340134013735000037B5AA36FA00B68A3F045F
S123B96027F7000000000004040400040A0A0000000A1F0A1F0A02060E06021102040811D7
S123B980080C0E0C08040400000004080808040804040408000A040A0000040E04000000FB
S123B9A000040400000E00000000000C0C01020408100E1315190E040C0404041E010E1080
S123B9C01F0E010E010E12121F02021F101E011E0F101E110E1F010204080E110E110E0E81
S123B9E0110F010E000400040000040004040204080402000E000E0008040204080E0204A2
S123BA0000041F1F1F1F1F0E111F11111E111E111E0F1010100F1E1111111E1F101E101F6E
S123BA201F101E10100F1013110F11111F11110E0404040E070202120C1112141A1110100D
S123BA4010101F111B15151111191513110E1111110E1E111E10100E1115120D1E111E126B
S123BA60110F100E011E1F04040404111111110E1111110A04111515150A110A040A1111FE
S123BA800A0404041F0204081F1A15151111000000000000000004040400000400000A0AB6
S123BAA00000000000000A0A1F0A1F0A0A00040F140E051E040018190204081313000C1233
S123BAC0140815120D000C04080000000000020408080804020008040202020408000004B4
S123BAE0150E150400000004041F04040000000000000C0408000000001F000000000000A0
S123BB000000000C0C0000010204081000000E11131519110E00040C040404040E000E111E
S123BB20010204081F001F02040201110E0002060A121F0202001F101E0101110E000608C9
S123BB40101E11110E001F010204040404000E11110E11110E000E11110F01020C00000C89
S123BB600C000C0C0000000C0C000C040800020408100804020000001F001F0000000804F7
S123BB800201020408000E1101020400040000000000000015000E1111111F1111001E11A0
S123BBA0111E11111E000E11101010110E001E11111111111E001F10101F10101F001F1047
S123BBC0101E101010000E11101311110F001111111F111111000E04040404040E000702D2
S123BBE0020202120C0011121418141211001010101010101F00111B15151111110011116D
S123BC001915131111000E11111111110E001E11111E101010000E11111115120D001E111A
S123BC20111E141211000E11100E01110E001F040404040404001111111111110E00111170
S123BC401111110A040011111115151B110011110A040A1111001111110A040404001F0151
S123BC60020408101F000E08080808080E0000100804020100000E02020202020E00040AEC
S123BC801100000000000000000000001F00100804000000000000000E010F110F001010F6
S123BCA0161911111E0000000E1010110E0001010D1311110F0000000E111F100E00060906
S123BCC0081C0808080000000D13130D010E101016191111110004000C0404040E00020027
S123BCE006020202120C0808090A0C0A09000C04040404040E0000001A1515111100000040
S123BD0016191111110000000E1111110E00000016191119161000000D1311130D0100009D
S123BD2016191010100000000E101E011E0004040E04040406000000121212120D000000C8
S123BD401111110A04000000111115150A000000110A040A110000001111130D010E0000BD
S123BD601F0204081F00020404080404020004040400040404000804040204040800081500
S123BD8002000000000000000102140808000000121212121D100814140800000000340590
S123BDA03FF4274F3A10319E0004050AB000F501CA0A27050008850837B80005B468F5006A
S123BDC037BDB962379D373DFF60C50F75053724277B3741000827D5CA0B851681088A005F
S123BDE085148A028514FC058802B312CB100B16C50A3705CD0034098502FA00B0063F04A6
S123BE00B01C27030008B0AAC50AB602F5013705B00037153705CD0034098502FA00B00694
S123BE203F04040B27030002B0B6CC0C3F1027F734073FE8274F3A10319E00040514B00017
S123BE40F501CA1485228A082705000A850A37B80050378401143745001A851C2703001C80
S123BE60B6002703001A37DC277A379DD500CA16B606378000F42703000AB0CCF50037BD87
S123BE80B962379D373DFF60370537AD8A008D02C5167505372427753706BAFE2770810248
S123BEA0374300008A12374A00102705000E850E37B80005B466374500108512270300129D
S123BEC0B6002703001037DC277A379DD500CA178524810E8A0485088A068508FC05880631
S123BEE0BF12CB101716C5143705CD0434098506FA00B0063F04B01C2703000EB0ACC5148B
S123BF00B602F5013705B00037153705CD0434098506FA00B0063F04041727030006B0B6BE
S123BF20C514B602F5013705B0003715370534018524FC04CD2434098508FC05FA00B3CAF1
S123BF403F068508FC068A0817F5319EF60FF8033786FF20C516F820B706F83AB702F82EFF
S123BF603786FF10270100083780FF08C514B602F5013705B0003715370537BD00013409D6
S123BF808524FC05CD0834098524FCFF34018522FCFFFA00B58E3F0AFA00AF70CC183F1E86
S123BFA027F734053FF4274F3A10319E0004050AB000F501CA0A27050008850837B800081F
S123BFC0B46CF50037BDBA8E379D373DFF00C50F3705277B2774277427743741000827D5C6
S123BFE0CA0B851681088A0085148A028514FC058802B312CB100B16C50A3705CD0034099B
S123C0008502FA00B0063F04B01C27030008B0A6C50AB602F5013705B00037153705CD0090
S123C02034098502FA00B0063F04040B27030002B0B6CC0C3F1027F700070001C08EC08ABF
S123C040C0DEC076C0FCC0D4C07C00000000C0FC34073FFC274F37DC277A379DD500CA03AA
S123C06037B500068A0017F5319E3705F60F37BDC038FA02E81827030000B07C27010000BE
S123C080C503F820B6002701000027030000C503F820B718F83AB714F82EB710F869B70CF7
S123C0A0F86CB708F874B704F831B700F86AB600270100008506CD08379DD501CA03F869DA
S123C0C0B708F86CB704F874B700F86BB62A27010000B024C503F820B60027030000C50394
S123C0E0F820B710F83AB70CF82EB708F869B704F86CB700F874B600270100008500CC04AD
S123C1003F0A27F734073FF4274F1733319F3A10319E0006F501CA05B0FE05053745000E90
S123C1208510FA02E4B68A08850ECD10379DD500CA0305048516FCFA8A00275C3D0337AD8D
S123C1403705277B37DCFA00C05081008A0A270500063745000637480008378C00848518AC
S123C160CD0A3409850ECD10379D27D53705FA00BFA23F048508FCFF8806BF36C50537057C
S123C18034018518FC07CD183409850AFC05FA00B3CA3F0617F5319EF60FF802B514C505EB
S123C1A0370534018518FC07CD183409850AFC06FA00B3CA3F068508FCFF8806B604850A9C
S123C1C0FC058A0AB01227758506BAFE277081103743000EFA00C050810A8A0A270300061C
S123C1E03780FF6CC505370537BD000134098518FC08CD0A34098518FCFF34018516FCFFC9
S123C200FA00B58E3F0A1731319FFA00AF70CC0C3F1227F734073FFA274FFA02E4B68A0012
S123C22037450008850AFA00C050FCFA8A042705000285028800BC1827758502BAFE2770D6
S123C240810A37430008FA00C05081048A0427030002B0DA8504CC063F0C27F717FA319E56
S123C26027F7F50A27FA17F51001277A37AC27FA277AF888B604F50117FA3393B000173516
S123C280339317F53393370527F7FA00C26227F7F50A27FA17F51000277A37AC27FA277AEA
S123C2A0370527F7340C274F37B50001FA02004EF501CA01C501F804B2063705FA020BCEE7
S123C2C00301B0EC351827F7340C274FF501CA01C501F804B2063705FA020B7E0301B0ECFD
S123C2E027F5FA02004E351827F734043FFC274F17F53393B77EF50A27FA17F51000277A9C
S123C30037AC27FA277A17F8338AB768F50A27FA17F51000277A37AC27FA277A17FA338A39
S123C320F8FFB7503710CA010502F501CA03C503B706C601B60204030302B0EEF50F37BD79
S123C340338B379DC5023705277B27D5F850B220C502277B27D5B71CC502277B27D537FABE
S123C3600048FA00EC7237F50048FA01B7CAFA00C2C8B000FA00C2A4CC043F0627F7FA0068
S123C3807FFA3735000B27F5277333A03735000037B5C856277333A837F533A817FD33AA3D
S123C3A0379D9502378700B637FA3396277537F133A2377333A0FC023733000037B020001B
S123C3C03732000BB5FEB0FA37F533A817FD33AA379D950027757C0F277333A4277133A024
S123C3E0FC02373300002773339C37B5038F37FA339437F53396FA00C61C37F533A017FD0E
S123C40033A2379D950037F83394B62037F533A817FD33AA379D95023401277133A0FC020D
S123C420373300003403277133A4FA02E45C3F0637F533A817FD33AA379D9502FC0227756A
S123C44037F133A2377333A0277333A037F533AAFC0437FA33AAB400273333A83780FF3605
S123C46027F700000002C5B20001C5B80002C5BE17F533ACF8013787008CF802378700AC8C
S123C480F803378700BEF8043787010CF8053787012CF8063787015037F533A817FD33AA6D
S123C4A0379D9502B71CFC02277537F133A2377333A0277333A037F533AAFC0437FA33AAA2
S123C4C0B400273333A837F533A817FD33AA379D9502B6123735000B27F5277333A03735D8
S123C4E0000037B5C856277333A837F533A817FD33AA379D950027757C0F277333A4F501CA
S123C50017FA33AC3780011037F533A817FD33AA379D950237FA3396277133A42773339C2A
S123C52037B5038F37FA3394F50217FA33AC37B50064FA00C61C27F6378700DCF50317FAAE
S123C54033AC378000D2FA007FEA27F6378700C837F533A017FD33A2379D950037F8339422
S123C560B62CF50417FA33AC37F533A817FD33AA379D950237FA3396277133A42773339CB7
S123C580277133A0FC02373300002773339837800086F50517FA33ACB07CFA007FEA27F68C
S123C5A0B77437B50064FA00C67A37BDC462FA02E818173533ACB05EF50517FA33ACB05683
S123C5C0FA007FEA27F6B74E37B5000234013735000F37B533943403277133A0FA00807AEB
S123C5E03F06F50617FA33ACB02CFA007FEA27F6B72437F533A817FD33AA379D9502340138
S123C600277133A43403277133A0FC0237330000FA00807A3F06173533AC27F73405274F6C
S123C62085022701000227F6B73837F53396B7322731339637F5339C17FD339E379DF50F82
S123C64027FAD50017F1339417FA3394D50017F4339517FA339537AC27FA2733339EB6BC17
S123C6602733339CB0B637F53396B60237B50001B0FE27F5CC003F0427F7340D274F37F8B0
S123C6803396B30237F533968A04850434012771339834032771339CFA02E05C3F068A00CF
S123C6A037F53396800437FA33968504277537F1339E3773339C2773339C8504277537F1B6
S123C6C0339A37733398277333988500B70237B50002B00E37F53396B60237B50001B0FE7D
S123C6E027F53705F601CC023F0627F73735000B27F5277333A03735000037B5C8562773A6
S123C70033A837F533A817FD33AA379D9502B76637F533A017FD33A2379D950037FA339471
S123C720F50F27FAF50117F4339417FA339437AC27FA37B5000234013735000F37B53394DB
S123C7403403277133A0FA00807A3F0637F533A817FD33AA379D9502FC02277537F133A200
S123C760377333A0277333A037F533AAFC0437FA33AAB400273333A8B084FA007FFA27F706
S123C780340C274F3735000B27F5277333A03735000037B5C856277333A827050000850043
S123C7A0FCFABC2E37F533A817FD33AA379D9502FC02277537F133A2377333A0277333A0B1
S123C7C037F533AAFC0437FA33AAB400273333A827030000B0C437F533A817FD33AA379DEB
S123C7E09502B76637F533A017FD33A2379D950037FA3394F50F27FAF50117F4339417FA3A
S123C800339437AC27FA37B5000234013735000F37B533943403277133A0FA00807A3F061D
S123C82037F533A817FD33AA379D9502FC02277537F133A2377333A0277333A037F533AA07
S123C840FC0437FA33AAB400273333A8B084FA007FFA351827F73188000231840004519E68
S123C8600001002000010010000851A00002338800010FA200015954000134E000E435C47A
S123C88000E436A800E4378C00E4387000E4395400E43A3800E43B1C00E43C0000E43CE479
S123C8A000E43DC800E43EAC00E43F9000E4407400E4415800E4423C00E4432000E4440420
S123C8C000E444E800E445CC00E446B000E4479400E4487800E4495C00E44A4000E44B24C8
S123C8E000E44C0800E44CEC00E44DD000E44EB400E4004A000200520001005300010024FE
S123C900000110040001533C000101940001533D0001338B0008019A0002019C00024F985D
S123C9200001019E000901A70009004C0001000000000000C96206000000C97A07000000D1
S123C940963C120000008EB00E000000C47003000000C2EA02000001B86401000000C99245
S123C9600100FA008B74277A37F533DC17FD33DE379D277AFA02E53227F7FA008C46277AA5
S123C98037F533E017FD33E2379D277AFA02E53227F737F533D817FD33DA379DFA02E53246
S123C9A027F7340C274F37B500088A0085002701000027F6B72C8500277537B133CE373300
S123C9C0000F37DC277A379D8500373500063726277537B1C9363733000037EC277A379EE2
S123C9E0E500DA00B0C2F50F37BD33BE379D37F533D627F437DD27150000351827F7F50F36
S123CA0037BD33AE379D37F533D627F437DD2713000027F734043FF2274F05052705000A8E
S123CA203735000F37B533CE8A08374A00062705000C850C37B80008B4268506CD08379DA3
S123CA40D500C805B302CA05850C8A0A8506CD08379D13002703000C27030008B6D0270328
S123CA600006B0CAC505B75C850A37FA33D637350006372627753706BAFE277037B1C932B2
S123CA80373300008A02374A00008500CD02379DD504277AF50F37BD33CE379D277A37755F
S123CAA033D627DA8500CD02379D9500DD02379DFA02E532F50F37BD33BE379D37F533D6F3
S123CAC027F437DD27130000CC0E3F1027F728206672656520636F6E666967202920002891
S123CAE02032696E342046756C6C2029002820342D57617920290028332D57617920496E26
S123CB0064705375622B46756C6C290028332D576179204D6F6E6F5375622B46756C6C29A9
S123CB20002820332D576179202B2046756C6C20290028322D576179204D6F6E6F53756236
S123CB402B46756C6C29002820322D57617920290020303132333435363738394161426256
S123CB6043634464456546664767486849694A6A4B6B4C6C4D6D4E6E4F6F50705171527261
S123CB8053735474557556765777587859795A7A2122232425262728292A2B2C2D2E2F3A97
S123CBA03B3C3D3E3F405B5D5E5F607B7C7D7E7F8081C316000040000000473B80003F005F
S123CBC0000041200000340F274F8504CD06379D17F533FBDA003735000F37B533EA340338
S123CBE0374500048506FC0137330000FA02E0D03F04270500003745000037380004378CF2
S123CC000122F50F37BD578C379D27D5277A8504CD06379D277A37450000375DDA16F500DB
S123CC2027FAF50F37BD595A379D27742774375D3755000095023778CBB2B60037F8CBB4D3
S123CC4037DC37AC27FA37DCB60E8504CD06379DF58137450000375DDA1AB034F50F37BD5C
S123CC60595A379D850027F427F437DD37550000F500379E950237BECBB6FA02E6BAFA025F
S123CC80E740277A8504CD06379D277A37450000375DDA1AF50F37BD5955379D37450000FD
S123CCA027D5277A8504CD06379D277A37450000375DDA1EF50F37BD579C379D850027F49B
S123CCC027F437DD37550000F500379E950237BECBBAFA02E6BA37ECF500379E37EC37BE19
S123CCE0CBBEFA02E620FA02E740277A8504CD06379D277A374500002774375D9A22F50FA5
S123CD0037BD516E379D3745000027D5277A8504CD06379D277A37450000375DDA12270378
S123CD2000003780FECE27050000850037B80003BC4CF50F37BD5790379D850027F427F453
S123CD4037DD37550000F500379E950237BECBBAFA02E6BA37ECF500379E37EC37BECBBE2A
S123CD60FA02E620FA02E740277A8504CD06379D277A374500002774375D9A2A270300007F
S123CD80B0A48504CD06379D17F55174DA3017F55173DA312771004EFA02E740277A850422
S123CDA0CD06379D277ADA3227050000850037B80004378C008E373500063726277537067E
S123CDC0BAFE277037B151863733000F37DC277A379D850037350006372627753706BAFE5B
S123CDE02770810637430004FC343733000037EC277A379EF506FA02E916850027F427F4AF
S123CE0027753706BAFE277037B151763733000F37DC277A379D850027F427F427753706A2
S123CE20BAFE2770810637430004FC4C3733000037EC277A379E9500AA009502AA022703A3
S123CE4000003780FF6427050000850037B80008BC5EF50F37BD57AC379D8500373500062C
S123CE603726277B27D5277A8504CD06379D277A3745000027742774375DDA5CF50F37BDCD
S123CE8057AE379D850037350006372637DD375500009502FA02E740277A8504CD06379D36
S123CEA0277A3745000027742774375D9A5E27030000B09227050000850037B8001A378CA6
S123CEC001ACF50F37BD57DC379D85003735000E3726277B27D53714371437143714371431
S123CEE0277A8504CD06379D277A3745000027742774375DDA7C8504CD06379D3745000074
S123CF0027742774375DF50F37BE57E6379E85003735000E372637ED37650000A502FA0279
S123CF20E740F61FD17CDA7CF50F37BD57DC379D85003735000E372637DD37550006F50018
S123CF40379E950837BECBC2FA02E6BA37ECF500379E37EC37BECBBEFA02E620FA02E7408A
S123CF60277A8504CD06379D277A3745000027742774375DDA7DF50F37BD57DC379D85001A
S123CF803735000E3726277B27D5F807B40EFA02E800CFA2CFE2CFB8CFB8CFE4CFE4D00EFF
S123CFA08504CD06379DF5073745000027742774375DDA7DB07CF50F37BD57DD379D8500F3
S123CFC03735000E3726277B27D5277A8504CD06379D277A3745000027742774375DDA7DC9
S123CFE0B050F50F37BD57DD379D85003735000E3726277B27D5F806B6388504CD06379D17
S123D000850027F427F437DD157DB026F50F37BD57DD379D85003735000E3726277B27D5DB
S123D020F80CB60E8504CD06379D850027F427F437DD1719807DF50F37BD57DE379D850072
S123D0403735000E372637DD375500009502FA02E740277A8504CD06379D277A37450000AD
S123D06027742774375D9A7E270300003780FE46CC023F0827F73F333333340F274F850C50
S123D080CD0E379DD500CA01370527FD27FD27FD27FD27FD277A8504CD06379D277ADA0001
S123D0A01708E001CB1001021709F001C50127F8FA02E7DA34018504CD06379D35409A0C5B
S123D0C0375A000A850CCD0E379DD5013705FA02E7DA37ECF500379E37EC37BECBC2FA0214
S123D0E0E95034018504CD06379D35409A08375A0006F506DA01D500F802B710F803B70CB6
S123D100F804B738F805B734F806B768378000B6850CCD0E379DD501277A8504CD06379DC7
S123D120277ADA01F50027FA2771D07637DC37AC27FA37DCCD069A08375A00063780008608
S123D140850CCD0E379DD501B61EF50027FA2771D07637DC37AC27FA37DC34018504CD0632
S123D160379D35409A08375A0006B0588504CD06379DF50CDA01B04C850CCD0E379DD50103
S123D180CA01F980B7088504CD06379DF50CDA01B0068504CD06379DF506DA011708800120
S123D1A0C5013705FA02E7DA37ECF500379E37EC37BECBC2FA02E95034018504CD06379D80
S123D1C035409A08375A0006850CCD0E379D9502FA02E93434018504CD06379D35409A0435
S123D1E0375A0002CC023F0827F734073FFC274F37DC277A379DD50017FA33FB374500065B
S123D2008508FC013733000034033735000F37B533EAFA02E0D03F04270500028502FCFCBF
S123D220378C01088506CD08379D850237DDD516277AF50F37BD578C379D277A37450002F5
S123D24027DA8506CD08379D850237DDD51AF881B624F50F37BD595A379D850227F427F47C
S123D26037DDF50027FA2771CBB237EC37AC27FA37EC9A02375A0000B034F50F37BD595A65
S123D280379D850227F427F437DD8506CE08379E850237EDE51A27F8FA02E7DA37ECF50011
S123D2A0379E37EC37BECBB6FA02E9509A02375A00008506CD08379D850237DDD51E277A37
S123D2C0F50F37BD5955379D277A3745000227DAF50F37BD579C379D850227F427F437DD20
S123D2E08506CE08379E850227F437EDA522FA02E93437ECF500379E37EC37BECBBAFA02C8
S123D300E9509A02375A00008506CD08379D850237DDD512277AF50F37BD516E379D277A20
S123D3203745000227DA270300023780FEEC27050002850237B80003BC3AF50F37BD579021
S123D340379D850227F427F437DD8506CE08379E850227F437EDA52AFA02E93437ECF50028
S123D360379E37EC37BECBBAFA02E9509A02375A000027030002B0B68506CD08379DD5300A
S123D38017FA5174D53117FA5173D53227F8FA02E7DA2773004E27050002850237B8000465
S123D3A0378C008E37350006372627753706BAFE2770810837430006FC343733000037DC6B
S123D3C0277A379D850237350006372627753706BAFE277037B151863733000F37EC277A5A
S123D3E0379EF506FA02E916850227F427F427753706BAFE2770810837430006FC4C3733BE
S123D400000037DC277A379D850227F427F427753706BAFE277037B151763733000F37EC50
S123D420277A379E9500AA009502AA02270300023780FF6427050002850237B80008BC4200
S123D440F50F37BD57AC379D850237350006372637DD8506CE08379E3745000227742774A5
S123D460376DE55CDA008506CE08379E850227F427F437EDA55EFA02E9349A04375A000285
S123D48027030002B0AE27050002850237B8001ABC3A27F427F427753706BAFE2770810863
S123D4A037430006FC7C37330000340385023735000E372627753706BAFE277037B157DC2E
S123D4C03733000FFA00D07A3F0427030002B0B6CC043F0A27F7340F274F37DC277A379D3E
S123D4E0D50017FA33FB374500048506FC013733000034033735000F37B533EAFA02E0D03B
S123D5003F04270500008500FCFC378C00A68504CD06379D850037DDD516277AF50F37BD65
S123D520578C379D277A3745000027DAF50F37BD595A379D850027F427F437DD8504CE0667
S123D540379E850027F427F437ED3765001AA51C9A02375A00008504CD06379D850037DDA6
S123D560D52A277AF50F37BD5955379D277A3745000027DAF50F37BD579C379D850027F410
S123D58027F437DD3765002EA5309A02375A00008504CD06379D850037DDD512277AF50F37
S123D5A037BD516E379D277A3745000027DA270300003780FF4E27050000850037B80003F1
S123D5C0BC2CF50F37BD5790379D850027F427F437DD8504CE06379E850027F427F437EDCC
S123D5E03765003EA5409A02375A000027030000B0C48504CD06379DD54A17FA5174D54B58
S123D60017FA5173D54C27F8FA02E7DA2773004E27050000850037B80004378C008E3735EB
S123D6200006372627753706BAFE2770810637430004FC4E3733000037DC277A379D850095
S123D64037350006372627753706BAFE277037B151863733000F37EC277A379EF506FA0207
S123D660E916850027F427F427753706BAFE2770810637430004FC663733000037DC277A3F
S123D680379D850027F427F427753706BAFE277037B151763733000F37EC277A379E950079
S123D6A0AA009502AA02270300003780FF6427050000850037B80008BC46373500063726BC
S123D6C027753706BAFE2770810637430004FC763733000037DC277A379D850037350006BE
S123D6E0372627753706BAFE277037B157AC3733000F37EC277A379EF506FA02E916270384
S123D7000000B0AA27050000850037B8001ABC483735000E372627753706BAFE2770810667
S123D7203743000437B100A63733000037DC277A379D85003735000E372627753706BAFEFA
S123D740277037B157DC3733000F37EC277A379EF50EFA02E91627030000B0A8CC023F086C
S123D76027F70000D7D10000D7C50000D7BA0000D7AC0000D79E0000D7960000D78A0000EC
S123D780D782554E4B4E4F574E0054574F5F494E5F464F555200464F5552574159005448A8
S123D7A05245455741595F49535F460054485245455741595F4D535F46005448524545571C
S123D7C041595F460054574F5741595F4D535F460054574F574159000000D7F50000D7F1F8
S123D7E00000D7ED0000D7E8494E313200494E3200494E31003F3F3F00000000D8CA0000B8
S123D800D8C20000D8BB0000D8B40000D8AD0000D8A60000D89F0000D8980000D8910000F8
S123D820D88A0000D8810000D8780000D86F0000D8660000D85D0000D8540000D84B0000D0
S123D840D8424C494E4B575A32340042555454455232340042455353454C3234004255541A
S123D86054455231380042455353454C3138004C494E4B575A3132004255545445523132AE
S123D8800042455353454C31320053313251323000533132513135005331325131320053D0
S123D8A03132513130005331325130380053313251303700533132513036005331325130CE
S123D8C0350042555454455236004F4646000000D9300000D9270000D91A0000D90D000046
S123D8E0D9020000D8F70000D8EA465459505F414C4C5041535300465459505F484943553B
S123D9005400465459505F4C4F43555400465459505F48495348454C5600465459505F4CE3
S123D9204F5348454C5600465459505F50455100465459505F425950415353002F2F207424
S123D9407970650025732C002F2F206E616D6500222573222C002F2F206C6162656C0030DC
S123D9607825303258202C002F2F20726F757465002C20002F2F206C6576656C00564F4C80
S123D9805F4F46462C0025332E3166202C002F2F20706F6C61726974790025692C20002FB9
S123D9A02F2064656C61790025392E36662C20002F2F206D617374657264656C6179002553
S123D9C0392E36662C20002F2F2064656C6179756E69740025692C2025692C002F2F207421
S123D9E0656D70657261747572650025692C002F2F20636F6D70726573736F720025692CAA
S123DA002025692C2025692C2025692C002F2F206C696D697465720025692C202025692C4C
S123DA20002F2F20786F7665720025732C2025752C002F2F2066696C746572002531317388
S123DA402C202532692C2025342E30662C2025332E31662C2025322E30662C2000003407F6
S123DA60373FFF0C274FF50037BDD762379D276C3E74F520FA02E916F50037BDD7D8379DF4
S123DA80276C3E64F510FA02E916F50037BDD7FA379D276C3E1CF548FA02E916F50037BDB1
S123DAA0D8CE379D276CF51CFA02E9163735000037B5D93CFA01726885F6CDF8379DD5001E
S123DAC03705277B277427747C74275C375D37550000950234033735000037B5D944340321
S123DAE0275C373D00B637AD3705277B37DCFA02B5CC3F08275C373D00B637AD3705277B6D
S123DB0037DCFA0172683735000037B5D948FA017268374500F685F8FC013733000034033E
S123DB203735000037B5D9503403275C373D00B637AD3705277B37DCFA02B5CC3F08275C60
S123DB40373D00B637AD3705277B37DCFA0172683735000037B5D956FA01726805B62705AA
S123DB6000F285F2FCFCBC4C85F6CDF8379D85F237DDD512370534013735000037B5D95FB1
S123DB803403275C373D00A237AD3705277B37DCFA02B5CC3F06275C373D00A2340837AD61
S123DBA034013D1437AD3705277B37DCFA02E0863F04270300F2B0A6275C373D00B637AD5E
S123DBC03705277B37DCFA0172683735000037B5D968FA01726805B6270500F285F2FCFCC5
S123DBE0BC5685F6CDF8379D85F237DDD51627F8277B277427747C64275C375D375500000B
S123DC0095023403275C373D00B637AD3705277B37DCFA02E0863F043735000037B5D97169
S123DC203403275C373D00B637AD3705277B37DCFA02E0863F04270300F2B09C275C373D23
S123DC4000B637AD3705277B37DCFA0172683735000037B5D974FA01726805B6270500F20D
S123DC6085F2FCFC378C009485F6CDF8379D85F237DDD51AF881B61C3735000037B5D97D53
S123DC803403275C373D00A237AD3705277B37DCFA02E0D03F04B03E85F6CDF8379D85F273
S123DCA037DDD51A27F8FA02E7DA37ECF500379E37EC37BECBB6FA02E95034033735000023
S123DCC037B5D9863403275C373D00A237AD3705277B37DCFA02B5CC3F08275C373D00A2F3
S123DCE0340837AD34013D1437AD3705277B37DCFA02E0863F04270300F23780FF60275C4B
S123DD00373D00B637AD3705277B37DCFA0172683735000037B5D98EFA01726805B62705B0
S123DD2000F285F2FCFCBC4C85F6CDF8379D85F237DDD51E27F834013735000037B5D99AC5
S123DD403403275C373D00A237AD3705277B37DCFA02B5CC3F06275C373D00A2340837AD9F
S123DD6034013D1437AD3705277B37DCFA02E0863F04270300F2B0A6275C373D00B637AD9C
S123DD803705277B37DCFA0172683735000037B5D99FFA01726805B6270500F285F2FCFCCC
S123DDA0BC6085F6CDF8379D85F227F437DD9522FA02E93437ECF500379E37EC37BECBBA2F
S123DDC0FA02E95034033735000037B5D9A83403275C373D00A237AD3705277B37DCFA0259
S123DDE0B5CC3F08275C373D00A2340837AD34013D1437AD3705277B37DCFA02E0863F049E
S123DE00270300F2B092275C373D00B637AD3705277B37DCFA0172683735000037B5D9B068
S123DE20FA01726805B6270500F285F2FCFDBC6085F6CDF8379D85F227F437DD952AFA022F
S123DE40E93437ECF500379E37EC37BECBBAFA02E95034033735000037B5D9BF3403275C01
S123DE60373D00A237AD3705277B37DCFA02B5CC3F08275C373D00A2340837AD34013D14B0
S123DE8037AD3705277B37DCFA02E0863F04270300F2B092275C373D00B637AD3705277B37
S123DEA037DCFA0172683735000037B5D9C7FA01726885F6CDF8379DD53137053401D53019
S123DEC034013735000037B5D9D43403275C373D00B637AD3705277B37DCFA02B5CC3F0887
S123DEE0275C373D00B637AD3705277B37DCFA0172683735000037B5D9DCFA01726885F66A
S123DF00CDF8379DD53227F834013735000037B5D9EB3403275C373D00B637AD3705277B47
S123DF2037DCFA02B5CC3F06275C373D00B637AD3705277B37DCFA0172683735000037B559
S123DF40D9EFFA01726805B6270500F285F2FCFCBC5685F6CDF8379D85F23735000637266C
S123DF6037DD95383401D53637053401D5353401D53427F834013735000037B5D9FD34030A
S123DF80275C373D00B637AD3705277B37DCFA02B5CC3F0C275C373D00B637AD3705277BC4
S123DFA037DCFA017268270300F2B09C3735000037B5DA0DFA017268270500F2374500F26D
S123DFC037380004BC4885F6CDF8379D27742774375D954E3401D54C27F8340137350000EF
S123DFE037B5DA183403275C373D00B637AD3705277B37DCFA02B5CC3F08275C373D00B615
S123E00037AD3705277B37DCFA017268270300F2B0A63735000037B5DA21FA01726827058C
S123E02000F2374500F237380008BC6885F6CDF8379D27742774375D955E340185F6CDF89B
S123E040379D85F227F427F437DDD55C27F8277B277427747C1C275C375D3755000095022D
S123E06034033735000037B5DA2A3403275C373D00B637AD3705277B37DCFA02B5CC3F0A8A
S123E080275C373D00B637AD3705277B37DCFA017268270300F2B0863735000037B5DA326F
S123E0A0FA017268270500F285F237B8001A378C009827F427F427753706BAFE277081F8B7
S123E0C0374300F6FC7C373300003403275C373D009437AD3705277B37DCFA00D07A3F04CC
S123E0E03745009E85A034033745009A859C34033745009685983403C59527F83401C594CB
S123E10027F8277B27742774275C375D37550000950234033735000037B5DA3C3403275C6B
S123E120373D00B637AD3705277B37DCFA02B5CC3F16275C373D00B637AD3705277B37DC88
S123E140FA017268270300F23780FF5ACCF4373F00FA27F725303269200034043FF8274F77
S123E16027050002850237B8001E378C00C6F50F37BD34E1379D8502373500E43726277B99
S123E18027D5378600923735000237B549A4FA00D4D68502373500E4372627753706BAFE80
S123E1A0277037B134E03733000FFA00CBC68502373500E4372627753706BAFE277037B180
S123E1C034E13733000FFA02E4B637B8000EB2468502FC0134013735000037B5E1543403A5
S123E1E0275C3D0437AD3705277B37DCFA02B5CC3F06275C3D04340837AD340185023735B4
S123E20000E4372627753706BAFE277037B134E13733000FFA02E0863F04F50F37BD34E06A
S123E220379D8502373500E4372637DD1511270300023780FF2CCC083F0A27F74E45573A2B
S123E2400053544F52452050524F4752414D20544F3A0045444954204E4557205449544C6B
S123E260453A005525303275000034043FE6274F37B50001FA00AF64FA00AE7037F5004871
S123E280FCE2BF1637F5004A37B8001EBE0437FF004A0048B00437B5000137FA004827F584
S123E2A0FA00C25C37B500173735000134033735000037B5E23CFA00C1043F0437B5001720
S123E2C03735001A34033735000F37B533EAFA00C1043F0437B50003FA00C25C17F5004D97
S123E2E0F801B706F802B726F50117FA004D37B500013735000334033735000037B5E2412B
S123E300FA00C1043F0437B50010FA00C25C378000A437B500013735000334033735000089
S123E32037B5E253FA00C1043F0437B5000237BD007937BE001F341937B5001AFA00B358EF
S123E3403F06377533E6B76CF50F37BD33EA379D3DFF27D5CA06050737B50010FA00C25C7B
S123E36037B500173401F50F37BD33EA379D3DFF370537AD8A028D04277537F533E6BAFE66
S123E3802770810437430002FA00C2148A003735000F37B533EAFA00C214FC1A8000340168
S123E3A0275C3D0637AD3705277B37DCFA00C1043F0427F5FA00C25C37F500483401373573
S123E3C0000037B5E2633403275C3D0637AD3705277B37DCFA02B5CC3F0637B5000C37BD88
S123E3E000013409275C3D0637AD3705277B37DCFA00C1043F0437B5000C37BD001A3409FB
S123E400F50F37BD34E0379D373DFF1D370537AD8A028D0437F50048373500E4372627758E
S123E4203706BAFE2770810437430002FA00C1043F0427F5FA00AF64CC1A3F1C27F74F561C
S123E44045525752495445205525303275203F0050524553532053544F524500544F204386
S123E4604F4E4649524D2021000034043FEC274FF50317FA004D37B50001FA00AF64FA0069
S123E480AE7027F5FA00C25C37F5004834013735000037B5E43E3403275C37AD3705277B87
S123E4A037DCFA02B5CC3F0637B5000137BD000A3409275C37AD3705277B37DCFA00C10444
S123E4C03F0437B5000C3735000A34033735000037B5E450FA00C1043F0437B50017373553
S123E4E0000A34033735000037B5E45CFA00C1043F0427F5FA00AF64CC143F1627F750521F
S123E5004F4752414D2053544F5245442E2E2E0034043FFC274FF50F37BD34E0379D373DC9
S123E520FF1C370537AD8A008D0237F50048373500E4372627753706BAFE2770810237433D
S123E5400000FA00CBC637FF0048004AFA00AE7027F5FA00C25C37B5001737350002340370
S123E5603735000037B5E4FEFA00C1043F0437B507D037FA3198173533E437B50001FA0153
S123E580BA00CC043F0627F7340D274F27F6B602CC023F0627F78504FCF6BD0237B50001A6
S123E5A08A048504FC0ABE0237B5FFFF8A0417F5004DF801B704F802B72C3780009E85043A
S123E5C037F1004837FA0048FCE2BF0837B5001E37FA00483780008437F50048FCFFBC7A46
S123E5E037B5000137FA0048B070270500003745000037380061B422F50037BDCB51379D6A
S123E60027D5277AF50F37BD33EA379D277A3DFF377533E627D8B70227030000B0CC8504E7
S123E62081008A00BC00FC618A00850037B80061B5002705000037F533E6B71EF50037BD6F
S123E640CB51379D3745000027D5277AF50F37BD33EA379D277A3DFF377533E627DAFA0027
S123E660E26AF50117FA33E9CC023F0627F700050002E69AE6D4E70CE760E738000000005C
S123E680E7603405274F27F6B602CC003F0427F7850237BDE66EFA02E81817F5004DF80161
S123E6A0B702F802B70EB020F50217FA004D37B5001037FA33E6B010273133E637F533E6FD
S123E6C037B80001BC02F50117FA004DFA00E26A3780009417F5004DF801B702F802B70ED9
S123E6E0B020F50217FA004D37B5000137FA33E6B010273333E637F533E637B80010BF0282
S123E700F50117FA004DFA00E26AB05A17F5004DF802B702F803B716B04CF50F37BD33EA6C
S123E720379DF5203DFF377533E627DAFA00E26AB034FA00E26AB02E17F5004DF803B6167C
S123E740FA00E5103735000F37B533EA340337F5004AFA01B0043F04B00CFA00E46AB006E9
S123E760173533E98502FA00A492CC003F0427F737F53198FC01BE0C27353198173533E900
S123E78037B50006FA00A49227F73735000F37B533FCFA00CBC627F755253032750046253A
S123E7A03032750034053FDC274F37B8001E378E00B634013735000037B5E7983403275C66
S123E7C03D0C37AD3705277B37DCFA02B5CC3F0637B5000D37BD00013409275C3D0C37AD7A
S123E7E03705277B37DCFA00C1043F04C52DB71A3735000F37B533EA3403275C3D0C37ADF4
S123E8003705277B37DCFA02E0D03F04B03AF50F37BD34E0379D373DFF1D370537AD8A0010
S123E8208D028526373500E4372627753706BAFE27708102374300003403275C3D0C37ADE1
S123E8403705277B37DCFA02E0D03F0437B5000D37BD001A3409275C3D0C37AD3705277B02
S123E86037DCFA00C1043F04B0768526FCE28A0834013735000037B5E79E3403275C3D0C29
S123E88037AD3705277B37DCFA02B5CC3F0637B5000D37BD00013409275C3D0C37AD3705C6
S123E8A0277B37DCFA00C1043F0437B5000D37BD001A3409F50237BD4BB6379D373DFDEF39
S123E8C0370537AD8A008D02850837350212372627753706BAFE2770810237430000FA0072
S123E8E0C1043F0437B50003FA00C25C8526FCE2BE28C52DB70617F533FB37058A0AB036F7
S123E900F50F37BD34E0379D373DFF1C8526373500E43726277B27D537058A0AB018F502FF
S123E92037BD4BB6379D373DFDEE8508373502123726277B27D537058A0A850AFCF9BF048C
S123E94037B500078A0AB004850ABC002705000A37B5001837BD00013409F50F37BD0028A1
S123E960379D3745000A27742774375D375500009502FA00C104CC243F2C27F744783338ED
S123E9802050524F4752414D3A0037B50001FA00AF64FA00AE7037B50003FA00C25C37B5FC
S123E9A000013735000134033735000037B5E97CFA00C1043F0427F5FA00C25C37B50001CE
S123E9C0340137F5004AFA00E7A43F0227F5FA00AF6437FF004A004827F7524543414C4C00
S123E9E02050524F4752414D3A00F50117FA004D37B50001FA00AF64FA00AE7027F5FA0025
S123EA00C25C37B500013735000334033735000037B5E9DAFA00C1043F0437B50010FA002E
S123EA20C25C27F5340137F50048FA00E7A43F0227F5FA00AF6427F7524543414C4C2050BF
S123EA40524F4752414D3A0041524520594F5520535552453F005052455353205245434155
S123EA604C4C2000F50317FA004D37B50001FA00AF64FA00AE7027F5FA00C25C37B5000151
S123EA803735000334033735000037B5EA38FA00C1043F0437B50010FA00C25C27F53401EB
S123EAA037F50048FA00E7A43F0227F5FA00C25C37B5001737BD007937BE000C341937B53A
S123EAC00019FA00B6543F0637B5001F37BD007937BE0017341927F5FA00B6543F0637B5AE
S123EAE0000D3735001A34033735000037B5EA48FA00C1043F0437B500183735001A3403FB
S123EB003735000037B5EA56FA00C1043F0427F5FA00AF6427F7524543414C4C2050524F4C
S123EB204752414D3A004348414E474520434F4E46494700535552453F200000340C274FA0
S123EB40F50417FA004D37F50048FCE18A0037F5004837B8001EBE1CF50F37BD34E0379D44
S123EB60373DFF1C37F50048373500E43726277B27D517F833FBB72037F5004837B8001EAE
S123EB80BF2AF50237BD4BB6379D8500373502123726277B27D517F833FBB61037F5004851
S123EBA0FA00EC7237F50048FA01B7CA351827F737B50001FA00AF64FA00AE7027F5FA0076
S123EBC0C25C37B500013735000334033735000037B5EB16FA00C1043F0437B50010FA002F
S123EBE0C25C27F5340137F50048FA00E7A43F0227F5FA00C25C37B5001737BD007937BECF
S123EC00000C341937B50019FA00B6543F0637B5001F37BD007937BE0017341927F5FA0062
S123EC20B6543F0637B5000D3735001A34033735000037B5EB26FA00C1043F0437B500185C
S123EC403735001A34033735000037B5EB34FA00C1043F0427F5FA00AF64351827F7505244
S123EC604F4752414D20524543414C4C45442E2E2E0034053FF6274FF501CA05850C37B80B
S123EC800050BF02CC0A3F0E27F7850CB60437F5004A8A0C0505850C37B8001EBE2CF50F31
S123ECA037BD34E0379D373DFF1C370537AD8A008D02850C373500E4372627753706BAFEDD
S123ECC02770810237430000FA00D1EAB01C850CFCE18A0637350212372627753706BAFEAF
S123ECE0277037B14BB637330002FA00D4D6850C37FA004AFA020C88173533E4C505B732CE
S123ED00FA00AE7027F5FA00C25C37B500173735000234033735000037B5EC5EFA00C1049A
S123ED203F04F50117FA33E837B507D037FA3198F50517FA004DFA02035637B50001FA0118
S123ED40BA00CC0A3F0E27F73405274F27F6B728850237F1004837FA0048FCB0BF0637B53C
S123ED60005037FA0048B00C37F50048FCFFBC0437B5000137FA0048FA00E9EACC003F0499
S123ED8027F700000003EDAC0002EDD80003EE040007EE4E3405274F27F6B602CC003F0423
S123EDA027F7850237BDED82FA02E8182731004837F50048FCB0BF0637B5005037FA004811
S123EDC0B00C37F50048FCFFBC0437B5000137FA0048FA00E9EAB0782733004837F50048D3
S123EDE0FCB0BF0637B5005037FA0048B00C37F50048FCFFBC0437B5000137FA0048FA009E
S123EE00E9EAB04C17F5004DF801B728F803B706F804B708F805B716B036FA00EB3CB030CA
S123EE2037F50048FA00EC7237F50048FA01B7CAB01E173533E8B01817F50053B702FA0003
S123EE40EA64B00C37B50007FA00A492B0028502FA00A492CC003F0427F737F5319837B807
S123EE60FFFFBE1417F533E8B602FA00EE7EB0082735319837B50007FA00A49227F737F52F
S115EE80319837B8FFFFBE0427353198FA00E9EA27F7F4
S2240100000000000104D40001000104C70002000104BA0003000104AD01000001049E010118
S2240100200001048F0102000104800103000104710104000104620105000104530106000152
S2240100400444010700010435010800010426010900010417010A00010406010B000103F59B
S224010060010C000103E4010D000103D3010E000103C2010F000103B10110000103A001113F
S2240100800001038F01120001037E01130001036D01140001035C01150001034B01160001BB
S2240100A0033A0117000103290118000103180119000103070200000102F50201000102E37B
S2240100C00202000102D10203000102BF0204000102AD02050001029B020600010289020783
S2240100E00001027703000001026603010001025503020001024204000001022F0401000132
S224010100021C0402000102090403000101F60500000101E60501000101D60502000101C610
S2240101200503000101B60600000101A906010001019C06020001018F060300010182070076
S2240101400001017707010001016C0702000101610703000101564F5554343A4C4556454CFE
S224010160004F5554333A4C4556454C004F5554323A4C4556454C004F5554313A4C45564531
S2240101804C004F5554343A4C494D49544552004F5554333A4C494D49544552004F555432EC
S2240101A03A4C494D49544552004F5554313A4C494D49544552004F5554343A434F4D505289
S2240101C04553534F52004F5554333A434F4D50524553534F52004F5554323A434F4D505236
S2240101E04553534F52004F5554313A434F4D50524553534F52004F5554343A4348414E4E2F
S224010200454C2044454C4159004F5554333A4348414E4E454C2044454C4159004F555432A1
S2240102203A4348414E4E454C2044454C4159004F5554313A4348414E4E454C2044454C4164
S2240102405900494E312B323A4D41535445522044454C415900494E323A4D41535445522096
S22401026044454C415900494E313A4D41535445522044454C4159004F5554343A4C4F50411A
S224010280535320584F564552004F5554343A48495041535320584F564552004F5554333AB7
S2240102A04C4F5041535320584F564552004F5554333A48495041535320584F564552004F82
S2240102C05554323A4C4F5041535320584F564552004F5554323A48495041535320584F5634
S2240102E04552004F5554313A4C4F5041535320584F564552004F5554313A4849504153534D
S22401030020584F564552004F5554343A4348414E4E454C20455134004F5554343A434841A8
S2240103204E4E454C20455133004F5554343A4348414E4E454C20455132004F5554343A43B1
S22401034048414E4E454C20455131004F5554333A4348414E4E454C20455134004F55543387
S2240103603A4348414E4E454C20455133004F5554333A4348414E4E454C20455132004F5571
S22401038054333A4348414E4E454C20455131004F5554323A4348414E4E454C20455134006F
S2240103A04F5554323A4348414E4E454C20455133004F5554323A4348414E4E454C204551DE
S2240103C032004F5554323A4348414E4E454C20455131004F5554313A4348414E4E454C2025
S2240103E0455134004F5554313A4348414E4E454C20455133004F5554313A4348414E4E45D8
S2240104004C20455132004F5554313A4348414E4E454C2045513100494E323A4D41535445E2
S224010420522045513500494E323A4D41535445522045513400494E323A4D415354455220D1
S22401044045513300494E323A4D41535445522045513200494E323A4D415354455220455191
S2240104603100494E313A4D41535445522045513500494E313A4D41535445522045513400D4
S224010480494E313A4D41535445522045513300494E313A4D41535445522045513200494E52
S2240104A0313A4D415354455220455131004F5554343A524F5554494E47004F5554333A52D3
S2240104C04F5554494E47004F5554323A524F5554494E47004F5554313A524F5554494E4729
S2240104E000000100000109B40101000109A5010200010996010300010987010400010978C7
S22401050003000001096701050001095801060001094901070001093A01080001092B01090B
S2240105200001091C03010001090B0302000108F80000000108EB010A000108DA010B000181
S22401054008C9010C000108B8010D000108A70200000108950201000108830400000108708C
S22401056005000001086006000001085307000001084800010001083B010E0001082A010FB6
S224010580000108190110000108080111000107F70202000107E50203000107D30401000129
S2240105A007C00501000107B00601000107A307010001079800020001078B01120001077A2C
S2240105C001130001076901140001075801150001074702040001073502050001072304023B
S2240105E0000107100502000107000602000106F30702000106E80003000106DB01160001D7
S22401060006CA0117000106B90118000106A801190001069702060001068502070001067395
S2240106200403000106600503000106500603000106430703000106384F5554343A4C4556FE
S224010640454C004F5554343A4C494D49544552004F5554343A434F4D50524553534F520014
S2240106604F5554343A4348414E4E454C2044454C4159004F5554343A4C4F504153532058D6
S2240106804F564552004F5554343A48495041535320584F564552004F5554343A4348414EB6
S2240106A04E454C20455134004F5554343A4348414E4E454C20455133004F5554343A434832
S2240106C0414E4E454C20455132004F5554343A4348414E4E454C20455131004F5554343A12
S2240106E0524F5554494E47004F5554333A4C4556454C004F5554333A4C494D495445520074
S2240107004F5554333A434F4D50524553534F52004F5554333A4348414E4E454C2044454C0E
S2240107204159004F5554333A4C4F5041535320584F564552004F5554333A48495041535301
S22401074020584F564552004F5554333A4348414E4E454C20455134004F5554333A43484166
S2240107604E4E454C20455133004F5554333A4348414E4E454C20455132004F5554333A436F
S22401078048414E4E454C20455131004F5554333A524F5554494E47004F5554323A4C4556DE
S2240107A0454C004F5554323A4C494D49544552004F5554323A434F4D50524553534F5200B7
S2240107C04F5554323A4348414E4E454C2044454C4159004F5554323A4C4F50415353205879
S2240107E04F564552004F5554323A48495041535320584F564552004F5554323A4348414E59
S2240108004E454C20455134004F5554323A4348414E4E454C20455133004F5554323A4348D4
S224010820414E4E454C20455132004F5554323A4348414E4E454C20455131004F5554323AB4
S224010840524F5554494E47004F5554313A4C4556454C004F5554313A4C494D495445520016
S2240108604F5554313A434F4D50524553534F52004F5554313A4348414E4E454C2044454CB1
S2240108804159004F5554313A4C4F5041535320584F564552004F5554313A484950415353A4
S2240108A020584F564552004F5554313A4348414E4E454C20455134004F5554313A43484109
S2240108C04E4E454C20455133004F5554313A4348414E4E454C20455132004F5554313A4312
S2240108E048414E4E454C20455131004F5554313A524F5554494E4700494E312B323A4D41DD
S224010900535445522044454C415900494E323A4D41535445522044454C415900494E323AA3
S2240109204D41535445522045513500494E323A4D41535445522045513400494E323A4D41B0
S224010940535445522045513300494E323A4D41535445522045513200494E323A4D4153547B
S22401096045522045513100494E313A4D41535445522044454C415900494E313A4D4153545F
S22401098045522045513500494E313A4D41535445522045513400494E313A4D415354455249
S2240109A02045513300494E313A4D41535445522045513200494E313A4D415354455220455F
S2240109C051310000001400150016001700180019001A001B001C001D001E001F002000211C
S2240109E000220023002400250026002700280029002A002B002C002D002E002F0030003159
S224010A000032003400360038003A003C003E003F00400042004400460048004A004C004ED1
S224010A2000500052005400560058005A005C005E0060006200640068006C007000740078A2
S224010A40007C007D008000840088008C009000940098009C00A000A400A800AC00B000B42B
S224010A6000B800BC00C000C400C800D200DC00E600F000FA0104010E01180122012C01367E
S224010A800140014A0154015E01680172017C01860190019A01A401AE01B801C201CC01D690
S224010AA001E001EA01F40208021C023002440258026C02760280029402A802BC02D002E457
S224010AC002F8030C032003340348035C03700384039803AC03C003D403E804100438046086
S224010AE0048804B004D804E2050005280550057805A005C805F0061806400668069006B85D
S224010B0006E0070807300758078007A807D00834089808FC096009C40A280A8C0AF00B5400
S224010B200BB80C1C0C800CE40D480DAC0E100E740ED80F3C0FA01004106810CC113011946C
S224010B4011F8125C12C0132413881450151815E016A817701838189C190019C81A901B588E
S224010B601C201CE81DB01E781F40200820D021982260232823F024B825802648271028A0CE
S224010B802A302BC02D502EE0307030D432003390352036B0384039D03B603CF03E80401055
S224010BA041A0433044C0465047E049704B004C904E20000400050006000700080009000A9B
S224010BC0000B000C000D000E000F00100012001400160018001A001C001E002000230028AB
S224010BE0002D00320037003C004100460050005A0064006E00780082008C009600A000B4AA
S224010C0000C8554E4B4E4F574E0054574F5F494E5F464F555200464F555257415900544882
S224010C205245455741595F49535F460054485245455741595F4D535F460054485245455765
S224010C4041595F460054574F5741595F4D535F460054574F57415900414C4C5041535300C5
S224010C604C4F5041535300484950415353004849534C56004C4F534C56005045510042593D
S224010C8050415353004C696E6B7769747A20323420644200427574746572203234206442AD
S224010CA00042657373656C20323420644200427574746572203138206442004265737365CD
S224010CC06C203138206442004C696E6B7769747A20313220644200427574746572203132B5
S224010CE02064420042657373656C20313220644200313220644220513D322E300031322097
S224010D00644220513D312E3500313220644220513D312E3200313220644220513D312E3017
S224010D2000313220644220513D302E3800313220644220513D302E3700313220644220513A
S224010D403D302E3600313220644220513D302E3500362064420074687275004C494E4B570E
S224010D603234444200425554544552323444420042455353454C3234444200425554544591
S224010D8052313844420042455353454C31384442004C494E4B57313244420042555454456D
S224010DA052313244420042455353454C31324442003132444251322E300031324442513116
S224010DC02E35003132444251312E32003132444251312E30003132444251302E38003132E3
S224010DE0444251302E37003132444251302E36003132444251302E3500364442005448523C
S224010E005500636D006D00696E63680066656574008073006D7300494E56455254454400C0
S224010E204E4F524D414C00314F564552382E3000314F564552342E3000314F564552322E14
S224010E403000314F564552312E3400314F564552312E3000494E312B3200494E3200494EDB
S224010E6031004F464600434D004D00494E43480046454554005553004D530046414852458F
S224010E804E484549540043454C5349555300564F4C545300444255004442000034053FEA61
S224010EA0274F37F54F9AB60637B50010FA00C25CB00227F5FA00C25CF50F37BD4FA6379D2A
S224010EC037754F9C27742774375D9500DD02379D3755000295043403275C37AD3705277BC0
S224010EE037DCFA02E0D03F04C51F37053401C5193401275C37AD277B37DCFA00C1043F0464
S224010F0037B5000237BD00793409C51F3705FC09340127F5FA00B358CC163F2027F754798C
S224010F2070653A253473000034053FEC274F37F54F9AFCFFB60637B50013FA00C25CB0045F
S224010F4037B50003FA00C25CF50F37BD0074379DC5173705277B27742774375D3755000034
S224010F60950234033735000137B50F1E3403275C37AD3705277B37DCFA02B5CC3F08C51FE0
S224010F8037053401C51D3401275C37AD277B37DCFA00C104CC143F1C27F7547970653A2093
S224010FA02573000034053FEA274F37F54F9AFCFFB60637B50013FA00C25CB00437B5000335
S224010FC0FA00C25CF50F37BD0090379DC5193705277B27742774375D3755000095023403B7
S224010FE03735000137B50F9A3403275C37AD3705277B37DCFA02B5CC3F08C521370534013F
S224011000C51F3401275C37AD277B37DCFA00C104CC163F1E27F7447A00003A83126E3FFE41
S224011020B851663A25342E31666B487A00663A25342E32666B487A00411FD70A663A25358F
S2240110402E31666B487A00663A25352E32666B487A00663A25342E3066487A0034073FEAC8
S224011060274F37F54F9AFCFEB60637B50013FA00C25CB00437B50003FA00C25C37450018C3
S224011080F501379E851A37BE1016FA02E662378D00FEF50127FA2771101A37DC37AC27FACF
S2240110A037DC276C3E18FA02E69EC521F841B37EF846B31637F54F9AFCFEB60637B5001789
S2240110C0FA00C25CB00437B50007FA00C25C37450018F501379E851A37BE101EFA02E662CE
S2240110E0BD2437450018851A34033735000137B510223403275C3D0237AD3705277B37DC46
S224011100FA02B5CC3F08378000AA37450018851A34033735000137B5102D3403275C3D02AB
S22401112037AD3705277B37DCFA02B5CC3F083780008237450018F501379E851A37BE10389C
S224011140FA02E662BD2237450018851A34033735000137B5103C3403275C3D0237AD37053E
S224011160277B37DCFA02B5CC3F08B04637450018851A34033735000137B510473403275C26
S2240111803D0237AD3705277B37DCFA02B5CC3F08B02037450018851A34033735000137B5DE
S2240111A010523403275C3D0237AD3705277B37DCFA02B5CC3F08275C3D0237AD3705277BB1
S2240111C037DCFA00C2148A0037F54F9A37B80002B70027010000C5213705810037B80079AC
S2240111E0BF04F579C0013713CA21C52337053401C5213401275C3D0237AD277B37DCFA00F9
S224011200C104CC163F2027F7513A25332E306600513A25332E31660034073FE6274F37F553
S2240112204F9A8828B60637B50013FA00C25CB00437B50003FA00C25C37B5000AFA02E7DACE
S2240112408A02374A00003745001C851E276CFA02E662BD223745001C851E340337350001AB
S22401126037B512083403275C3D0637AD3705277B37DCFA02B5CC3F08B0203745001C851EC1
S22401128034033735000137B512103403275C3D0637AD3705277B37DCFA02B5CC3F08C52714
S2240112A037053401C5253401275C3D0637AD277B37DCFA00C104CC1A3F2427F7536C6F7075
S2240112C0653A25326964420034053FEA274F37F54F9AFCFDB60637B50013FA00C25CB00496
S2240112E037B50003FA00C25CC519370534013735000137B512BC3403275C3D0237AD370552
S224011300277B37DCFA02B5CC3F06C52137053401C51F3401275C3D0237AD277B37DCFA008B
S224011320C104CC163F1E27F74F726465723A326E64004F726465723A3173740034053FEA9B
S224011340274F37F54F9AFCFDB60637B50013FA00C25CB00437B50003FA00C25CC519F80C93
S224011360B61A3735000137B513283403275C3D0237AD3705277B37DCFA02E0D03F04B0187E
S2240113803735000137B513323403275C3D0237AD3705277B37DCFA02E0D03F04C5213705CA
S2240113A03401C51F3401275C3D0237AD277B37DCFA00C104CC163F1E27F74761696E3A2584
S2240113C02B332E306664420034073FEC274F37F54F9AFCFCB60637B50013FA00C25CB004CF
S2240113E037B50003FA00C25C37450016851834033735000137B513BA3403275C37AD37057A
S224011400277B37DCFA02B5CC3F08C52137053401C51F3401275C37AD277B37DCFA00C10402
S224011420CC143F1E27F73F000000497424003B03126E4000000044656C61793A25342E314C
S2240114406625730044656C61793A25342E306625730034073FE2274FC52DB70417F551745A
S224011460CA01B00217F55173CA01C5013705FA0115DA8A04374A0002C501F801B64A374516
S22401148000208522276C3E02FA02E6BA37ECF501379E37EC37BE1426FA02E620FA02E740AB
S2240114A0FA02E8B2276C3E02FA02E9508A08374A0006F50127FA2771142A37DC37AC27FA6B
S2240114C037DC276C3E06FA02E69EB010374500208522276C3E02FA02E6BA8A08374A000611
S2240114E037450020F501379E852237BE142EFA02E662BC5237450006F501379E850837BE80
S2240115001432FA02E662BC3EF50F37BD0120379DC5013705277B27742774375D375500005A
S2240115209502340337450006850834033735000137B514363403275C3D0A37AD3705277B2B
S22401154037DCFA02B5CC3F0CB03CF50F37BD0120379DC5013705277B27742774375D3755D7
S22401156000009502340337450006850834033735000137B514443403275C3D0A37AD37057F
S224011580277B37DCFA02B5CC3F0C37F54F9AFCFFB60637B50013FA00C25CB00437B5000342
S2240115A0FA00C25CC52B37053401C5293401275C3D0A37AD277B37DCFA00C104CC1E3F2816
S2240115C027F743888000473B80004487DCCC464BCD3343A5A66647016A0034053FF8274F0A
S2240115E0F801B326F501379E2771004E37BE15C2FA02E62037ECF501379E37EC37BE15C2B7
S224011600FA02E950FA02B6168A02374A0000C50BB712F801B728F802B73CF803B756F80458
S224011620B770F8053787008AF50127FA2771101637DC37AC27FA37DC8A06374A000437806D
S224011640008CF50127FA277115C637DC37AC27FA37DC8A06374A0004B072F50127FA27715E
S22401166015CA37DC37AC27FA37DC276CFA02E6BA8A06374A0004B054F50127FA277115CE81
S22401168037DC37AC27FA37DC276CFA02E6BA8A06374A0004B036F50127FA277115D237DC47
S2240116A037AC27FA37DC276CFA02E6BA8A06374A0004B018F50127FA277115D637DC37AC71
S2240116C027FA37DC276CFA02E6BA8A06374A0004374500048506CC083F0C27F7556E6974A4
S2240116E03A253473000034053FEA274FC521B70417F55174CA01B00217F55173CA0137F550
S2240117004F9AFCFEB60637B50013FA00C25CB00437B50003FA00C25CF50F37BD0120379D65
S224011720C5013705277B27742774375D37550000950234033735000137B516DC3403275CD6
S2240117403D0237AD3705277B37DCFA02B5CC3F08C51F37053401C5193401275C3D0237AD9D
S224011760277B37DCFA00C104CC163F1E27F73FE6666654656D703A25332E306681004300F1
S224011780460034053FE4274F37F54F9AFCFDB60637B50013FA00C25CB00437B50003FA00AD
S2240117A0C25C17F54F98B6082771004E8A06374A0004B02637B50020FA02E7DA8A02374AAD
S2240117C00000F501379E2771004E37BE176EFA02E6BA276CFA02E6208A06374A0004374516
S2240117E00004850634033735000137B517723403275C3D0837AD3705277B37DCFA02B5CCEA
S2240118003F0817F54F98B61A3735000137B5177E3403275C3D0837AD3705277B37DCFA02FA
S224011820E0863F04B0183735000137B517803403275C3D0837AD3705277B37DCFA02E0860B
S2240118403F04C52537053401C51F3401275C3D0837AD277B37DCFA00C104CC1C3F2427F742
S22401186054687273683A25326964420054687273683A25326964427500004120000041A059
S22401188000003F46666654687273683A25342E326656000034053FE8274F37F54F9AFCFF53
S2240118A0B60637B50013FA00C25CB00437B50003FA00C25C17F50052B708F801B72AF802A3
S2240118C0B74C378000B0C51B27F834013735000137B518603403275C3D0437AD3705277BD6
S2240118E037DCFA02B5CC3F063780008AC51B27F8FC1534013735000137B5186C3403275CF0
S2240119003D0437AD3705277B37DCFA02B5CC3F06B062C51B27F8FC15FA02E7DA37ECF501F1
S224011920379E37EC37BE187EFA02E9503403F50127FA2771187A37DC37AC27FA37DCFA024B
S224011940B3563F0437ECF501379E37EC37BE1882FA02E6BA8A02374A000034033735000148
S22401196037B518863403275C3D0437AD3705277B37DCFA02B5CC3F08C52337053401C52104
S2240119803401275C3D0437AD277B37DCFA00C104CC183F2027F75261743A312F25322E3118
S2240119A0660034073FEC274F37F54F9AFCFEB60637B50013FA00C25CB00437B50003FA0060
S2240119C0C25C37B50001FA02E7DA276C3E16FA02E95034033735000137B519963403275C24
S2240119E037AD3705277B37DCFA02B5CC3F08C52137053401C51F3401275C37AD277B37DCBC
S224011A00FA00C104CC143F1E27F741747461636B3A2532756D73000034053FEC274F37F562
S224011A204F9A8820B60637B50011FA00C25CB00437B50001FA00C25CC517370534013735CC
S224011A40000137B51A0A3403275C37AD3705277B37DCFA02B5CC3F06C51F37053401C51DE7
S224011A603401275C37AD277B37DCFA00C104CC143F1C27F752656C656173653A2532756DC3
S224011A80730052656C733A2532756D73000034053FEC274F37F54F9A8820B60637B5001101
S224011AA0FA00C25CB00437B50001FA00C25CC51DF82FB21C851634013735000137B51A74C1
S224011AC03403275C37AD3705277B37DCFA02B5CC3F06B01A851634013735000137B51A8220
S224011AE03403275C37AD3705277B37DCFA02B5CC3F06C51F37053401C51D3401275C37ADBC
S224011B00277B37DCFA00C104CC143F1C27F7536F757263653A25730034053FEC274F37F5A9
S224011B204F9AFCFFB60637B50013FA00C25CB00437B50003FA00C25CF50F37BD0154379D0C
S224011B40C5173705277B27742774375D37550000950234033735000137B51B0E3403275C65
S224011B6037AD3705277B37DCFA02B5CC3F08C51F37053401C51D3401275C37AD277B37DC3E
S224011B80FA00C104CC143F1C27F700011BED00011BE900011BE600011BE200011BDF00011D
S224011BA01BD800011BD100011BCA00011BC000011BB25355422D4C4F2D4D49442D48490038
S224011BC04C4F2D4D49442D4849004D49442D4849004C4F2D4D4944005355422D4C4F00486B
S224011BE049004D4944004C4F00535542004F4646004C6162656C3A25730034053FC4274FF8
S224011C00F50137BD1B8A379D276CF528FA02E91637F54F9AFCFEB60637B50013FA00C25CCE
S224011C20B00437B50003FA00C25CC53F3705277B27742774275C375D37550000950234035A
S224011C403735000137B51BF13403275C3D2837AD3705277B37DCFA02B5CC3F08C547370519
S224011C603401C5453401275C3D2837AD277B37DCFA00C104CC3C3F4427F7C31600004C6577
S224011C8076656C3A204F66660000000000004C6576656C3A25342E31666442004C65766500
S224011CA06C3A252B342E31666442000034073FEC274F37F54F9AFCFFB60637B50016FA00E5
S224011CC0C25CB00437B50006FA00C25CF50127FA37450016851837781C7AB60037F81C7C1A
S224011CE037DC37AC27FA37DCB6183735000137B51C7E3403275C37AD3705277B37DCFA0268
S224011D00E0D03F04B060F50127FA37450016851837781C8AB60037F81C8C37DC37AC27FA7B
S224011D2037DCB62037450016851834033735000137B51C8E3403275C37AD3705277B37DCBC
S224011D40FA02B5CC3F08B01E37450016851834033735000137B51C9C3403275C37AD37059A
S224011D60277B37DCFA02B5CC3F08C52137053401C51F3401275C37AD277B37DCFA00C10499
S224011D80CC143F1E27F700011D9700011D8E696E766572746564006E6F726D616C00000196
S224011DA01DAA00011DA6696E76006E6F726D00506F6C61726974793A25387300506F6C3AC6
S224011DC02534730034053FDC274FF50137BD1D86379D276C3E1CF508FA02E916F50137BD37
S224011DE01D9E379D276C3E14F508FA02E91637F54F9A8830B60637B50013FA00C25CB0041D
S224011E0037B50003FA00C25C1708FE27C52DF818B430C5273705277B277427747C1C275C70
S224011E20375D37550000950234033735000137B51DAF3403275C37AD3705277B37DCFA02FE
S224011E40B5CC3F08B02EC5273705277B277427747C14275C375D3755000095023403373569
S224011E60000137B51DBC3403275C37AD3705277B37DCFA02B5CC3F08C52F37053401C52DEC
S224011E803401275C37AD277B37DCFA00C104CC243F2C27F7000700001F1E1F281F281F289A
S224011EA01F321F321F32000000001F1E34043FFC274FF50F37BD4FA6379D37754F9C277410
S224011EC02774375D9500DD02379DD500F808B410FA02E8001FFA1EEA1F761FB21FCA1FE297
S224011EE01FEA1FF237800116F50F37BD57DC379DF50F37BE4FA6379E37754F9C2774277465
S224011F00376DA500EE02379EE501750E3724277B27D527F88A0037BD1E94FA02E81837B514
S224011F2000018A02378000DC37B500048A02378000D2F50F37BD57DD379DF50F37BE4FA688
S224011F40379E37754F9C27742774376DA500EE02379EE501750E3724277B27D5F80CB606A9
S224011F6037B500048A023780009A37B500038A0237800090F50F37BD57AC379DF50F37BE04
S224011F804FA6379E37754F9C27742774376DA500EE02379EE50175063724277B27D5B60482
S224011FA037B500018A02B05A37B500038A02B05217F55174F801BF0437B500038A02B04221
S224011FC037B500028A02B03A17F55173F801BF0437B500038A02B02A37B500028A02B0226A
S224011FE037B500048A02B01A37B500028A02B01237B500028A02B00A37B500028A02B002F9
S22401200037B500018A028502CC043F0627F700000003203A0000206200012056FFFF20749F
S22401202034053FFC274F27050000FA011EAC8A02850637BD200EFA02E81837F54F9A8802EB
S224012040BF04850237FA4F9AB02637F54F9ABC2027354F9AB01A27314F9ABC1427354F9AEA
S224012060B00E27334F9A37F54F9A8802BF02850237FA4F9AFA00AE7037B50001FA00AF6446
S22401208037B500013401FA010E9C3F02F50F37BD4FA6379D37754F9C27742774375D95007B
S2240120A0DD02379DD50137058A00F50F37BD4FA6379D37754F9C27742774375D9500DD0235
S2240120C0379DD500F808B410FA02E80025EC20E2236223F8245024AA2550259E3780053E82
S2240120E037B5000D37BD00013409F50F37BD57DC379D85003735000E3726277B27D527F897
S224012100FA010F283F04F50F37BD57DC379D85003735000E3726277B27D5F80137870096FE
S224012120F802B716F803B712F80437870108F80537870102F80637870190378004E037B5B9
S224012140000D37BD00463409F50F37BD57DE379D85003735000E372637DD37550000950261
S224012160FA01105C3F0437B5001737BD00013409F50F37BD57DD379D85003735000E37261E
S224012180277B27D527F8FA0112C83F0437B5001737BD00403409F50F37BD57E6379D850062
S2240121A03735000E372637DD375500009502FA0113C83F043780046637B5000D37BD00469E
S2240121C03409F50F37BD57DE379D85003735000E372637DD375500009502FA01105C3F047E
S2240121E037B5000337BD001737BE00023419F50F37BD57E2379D85003735000E372637DD26
S224012200375500009502FA0112183F0637B5001737BD00353409F50F37BD57E6379D850034
S2240122203735000E372637DD375500009502FA0113C83F04378003E637B5000D37BD00469E
S2240122403409F50F37BD57DE379D85003735000E372637DD375500009502FA01105C3F04FD
S22401226037B5001737BD00013409F50F37BD57DD379D85003735000E3726277B27D527F80A
S224012280FA0112C83F04F50F37BD57DD379D85003735000E3726277B27D5F80C3786037EE4
S2240122A037B5000437BD001737BE0046341937BD57E285003735000E372637DD375500006C
S2240122C09502FA0112183F063780035237B5000D37BD00493409F50F37BD57DE379D8500F2
S2240122E03735000E372637DD375500009502FA01105C3F0437B5001737BD00013409F50FE7
S22401230037BD57DD379D85003735000E3726277B27D527F8FA01133C3F04F50F37BD57DDE9
S224012320379D85003735000E3726277B27D5F80C378602EA37B5000437BD001737BE0046E6
S224012340341937BD57E285003735000E372637DD375500009502FA0112183F06378002BE89
S22401236037B5000D37BD00013409F50F37BD57AC379D8500373500063726277B27D527F84C
S224012380FA010FA43F04F50F37BD57AC379D8500373500063726277B27D53787028037B559
S2240123A0001737BD0002340937BD57AE850037350006372637DD375500009502FA01105CE2
S2240123C03F0437F54F9CFA012818FCFF8A0037B5000337BD001737BE00463419F50F37BD63
S2240123E05955379D3745000027D527F8FA011DC43F063780022837B5000137BD000D340991
S2240124003401F50F37BD5790379D3745000027742774375D375500009502FA0114523F06BF
S22401242037B5000137BD00173409FA0116E63F0417F55174F801378F01E437B5001734017A
S22401244037B5003AFA0117823F02378001D027F53401FC0D37BD00013409F50F37BD579C7C
S224012460379D3745000027742774375D375500009502FA0114523F0627F53401FC173401DA
S22401248037B50001FA0116E63F0417F55173F801378F018A37B50017340137B5003AFA019C
S2240124A017823F023780017637B5000D37BD00013409F50F37BD5186379D85003735000649
S2240124C03726277B27D527F8FA0118943F0437B5000D37BD00473409F50F37BD5187379DDD
S2240124E08500373500063726277B27D53705FA01414EFA0119A23F0437B5000337BD00172B
S22401250037BE00013419F50F37BD5188379D8500373500063726277B27D53705FA011A1872
S2240125203F0637B5000437BD001737BE00413419F50F37BD518A379D8500373500063726D7
S224012540277B2795FA011A8E3F06378000D037B5000D37BD00013409F50F37BD5176379DEA
S224012560374500002774277427D527F8FA0118943F0437B5000237BD001737BE0001341962
S224012580F50F37BD5178379D37450000277427742795FA011A8E3F063780008237B5000D18
S2240125A037BD00013409F50F37BD595A379D3745000027742774375D375500009502FA0100
S2240125C01CAC3F0437B5000237BD001737BE00013419F50F37BD5955379D3745000027D5BC
S2240125E027F8FA011DC43F06B03237B5000D37BD00013409F50F37BD578C379D374500005D
S22401260027D527F8FA011B183F0437B5001737BD000134098500FA0202D6FA011BFA3F0447
S22401262027F5FA00AF64CC043F0827F7340C274F27050000850037B80039B430F50F37BDCB
S2240126404FA6379D850027F427F437DD850037350006372627753706BAFE277037B104E292
S224012660373300019A02375A000027030000B0C027050000850037B80039B430F50F37BD6D
S224012680508A379D850027F427F437DD850037350006372627753706BAFE277037B1000053
S2240126A0373300019A02375A000027030000B0C0351827F7340F274F850CBC2A37B500F665
S2240126C08A008500BD50F50137BD09C4379D850027F437DD9500FA02E934276C3E04FA021A
S2240126E0E662BF3227010000B0D427050000850037B800F7B420F50137BD09C4379D850074
S22401270027F437DD9500FA02E934276C3E04FA02E662BC0227030000B0D0850C81008A00B9
S224012720BC0027050000850037B800F7B50237B500F68A00F50137BD09C4379D850027F4F2
S22401274037DD9500FA02E9348A06374A0004CC023F0827F734073FFC274F37ECF501379E8F
S22401276037EC37BE187AFA02E6BA37ECF501379E37EC37BE1426FA02E620FA02E7408A001E
S224012780850EBC1E37B500278A0237450002BD36F50137BD0BB2379D277427958800B32683
S2240127A027010002B0E0270500023745000237380028B412F50137BD0BB2379D277427957E
S2240127C08800B40227030002B0DC850E81028A02BC0027050002850237B80028B50237B530
S2240127E000278A02F50137BD0BB2379D37450002277427958A00FA02E93437ECF501379E3F
S22401280037EC37BE187AFA02E950CC043F0A27F74F555400494E0000340D274F270500002A
S22401282037B80039378C00BA37B5000334013735000137B528103403F50F37BD4FA6379D40
S2240128403745000427742774375D9500DD02379D375500029504FA02E11E3F06B624F50F9B
S22401286037BD4FA6379D3745000427742774375D9500DD02379D9502DD04379DD5033705A3
S224012880FCD08A00B05A37B5000234013735000137B528143403F50F37BD4FA6379D3745A6
S2240128A0000427742774375D9500DD02379D375500029504FA02E11E3F06B624F50F37BDC3
S2240128C04FA6379D3745000427742774375D9500DD02379D9502DD04379DD502370537B150
S2240128E000D08A008500CC023F0627F74F5554004F5554253175000034053FEA274F37B543
S224012900000334013735000137B528EC3403F50F37BD4FA6379D37754F9C27742774375DB3
S2240129209500DD02379D375500029504FA02E11E3F0637860084F50F37BD4FA6379D377534
S2240129404F9C27742774375D9500DD02379D3755000295043403275C3D0237AD3705277B92
S22401296037DCFA02E0D03F04C519F130CA05270500003745000037380039378C00A8F50FC2
S22401298037BD4FA6379D27742774375D9500DD02379D3755000295043403275C3D0237AD5E
S2240129A03705277B37DCFA02E0AE3F04B604850037FA4F9CB06E27030000B0B2851834017C
S2240129C03735000137B528F03403275C3D0237AD3705277B37DCFA02B5CC3F0627050000C4
S2240129E03745000037380039BC3A37B50004275C3D02340937AD3401F50F37BD4FA6379DEE
S224012A0027742774375D9500DD02379D375500029504FA02E11E3F06B604850037FA4F9CDC
S224012A20B00227030000B0B427354F9ACC163F1A27F734053FFA274FFA008BA2FCFC3786EE
S224012A4000EA850837B8000ABC0437B8FFF6378E00DA85083735000AFA02E7B48A08270565
S224012A600004850437B80039BC48F50F37BD4FA6379D37754F9C27742774375D9500DD0201
S224012A80379D3755000295043403F50F37BD508A379D3745000427742774375D9500DD029A
S224012AA0379D375500029504FA02E0AE3F04B70227030004B0A8850481088A00FCC8BF04E6
S224012AC037B500388A00B0048500BC0027050000270500043745000437380039BC44F50FC5
S224012AE037BD4FA6379D27742774375D9500DD02379D3755000295043403F50F37BD508AD1
S224012B00379D3745000027742774375D9500DD02379D375500029504FA02E0AE3F04B702A0
S224012B2027030004B0AA850437FA4F9CB006850837F14F9C37FA4F9C37F54F9CFCC8BF0650
S224012B4037B5003837FA4F9CB00637F54F9CBC0027354F9CCC063F0A27F734053FFA274F3E
S224012B6017F5533FF801B752F50F27FA27714FA637DC37AC27FA37DC8A04374A0002270596
S224012B8000008500FCC7BC288502CD04379DD500C809B60AD501C80FB604850037FA4F9C69
S224012BA0B00E270300008504FC068A04B4D027030002B0CAF50117FA517217FA33E4CC0620
S224012BC03F0A27F73F6666663AFB43D834073FF0274FC51BB70417F55174CA01B00217F5F2
S224012BE05173CA01C5013705FA0115DA8A08374A00063745001285142773004EC50137052A
S224012C00FA0115DA8A04374A00022705000E850E37B80004378C01C8C51B378700E0F50FE5
S224012C2037BD5790379D850E27F427F437DD375500009502276C3E06FA02E6BA8A0C374A55
S224012C40000AF50F37BD5790379D850E27F427F437DD850C276C3E02FA02E9509A02375A0E
S224012C600000F50F37BD579C379D850E27F427F437DD37550000F501379E950237BE2BC4E0
S224012C80FA02E662BF2AF50F37BD579C379D850E27F427F437DDF50127FA27712BC437ECA4
S224012CA037AC27FA37EC9A02375A00002703000E3780FF58F50F37BD579C379D850E27F407
S224012CC027F437DD37550000F501379E950237BE2BC8FA02E662BCD0F50F37BD579C379D5A
S224012CE0850E27F427F437DDF50127FA27712BC837EC37AC27FA37EC9A02375A0000B0A880
S224012D00F50F37BD579C379D850E27F427F437DD375500009502276C3E06FA02E6BA8A0CE5
S224012D20374A000AF50F37BD579C379D850E27F427F437DD850C276C3E02FA02E9509A0231
S224012D40375A0000F50F37BD579C379D850E27F427F437DD37550000F501379E950237BE5D
S224012D602BC4FA02E662BF26F50F37BD579C379D850E27F427F437DDF50127FA27712BC4FB
S224012D8037EC37AC27FA37EC9A02375A00003780FF18F50F37BD579C379D850E27F427F460
S224012DA037DD37550000F501379E950237BE1C8AFA02E662378CFEF2F50F37BD579C379DBA
S224012DC0850E27F427F437DDF50127FA27711C8A37EC37AC27FA37EC9A02375A000037808D
S224012DE0FEC8FA01F88CFA01A812CC103F1627F73405274F27F6B70E37F54F9AB60285029F
S224012E00FA012A3227F5FA012020CC003F0427F74000A3D73ECCCCCC40C000000005000070
S224012E202F382F6A3120315032E200000000357A00040000359835A23606363C00000000A1
S224012E4036803F800000000400003690369A388638AE0000000039D80004000039E839F258
S224012E603B1A3B42000000003C6A000500003C7A3C843CCC3D143D5A000000003DA200008A
S224012E8000033DC000003DCA00013E0C00023E50000000033E6E00003E7800013EBA0002EA
S224012EA03EEA000000033EFA00003F0400013FDA0002401234053FEE274F27F6B602CC1269
S224012EC03F1627F7F50F37BD4FA6379D37754F9C27742774375D9500DD02379DD5013705FD
S224012EE08A1037F54F9AB706F50117FA33E4050DB000F501CA0DF50F37BD4FA6379D377546
S224012F004F9C27742774375D9500DD02379DD500F808B410FA02E8003E642F2E358E3686B3
S224012F2039DE3C703DB63EF0378010E437F54F9A37BD2E1CFA02E8188514FA012A32F501C7
S224012F4027FA27711C8A37DC37AC27FA37DC27734F9EF50127FA27711C8A37DC37AC27FAEF
S224012F6037DC27734FA23780060EF50F37BD57DC379D85103735000E3726277BC51527D103
S224012F8027DA851037B8000ABC3E3735000E3726277B27D5F805BF0C85103735000E3726F9
S224012FA0277BF50527DAB06AF50F37BD57DC379D85103735000E3726277B27D5BC548510A6
S224012FC03735000E372637DD1500B046F50F37BD57DC379D85103735000E3726277B27D5EC
S224012FE0F806BF0C85103735000E3726277BF50627DAB01EF50F37BD57DC379D851037352A
S224013000000E3726277B27D5BC0885103735000E372637DD1500F50F37BD57DC379D8510B4
S2240130203735000E3726277B27D5F801B708F804B738F805B734F806B730F501379E277142
S2240130404F9E37BE2E10FA02E662378F052AF50F37BD57DC379D85103735000E372637DD92
S22401306027714F9E9A08375A00063780050AF50F37BD57DC379D85103735000E372637DD47
S2240130803755000695088A0A374A000837ECF501379E37EC37BE2E10FA02E662BF06374515
S2240130A00008850A27734F9E37B50002FA02E7DA8A02374A000037450008850A276CFA0292
S2240130C0E662BF0C37B50002FA02E7DA8A0A374A0008B02637450008F501379E850A37BE66
S2240130E02E14FA02E662BC12F50127FA27712E1437DC37AC27FA37DC8A0A374A0008F50F3A
S22401310037BD57DC379D85103735000E372637DD37450008850A9A08375A000637800458CF
S224013120F50F37BD57DC379D85103735000E372637DD342885143401375500029504FA01BE
S22401314026B43F02350A9A04375A000237800428F50F37BD57DC379D85103735000E372690
S224013160277B27D5F8013787012AF802B70EF803B70AF804B706F805B702F806378603F829
S224013180F50F37BD57DD379D85103735000E3726277BC5157506372427D127DA8510373571
S2240131A0000E3726277B27D5F80CBF0C85103735000E3726277BF50C27DAB022F50F37BD57
S2240131C057DD379D85103735000E3726277B27D5F806BC0A85103735000E3726277BF5060A
S2240131E027DAF50F37BD57DC379D85103735000E3726277B27D5F8033786037C37BD57DD60
S22401320085103735000E3726277B27D5F80CB64E37BD57DC85103735000E372637DD375563
S224013220000AF501379E950C37BE2E18FA02E662378F0344F50F37BD57DC379D8510373586
S224013240000E372637DD3755000A950C27734FA237B50006FA02E7DA9A0C375A000A378080
S2240132600316F501379E27714FA237BE2E18FA02E662378F0302F50F37BD57DC379D8510FD
S2240132803735000E372637DD27714FA29A0C375A000A378002E2F50F37BD57DC379D851044
S2240132A03735000E372637DD342885143401375500069508FA0127543F02350A9A08375A9B
S2240132C00006F50F37BD57DC379D85103735000E372637DD37550006950827734F9E3780F6
S2240132E00296F50F37BD57DC379D85103735000E3726277B27D5F804378701DCF8053787D5
S22401330001D6F806378701D0F50F37BD57E6379D85103735000E372637DD37550000950297
S224013320FA02E74081148A0EF50F37BD57DC379D85103735000E372637DD850EFA02E7DA68
S2240133409A0C375A000AF50F37BD57DC379D85103735000E3726277B27D5F803378600BAAB
S22401336037BD57DD85103735000E3726277B27D5F80C378600A437B50006FA02E7DA8A0275
S224013380374A0000F50F37BD57DC379D85103735000E372637DD3755000A950C276CFA0261
S2240133A0E662BF20F50F37BD57DC379D85103735000E372637DD37B50006FA02E7DA9A0C0C
S2240133C0375A000A378000F037B5FFF4FA02E7DA8A02374A0000F50F37BD57DC379D851068
S2240133E03735000E372637DD3755000A950C276CFA02E662378C00C0F50F37BD57DC379D4C
S22401340085103735000E372637DD37B5FFF4FA02E7DA9A0C375A000A3780009C37B5000CFE
S224013420FA02E7DA8A02374A0000F50F37BD57DC379D85103735000E372637DD3755000AA7
S224013440950C276CFA02E662BF1EF50F37BD57DC379D85103735000E372637DD37B5000C9A
S224013460FA02E7DA9A0C375A000AB04A37B5FFF4FA02E7DA8A02374A0000F50F37BD57DC7A
S224013480379D85103735000E372637DD3755000A950C276CFA02E662BC1CF50F37BD57DCC1
S2240134A0379D85103735000E372637DD37B5FFF4FA02E7DA9A0C375A000AF50F37BD57DCAA
S2240134C0379D85103735000E372637DD3755000A950C27734FA23780009E85143401F50FA9
S2240134E037BD57DC379D85103735000E372637DD375500069508FA0127543F028A0A374A50
S224013500000837B50002FA02E7DA8A02374A000037450008850A276CFA02E662BF0C37B544
S2240135200002FA02E7DA8A0A374A0008B02637450008F501379E850A37BE2E14FA02E6627A
S224013540BC12F50127FA27712E1437DC37AC27FA37DC8A0A374A0008F50F37BD57DC379D60
S22401356085103735000E372637DD37450008850A9A08375A000627734F9E37F54F9A37871F
S2240135800A8E8510FA01EE0437800A8437F54F9A37BD2E30FA02E8188514FA012A323780BC
S2240135A00A6EF50F37BD57AC379D8510373500063726277BC51527D127DA851037350006DE
S2240135C03726277B27D5F811BF0C8510373500063726277BF51127DAB01EF50F37BD57AC40
S2240135E0379D8510373500063726277B27D5BC08851037350006372637DD15008510FA010E
S224013600F1F837800A0AF50F37BD57AC379D851037350006372637DD3428851434013755F3
S22401362000029504FA0126B43F02350A9A04375A00028510FA01F1F8378009D437F54F9C3F
S224013640FA012818FCFF8A10F50F37BD5955379D37450010C51527D127DAF801BF02F5010B
S22401366027DAB012F50F37BD5955379D3745001027D5BC02851037DD15008510FA02092A3F
S2240136803780098C37F54F9A37BD2E46FA02E8188514FA012A323780097617F5517427F849
S2240136A0FA0115DA8A0A374A000817F55174B67A8514BF3AF50F37BD5790379D851027F407
S2240136C027F437DD37550000F501379E950237BE142EFA02E662BC52F50127FA2771187AFD
S2240136E037DC37AC27FA37DC276C3E08FA02E69EB038F50F37BD5790379D851027F427F4DB
S22401370037DD37550000F501379E950237BE142EFA02E662BE14F50127FA2771187A37DC00
S22401372037AC27FA37DC276C3E08FA02E69E17F55174F804B634F50127FAF50F37BD579066
S224013740379D3745001027742774375D37550000950237782BC8B60037F82BCA37DC37ACA4
S22401376027FA37DCB6048514BF0027050014F50F37BD5790379D851027F427F437DD851492
S224013780FA02E7DA276C3E08FA02E950276DFA02E556F50F37BD5790379D851027F427F40F
S2240137A037DDF50F37BE5790379E851027F427F437ED37650000A502276C3E08FA02E6BA93
S2240137C037ECF501379E37EC37BE1426FA02E620FA02E740FA02E8B2276C3E08FA02E950DA
S2240137E09A02375A0000F50F37BD5790379D851027F427F437DD37550000F501379E950216
S22401380037BE2BC4FA02E662BF24F50F37BD5790379D851027F427F437DDF50127FA277156
S2240138202BC437EC37AC27FA37EC9A02375A0000B046F50F37BD5790379D851027F427F4A8
S22401384037DD37550000F501379E950237BE2BC8FA02E662BC22F50F37BD5790379D85100E
S22401386027F427F437DDF50127FA27712BC837EC37AC27FA37EC9A02375A00008510FA014F
S224013880F8AA3780078AC51517F1517417FA5174F805BF06F50517FA51743780077217F5ED
S2240138A05174378C076A173551743780076217F54F98B614F50127FA27712E4237DC37AC06
S2240138C027FA37DC8A06374A0004B012F50127FA2771176E37DC37AC27FA37DC8A06374A68
S2240138E000048514FA02E7DA276C3E04FA02E95037ECF50F379E37EC37BE004EFA02E620FA
S2240139008A0A374A0008BF2C276C3E04FA02E6BA37ECF501379E37EC37BE1426FA02E620E6
S224013920FA02E740FA02E7DA276C3E04FA02E9508A0A374A0008B03037450008850A276CF4
S2240139403E04FA02E6BA37ECF501379E37EC37BE1426FA02E642FA02E740FA02E7DA276CAC
S2240139603E04FA02E9508A0A374A000837B5003CFA02E7DA8A02374A000037450008850AA8
S224013980276CFA02E662BF0C37B5003CFA02E7DA8A0A374A0008B02637B5FFECFA02E7DA13
S2240139A08A02374A000037450008850A276CFA02E662BC0A37B5FFECFA02E7DA8A0A374A9B
S2240139C0000837B50001340137450008850AFA012BCC3F02F501CA0D3780063437F54F9A9E
S2240139E037BD2E58FA02E8188514FA012A323780061E17F5517327F8FA0115DA8A0A374A92
S224013A000008F50F37BD579C379D851027F427F437DD8514FA02E7DA276C3E08FA02E95096
S224013A20276DFA02E556F50F37BD579C379D851027F427F437DDF50F37BE579C379E8510C1
S224013A4027F427F437ED37650000A502276C3E08FA02E6BA37ECF501379E37EC37BE14260E
S224013A60FA02E620FA02E740FA02E8B2276C3E08FA02E9509A02375A0000F50F37BD579C5F
S224013A80379D851027F427F437DD37550000F501379E950237BE2BC4FA02E662BF24F50F70
S224013AA037BD579C379D851027F427F437DDF50127FA27712BC437EC37AC27FA37EC9A02E2
S224013AC0375A0000B046F50F37BD579C379D851027F427F437DD37550000F501379E9502CD
S224013AE037BE1C8AFA02E662BC22F50F37BD579C379D851027F427F437DDF50127FA2771B6
S224013B001C8A37EC37AC27FA37EC9A02375A00008510FA01F8CA378004F6C51517F15173D9
S224013B2017FA5173F805BF06F50517FA5173378004DE17F55173378C04D61735517337804C
S224013B4004CE17F54F98B614F50127FA27712E4237DC37AC27FA37DC8A06374A0004B012B0
S224013B60F50127FA2771176E37DC37AC27FA37DC8A06374A00048514FA02E7DA276C3E04A1
S224013B80FA02E95037ECF50F379E37EC37BE004EFA02E6208A0A374A0008BF2C276C3E04A9
S224013BA0FA02E6BA37ECF501379E37EC37BE1426FA02E620FA02E740FA02E7DA276C3E046C
S224013BC0FA02E9508A0A374A0008B03037450008850A276C3E04FA02E6BA37ECF501379E3B
S224013BE037EC37BE1426FA02E642FA02E740FA02E7DA276C3E04FA02E9508A0A374A000842
S224013C0037B5003CFA02E7DA8A02374A000037450008850A276CFA02E662BF0C37B5003CCF
S224013C20FA02E7DA8A0A374A0008B02637B5FFECFA02E7DA8A02374A000037450008850A1A
S224013C40276CFA02E662BC0A37B5FFECFA02E7DA8A0A374A000827F5340137450008850AAC
S224013C60FA012BCC3F02F501CA0D378003A237F54F9A37BD2E6AFA02E8188514FA012A3255
S224013C803780011CF50F37BD5186379D8510373500063726277B27D527F881148A0EBF0298
S224013CA02705000EB008850EFC1EBC0237B5FFE28A0EF50F37BD5186379D85103735000692
S224013CC03726277BC50F27DA378000D4F50F37BD5187379D8510373500063726277B27D5D9
S224013CE0370581148A0EFCFCBF0437B500048A0EB004850EBC002705000EF50F37BD518705
S224013D00379D8510373500063726277BC50F27DA3780008CF50F37BD5188379D8510373505
S224013D2000063726277B27D5370581148A0EFC9DBF0437B500638A0EB004850EBC002705A1
S224013D40000EF50F37BD5188379D8510373500063726277BC50F27DAB044F50F37BD518A08
S224013D60379D8510373500063726277B279581148A0E37B1FC19BF0437B503E78A0EB00894
S224013D80850EFCCEBC0237B500328A0EF50F37BD518A379D8510373500063726277B850E0C
S224013DA0279A37F54F9A378702668510FA0141AE3780025C37F54F9A37BD2E7EFA02E818BC
S224013DC08514FA012A3237800084F50F37BD5176379D374500102774277427D527F88114AD
S224013DE08A0EBF022705000EB008850EFC1EBC0237B5FFE28A0EF50F37BD5176379DC50F3B
S224013E00374500102774277427DAB040F50F37BD5178379D37450010277427742795811441
S224013E208A0E37B1FC19BF0437B503E78A0EB008850EFCCEBC0237B500328A0EF50F37BD35
S224013E405178379D850E3745001027742774279A37F54F9A378701B88510FA0148C43780CA
S224013E6001AE37F54F9A37BD2E90FA02E8188514FA012A3237800198F50F37BD578C379DDB
S224013E803745001027D527F881148A0EFCFDBF0437B500038A0EB008850EFCFFBC0237B515
S224013EA000018A0E850E34018510FA01F8583F02F50717FA33FB378001568510FA0202D6C8
S224013EC081148A0EFCF7BF0437B500098A0EB004850EBC002705000E850E34018510FA02D6
S224013EE001F83F02F50717FA33FB3780012237F54F9A37BD2EA2FA02E8188514FA012A32A8
S224013F003780010C37B50002FA02E7DA8A02374A0000F50F37BD595A379D851027F427F4D5
S224013F2037DD375500009502276CFA02E6BAFA02E7408A0EFCF4BF0437B5000C8A0EB0085F
S224013F40850EFC3DBC0237B5FFC38A0E8514810E8A0EFCF4BF0437B5000C8A0EB008850E3D
S224013F60FC3DBC0237B5FFC38A0E850E37B8FFC3B624F50F37BD595A379D851027F427F496
S224013F8037DDF50127FA27711C7A37EC37AC27FA37EC9A02375A0000B028F50F37BD595AC8
S224013FA0379D851027F427F437DD850EFA02E7DA37ECF501379E37EC37BE1432FA02E95077
S224013FC09A02375A00008514BF048510FA02092AB03C8510FA02092AB034F50F37BD595554
S224013FE0379D37450010C51527D127DAF801BF02F50127DAB012F50F37BD5955379D37451F
S224014000001027D5BC02851037DD15008510FA02092A27F5FA012020C50DB618F50F37BD5F
S2240140204FA6379D37754F9C27742774375D375500009502FA019E04CC123F1627F700043B
S224014040000940824096409E40A600000003406E0002407800034080000440AE340D274F1E
S22401406027F6B74C850437BD403EFA02E81837B5FFFFFA012020B03837B50001FA012020EE
S224014080B02E37B500018A008500FA0128F827F5FA012020B01A37B500028A00B0E637B50A
S2240140A000038A00B0DE37B500048A00B0D68504FA00A492CC023F0627F70000000341149D
S2240140C0000041160001411EFFFF412437F53198FC01BE062735319827F5FA01202017F582
S2240140E05172B71A37F53198B61417F55172173351723705FCFEBD0627F5FA0120201735EF
S224014100517217F533E4B718FA00A02037BD40BAFA02E818B00A27F5FA0204ACB00227F5F0
S224014120FA01202027F73F8000003F36DB6D3F0000003E8000003E000000000000003ECA61
S224014140F4F03EDE0DED3EF460AA3EFF7CED3405274FF50137BD4126379DC503370527F48A
S22401416027F437DD375500009502CC003F0427F74120000041A00000400000003F80000079
S224014180BF000000BF8000003F00000000040000466E468846A246BC0000000046D4BD8015
S2240141A000003CF5C28FBCAAAAAA3DCCCCCC3405373FFF6E274F373500063726277537B137
S2240141C051873733000F37DC277A379DD50037058A10F50137BD4126379D851027F427F465
S2240141E027FF37DD37DDB4FE3D013755000095028A64374A0062859427F427F4277537B1B4
S224014200595A3733000F37DC277A379D9500378F00D48594373500063726277537B1518672
S2240142203733000F37DC277A379DD500378C00B6F50F37BD595A379D859427F427F427FF35
S22401424037DD37DDB4FE3D01F50F37BE5186379E859437350006372627FF37ED37EDB4FE93
S2240142603E01E50027F8FA02E7DA276DFA02E6428A60374A005E855EBF0A27F527758A6069
S224014280374A005E378000C2F50F37BD595A379D859427F427F427FF37DD37DDB4FE3D01B4
S2240142A037B5FFE2FA02E7DA276DFA02E642276C3E5EFA02E662378F0090F50F37BD595A42
S2240142C0379D859427F427F427FF37DD37DDB4FE3D0137B5FFE2FA02E7DA276DFA02E64235
S2240142E08A60374A005EB060F50F37BD5186379D859437350006372627FF37DD37DDB4FE54
S2240143003D01D50027F8FA02E7DA8A60374A005E855EBF0827F527758A60374A005EB028DC
S22401432037B5FFE2FA02E7DA8A06374A00043745005E8560276C3E04FA02E662BC0A37B54E
S224014340FFE2FA02E7DA8A60374A005E3745005EF501379E856037BE4174FA02E950340350
S224014360F50127FA2771417037DC37AC27FA37DCFA02B3563F048A5C374A005AF50137BDBA
S224014380413A379D851027F427F427FF37DD37DDB4FE3D013755000095028A58374A0056E3
S2240143A037450062F501379E856437BE417CFA02E64237ECF501379E37EC37BE4180FA02CC
S2240143C0E6BA3403F50127FA2771417837DC37AC27FA37DCFA02B3563F048A54374A005275
S2240143E0F50127FA2771417C37DC37AC27FA37DC8A50374A004E8A68374A006637B50001B2
S2240144008A148514FCF5BC26374500528554276C3E4EFA02E69E851427F427F4275C37DDE0
S2240144203745004E85509A68375A006627030014B0CC37450062F501379E856437BE417CE0
S224014440FA02E64234033745005A855CFA02B3563F048A50374A004E27050014851437B88B
S224014460000BBC1827F427F4275C37DD3745004E8550276D3E66FA02E68227030014B0D889
S22401448027050014851437B8000B378C008227F427F4275C37DD37550066F501379E956877
S2240144A037BE417CFA02E662BF24851427F427F4275C37DDF50127FA2771417C37EC37AC45
S2240144C027FA37EC9A68375A0066B00227030014B0AE851427F427F4275C37DD37550066F3
S2240144E0F501379E956837BE4184FA02E662BCD8851427F427F4275C37DDF50127FA277147
S224014500418437EC37AC27FA37EC9A68375A0066B0B627050014851437B8000BBC4227F43B
S22401452027F4275C37DD3735007F37B5FFFFFA02E8B28A06374A000437B5000B801427F49D
S22401454027F4276C37ED37650062A564276C3E04FA02E6BAFA02E7409A1C375A001A27035D
S2240145600014B0AE85142703001427F427F4275C37DD3735007F37B5FFFFFA02E8B28A0624
S224014580374A0004374500568558276C3E04FA02E6BAFA02E7409A1C375A001AF50127FAD5
S2240145A02771418837DC37AC27FA37DCFA02D44E37ECF501379E37EC37BE4170FA02E6BAF9
S2240145C08A50374A004E3745005E8560276C3E4EFA02E950FA02E740FC018A12FA02E7DAA0
S2240145E08A06374A00043745004E8550276C3E04FA02E6BA8A60374A005E37ECF501379ED9
S22401460037EC37BE4174FA02E9503403F50127FA2771417037DC37AC27FA37DCFA02B356CC
S2240146203F048A5C374A005A851427F427F4275C37DD3735007F37B5FFFFFA02E8B28A060F
S224014640374A00043745005A855C276C3E5AFA02E6BA276C3E04FA02E6BAFA02E7409A1C07
S224014660375A001A859437BD418CFA02E81837B501388A0E37B501048A0C37B501008A0AEE
S22401468037B501038A08B04837B501528A0E37B5015A8A0C37B501568A0A37B501598A0837
S2240146A0B02E37B501458A0E37B5012F8A0C37B5012B8A0A37B5012E8A08B01437B5015F31
S2240146C08A0E37B501D38A0C37B501CF8A0A37B501D28A0837B50008275C3D1A340937AD56
S2240146E0CD0E340937B50001FA0078A83F0837B50005275C3D3A340937AD3401850EFC0876
S224014700340137B50001FA0078A83F088594373500063726277537B1518A3733000F37DC3D
S224014720277A379D9500B75AF50F37BD5186379D859437350006372627FF37DD37DDB4FECD
S2240147403D019504FA02E9348A06374A0004F50127FA2771419E37DC37AC27FA37DC276C03
S2240147603E04FA02E950FA02D0628A02374A000037B50001FA02E7DA276CFA02E6428A5046
S224014780374A004EB012F50127FA277141A237DC37AC27FA37DC8A50374A004E3735007F32
S2240147A037B5FFFFFA02E8B28A06374A00043745004E8550276C3E04FA02E6BAFA02E7402B
S2240147C08A18374A001634038508FA0077FC3F048594373500063726277537B15188373377
S2240147E0000F37DC277A379DD500B75CF50F37BD5186379D859437350006372627FF37DD6F
S22401480037DDB4FE3D01D5023705FA02E7DA8A06374A0004F50127FA277141A637DC37AC1D
S22401482027FA37DC276C3E04FA02E950FA02D0628A02374A000037B50001FA02E7DA276CBC
S224014840FA02E6428A50374A004EB012F50127FA277141AA37DC37AC27FA37DC8A50374AA4
S224014860004E3735007F37B5FFFFFA02E8B28A06374A00043745004E8550276C3E04FA02F4
S224014880E6BAFA02E7408A18374A00163403850CFA0077FC3F0427F58A16FC018A183745C7
S2240148A000163403850AFA0077FCCC92373F009A27F7000400004A524A6C4A864AA000000D
S2240148C000004AB834053FE4274F27F427F4277537B1595A3733000F37DC277A379D9500FB
S2240148E0378F00D0851E27F427F4277537B151763733000F37DC277A379DD500378C00B4AB
S224014900F50F37BD595A379D851E27F427F427FF37DD37DDB4FE3D01F50F37BE5176379E66
S224014920851E27F427F427FF37ED37EDB4FE3E01E50027F8FA02E7DA276DFA02E6428A0A2C
S224014940374A00088508BF0A27F527758A0A374A0008378000C0F50F37BD595A379D851E04
S22401496027F427F427FF37DD37DDB4FE3D0137B5FFE2FA02E7DA276DFA02E642276C3E08A2
S224014980FA02E662378F008EF50F37BD595A379D851E27F427F427FF37DD37DDB4FE3D01E3
S2240149A037B5FFE2FA02E7DA276DFA02E6428A0A374A0008B05EF50F37BD5176379D851E4E
S2240149C027F427F427FF37DD37DDB4FE3D01D50027F8FA02E7DA8A0A374A00088508BF083B
S2240149E027F527758A0A374A0008B02837B5FFE2FA02E7DA8A06374A000437450008850A52
S224014A00276C3E04FA02E662BC0A37B5FFE2FA02E7DA8A0A374A000837450008F501379EBB
S224014A20850A37BE4174FA02E9503403F50127FA2771417037DC37AC27FA37DCFA02B3563C
S224014A403F048A0A374A0008851E37BD48B2FA02E81837B501078A1A37B501098A1837B547
S224014A6001088A1637B5010A8A14B04837B5015D8A1A37B5015F8A1837B5015E8A1637B547
S224014A8001608A14B02E37B501328A1A37B501348A1837B501338A1637B501358A14B01469
S224014AA037B501D68A1A37B501D88A1837B501D78A1637B501D98A143735007F37B5FFFF85
S224014AC0FA02E8B28A06374A000437450008850A276C3E04FA02E6BAFA02E7408A12374A61
S224014AE000103403851AFA0077FC3F04851E27F427F4277537B151783733000F37DC277AC7
S224014B00379D9500B758F50F37BD5176379D851E27F427F427FF37DD37DDB4FE3D019502D6
S224014B20FA02E9348A06374A0004F50127FA2771419E37DC37AC27FA37DC276C3E04FA02B8
S224014B40E950FA02D0628A02374A000037B50001FA02E7DA276CFA02E6428A0E374A000C55
S224014B60B012F50127FA277141A237DC37AC27FA37DC8A0E374A000C3735007F37B5FFFFB7
S224014B80FA02E8B28A06374A00043745000C850E2776B70037348000276C3E04FA02E6BA99
S224014BA0FA02E7408A12374A001034038518FA0077FC3F04F50127FA2771417C37DC37ACB9
S224014BC027FA37DC8A0E374A000C3735007F37B5FFFFFA02E8B28A06374A00043745000C6E
S224014BE0850E276C3E04FA02E6BAFA02E7408A12374A001034038516FA0077FC3F0427F5BD
S224014C008A10FC018A123745001034038514FA0077FCCC1C3F2427F734043FF8274F270518
S224014C2000002705000237B50001275C340937AD37BD0102340937B50001FA0078A83F082D
S224014C4027050006850637B80004B40CFA0141AE8506FA0148C427030006B0E4CC083F0A81
S224014C6027F700014FCA000153FA000151F0000150E200014E00000152FE000156D000016B
S224014C805718000157A2000158CE000159C000015D7C00015D9600015DC034043FFC274F8F
S224014CA02705000227050000374500003738000E37840102F50137BD4C62379D277427743B
S224014CC0375D37550000950237380001B60E37B858CEB60817F5317EF801B700270300007B
S224014CE0F50137BD4C62379D3745000027742774375D37550000950237380001B60E37B8B6
S224014D0059C0B60817F5317EF802B70027030000F50137BD4C62379D374500002774277402
S224014D20375D37550000950237380001B60C37B85D7CB60617F53393B60027030000F50158
S224014D4037BD4C62379D3745000027742774375D37550000950237380001B60C37B85D965A
S224014D60B60617F53393B60027030000850027F427F427753706BAFE277037B14C623733DC
S224014D80000137DC277A379D850227F427F427753706BAFE277037B151AA3733000F37EC20
S224014DA0277A379E9500AA009502AA0227030002270300003780FEEE8502FCFF37FA51E414
S224014DC0CC043F0627F74C4F434B20434F44453A00253034640050524553532053544F521A
S224014DE04520544F20554E4C4F434B0050524553532053544F524520544F204C4F434B0073
S224014E0034053FEC274F37F151A237FA51A237B1D8F1BF0637B5270F37FA51A2B00637F5D5
S224014E2051A2BC00273551A237B50003FA00C25C37B5000D3735000334033735000137B56F
S224014E404DC6FA00C1043F0437F551A234013735000137B54DD13403275C37AD3705277BF0
S224014E6037DCFA02B5CC3F0637B50013FA00C25C37B5000D37BD00403409275C37AD370533
S224014E80277B37DCFA00C1043F0437B50003FA00C25C17F5519EB71A37B50017340127F52E
S224014EA034013735000137B54DD6FA00C1043F04173551E2B01A37B5001737350003340347
S224014EC03735000137B54DECFA00C1043F04F50117FA51E2CC143F1827F741524520594F09
S224014EE05520535552453F0050524553532053544F524500544F20434F4E4649524D20216D
S224014F00000037B50001FA00AF64FA00AE7027F5FA00C25C37B500013735000A340337353F
S224014F20000137B54EDAFA00C1043F0437B5000C3735000A34033735000137B54EE8FA0026
S224014F40C1043F0437B500173735000A34033735000137B54EF4FA00C1043F0427F5FA00E0
S224014F60AF64173551E227F7340C274F37B504548A0017F5519EB72237F551A237F851A0E4
S224014F80B606273551A21735519EB01A37F551A28800B612273551A21735519EB00837FF14
S224014FA051A251A0F50117FA519E351827F74C434420434F4E54524153543A002532640050
S224014FC0252B3264002B3130000034053FF0274FFA00AE3C81128A00FCF6BF0437B5000ACF
S224014FE08A00B0088500FC0ABC0237B5FFF68A008500FA00AE2237B50003FA00C25C37B573
S22401500000518A0E37B500108A0C3735000334033735000137B54FAEFA00C1043F0485008C
S224015020B61C34013735000137B54FBC3403275C3D0237AD3705277B37DCFA02B5CC3F066F
S224015040B01C850034013735000137B54FC03403275C3D0237AD3705277B37DCFA02B5CC11
S2240150603F0637B50013FA00C25C850CFC0834013735000137B54FC5FA00C214810E340103
S224015080850CFCFF3401850EFCFFFA00B6543F06850CCD0E3409275C3D0237AD3705277B45
S2240150A037DCFA00C104CC103F1827F7000150CD000150C3000150B8536C6F77206465639B
S2240150C06179005065616B20686F6C64004E6F726D616C2066617374005655204D4F444581
S2240150E03A0034053FEE274FF50137BD50AC379D276CF50CFA02E91617F50FA237058114BD
S2240151008A0CFCFEBF0437B500028A0CB004850CBC002705000CC50D17FA0FA237B50003F6
S224015120FA00C25C37B500338A1037B500108A0E3735000334033735000137B550D9FA00E2
S224015140C1043F0437B50013FA00C25C850E3745001034033745000C27742774275C375DFF
S224015160375500009502FA00C1043F043745000C27742774275C375D375500009502FA0012
S224015180C21481108A10FC87BE14850EFC0837BD00793409850EFCFF34018510FA00B65416
S2240151A03F06CC123F1627F7000151C7000151BA000151B4566F6C7473006442752028307D
S2240151C02E37373556290064422066726F6D20636C697000434F4D50522026204C494D4925
S2240151E0542054485245534800554E49543A000034053FEE274FF50137BD51A8379D276CC7
S224015200F50CFA02E91617F50052370581148A0CFCFEBF0437B500028A0CB004850CBC0085
S2240152202705000CC50D17FA005237B50003FA00C25C37B5000D37350003340337350001E8
S22401524037B551D4FA00C1043F0437B500173735000F34033735000137B551E9FA00C1042E
S2240152603F0437B50013FA00C25C37B500328A1037B500178A0E3745001034033745000C30
S22401528027742774275C375D375500009502FA00C1043F043745000C27742774275C375DC1
S2240152A0375500009502FA00C21481108A10FC87BE14850EFC0837BD00793409850EFCFFA6
S2240152C034018510FA00B6543F06CC123F1627F7000152E3000152D846616872656E6865E2
S2240152E069740043656C736975730054454D504552415455524520554E49543A00003405D2
S2240153003FF2274FF50137BD52D0379D276CF508FA02E91617F54F98370581108A08FCFF28
S224015320BF0437B500018A08B0048508BC0027050008C50917FA4F9837B50003FA00C25C27
S22401534037B5000D3735000334033735000137B552EBFA00C1043F0437B50013FA00C25CF9
S22401536037B500288A0C37B500178A0A3745000C34033745000827742774275C375D3755CA
S22401538000009502FA00C1043F043745000827742774275C375D375500009502FA00C214AA
S2240153A0810C8A0CFC87BE14850AFC0837BD00793409850AFCFF3401850CFA00B6543F0699
S2240153C0CC0E3F1227F7000153E7000153DD000153D273757065727669736F720046756C63
S2240153E06C2065646974004E6F20656469740045444954204D4F44453A0034053FEE274F71
S224015400F50137BD53C6379D276CF50CFA02E91617F50053370581148A0C8514B71A850C5F
S224015420FCFFBF0437B500018A0CB004850CBC002705000CC50D17FA0053B012850CFCFE69
S224015440BF0437B500028A0CB004850CBC002705000C37B50003FA00C25C37B5003F8A10FA
S22401546037B500108A0E3735000334033735000137B553EFFA00C1043F0437B50013FA0056
S224015480C25C850E3745001034033745000C27742774275C375D375500009502FA00C104DB
S2240154A03F043745000C27742774275C375D375500009502FA00C21481108A10FC87BE145B
S2240154C0850EFC0837BD00793409850EFCFF34018510FA00B6543F06CC123F1627F74D49FD
S2240154E04449205258204348414E4E454C3A004F6666004F6D6E6900253264004D49444970
S224015500205458204348414E4E454C3A004F666600253264000034053FF0274F37B50003C3
S224015520FA00C25C37B5005F8A0E37B5000D8A0C3735000134033735000137B554DEFA00B2
S224015540C1043F0417F50024F8FEB726F8FFB73E17F500243705FC0134013735000137B557
S22401556054F83403275C37AD3705277B37DCFA02B5CC3F06B0323735000137B554EF3403D3
S224015580275C37AD3705277B37DCFA02E0D03F04B0163735000137B554F33403275C37ADBA
S2240155A03705277B37DCFA02E0D03F04C513F801B60637B50010FA00C25CB00227F5FA009C
S2240155C0C25C850CCD0E3409275C37AD3705277B37DCFA00C1043F04275C37AD3705277B5F
S2240155E037DCFA00C214810E8A0EFC87BE14850CFC0837BD00793409850CFCFF3401850EB3
S224015600FA00B6543F0637B50003FA00C25C37B5005F8A0E37B500178A0C37350001340314
S2240156203735000137B554FCFA00C1043F0417F51004F8FFB6183735000137B5550D3403E2
S224015640275C37AD3705277B37DCFA02E0D03F04B02017F510043705FC0134013735000132
S22401566037B555113403275C37AD3705277B37DCFA02B5CC3F06C513F802B60637B50010F7
S224015680FA00C25CB00227F5FA00C25C850CCD0E3409275C37AD3705277B37DCFA00C10446
S2240156A03F04275C37AD3705277B37DCFA00C214810E8A0E850CFC0837BD00793409850C82
S2240156C0FCFF3401850EFA00B654CC103F1A27F7340D274F17F5002437058A00F9F0B7025B
S2240156E037B1FF008A00850481008A00FCF1BF0437B5000F8A00B0088500FC02BC0237B585
S224015700FFFE8A00C50117FA002437B50001FA015516CC023F0627F7340D274F17F51004A6
S22401572037058A00F9F0B70237B1FF008A00850481008A00FCF1BF0437B5000F8A00B00809
S2240157408500FC01BC0237B5FFFF8A00C50117FA100437B50002FA015516CC023F0627F71F
S22401576000015789000157810001577800015770546F20626F746800546F20525332333222
S22401578000546F204D494449004F66660053454E442045444954454420504152414D533ACB
S2240157A0000034053FE8274FF50137BD5760379D276CF510FA02E91617F50194370527F40D
S2240157C017F1533C7300811A8A1217F5317EB700F802B60E37B500018A1085128810BF0AD3
S2240157E085108A12B00C37B500028A10B0E88512BC00270500128512F901B704F50117FAB2
S224015800533CB0001735533C8512F902B704F50117FA0194B0001735019437B50003FA0005
S224015820C25C37B5000D3735000334033735000137B5578DFA00C1043F0437B500468A1694
S22401584037B500178A1437B50013FA00C25C85143745001634033745001227742774275CE1
S224015860375D375500009502FA00C1043F043745001227742774275C375D3755000095026B
S224015880FA00C21481168A16FC87BE148514FC0837BD007934098514FCFF34018516FA0001
S2240158A0B6543F06CC183F1C27F7000158BA000158B6000000004F6E20004F666600525377
S2240158C032333220544F204D4944493A000034053FEE274FF50137BD58AA379D276CF50CBB
S2240158E0FA02E91617F5533D370581148A0CFCFFBF0437B500018A0CB004850CBC00270536
S224015900000CC50D17FA533D37B50003FA00C25C37B5005A8A1037B500108A0E3735000318
S22401592034033735000137B558BEFA00C1043F0437B50013FA00C25C850E3745001034034C
S2240159403745000C27742774275C375D375500009502FA00C1043F043745000C2774277489
S224015960275C375D375500009502FA00C21481108A10FC87BE14850EFC0837BD0079340956
S224015980850EFCFF34018510FA00B6543F06CC123F1627F73A0052533438352044657669E7
S2240159A063652000253264004F46460043757272656E742047726F7570003A00253264005E
S2240159C034053FF2274F37F1019A8A0837B1FF01BF0437B500FF8A08B0048508BC0027053B
S2240159E00008850837FA019A37B50003FA00C25C37B5005A8A0C37B5000E8A0A373500540F
S224015A0034033735000137B55994FA00C1043F04850A3735000334033735000137B5599684
S224015A20FA00C1043F0437F5019AB71A34013735000137B559A43403275C37AD3705277BBF
S224015A4037DCFA02B5CC3F06B0163735000137B559A83403275C37AD3705277B37DCFA02C0
S224015A60B5CC3F0437B50013FA00C25C850ACD0C3409275C37AD3705277B37DCFA00C10489
S224015A803F04275C37AD3705277B37DCFA00C214810C8A0CFC87BE14850AFC0837BD00791D
S224015AA03409850AFCFF3401850CFA00B6543F0637B500188A0A37B50013FA00C25C850ACC
S224015AC03735000334033735000137B559ACFA00C1043F0437B50003FA00C25C850A3735B8
S224015AE0005434033735000137B559BAFA00C1043F0437B50013FA00C25C37F5019C340192
S224015B003735000137B559BC3403275C37AD3705277B37DCFA02B5CC3F06850A37BD005AE3
S224015B203409275C37AD3705277B37DCFA00C1043F0437B50003FA00C25CFA009568FA00D0
S224015B4047BACC0E3F1227F7434F4E5441435420494E5445524641434500434E5443543A82
S224015B602000253275003D3E2050474D3A20004F6666005525303275004625303275004D5F
S224015B807574650034053FEE274F27F5FA00C25C37B5000D3735000134033735000137B5AB
S224015BA05B48FA00C1043F04851437F151A637FA51A6FCF8BF0637B5000837FA51A6B00CC9
S224015BC037F551A6FCFFBC0437B5000137FA51A637B500268A1037B500178A0E3735000118
S224015BE034033735000137B55B5AFA00C1043F0437F551A634013735000137B55B623403B3
S224015C00275C37AD3705277B37DCFA02B5CC3F06C51DF801B60437B50010FA00C25C850E28
S224015C20CD103409275C37AD3705277B37DCFA00C1043F0437B50003FA00C25C373500383F
S224015C40374A0010850E34033735000137B55B66FA00C1043F04F50F37BD338B379D3DFF01
S224015C60377551A627D53705811A8A0CFCAFBF0437B500518A0CB004850CBC002705000C98
S224015C80F50F37BD338B379DC50D3DFF377551A627DA850CB6183735000137B55B6F340309
S224015CA0275C37AD3705277B37DCFA02E0D03F04B064850C37B8001EBE1A3401373500016B
S224015CC037B55B733403275C37AD3705277B37DCFA02B5CC3F06B03E850C37B80050BE1C1B
S224015CE0FCE234013735000137B55B793403275C37AD3705277B37DCFA02B5CC3F06B01647
S224015D003735000137B55B7F3403275C37AD3705277B37DCFA02E0D03F04C51DF802B60436
S224015D2037B50010FA00C25C37BD00628D10850E3409275C37AD3705277B37DCFA00C1046F
S224015D403F0427F5FA00C25C275C37AD3705277B37DCFA00C21481108A10FC87BE14850E8B
S224015D60FC0837BD00793409850EFCFF34018510FA00B6543F06CC123F1627F73405274FCE
S224015D8037B50001340127F534018502FA015B84CC003F0827F73405274F37B50002CD028C
S224015DA0340927F5FA015B84CC003F0827F7534F465457415245205245563A00257300002F
S224015DC034053FE8274F37B50003FA00C25C37B500518A1637B500108A14373500033403C3
S224015DE03735000137B55DAEFA00C1043F043735000037B5447634033735000137B55DBC7C
S224015E003403275C37AD3705277B37DCFA02B5CC3F0837B50001FA00AF648514CD16340976
S224015E20275C37AD3705277B37DCFA00C1043F0427F5FA00AF64CC183F1C27F720204849AB
S224015E4020464F4C4B53202120205448414E4B20594F5520464F52205553494E4720544820
S224015E6049532050524F434553534F522021202E2E20204D414445204259202E2E2E2047C0
S224015E80204B5241555353202E2E2E2046204C45524D4552202E2E2E2057204B415550207A
S224015EA02E2E2E202020494620594F552048415445205448452055534552494E54455246DC
S224015EC04143452C20555345205448452046414D4F55532057494E444F575320454449543D
S224015EE04F522046524F4D204D52204D2041554D45522C202E2E20594F555220534C415674
S224015F004550524F4752414D4D455253204A4C20464620414E44204D4155203A2D293E3E63
S224015F20202000003735000137B55E3CFA0203C227F74F5054494F4E204D4F4445003C20CF
S224015F403E0020203E003C202000FA00AE7027F5FA00C25C37B500013735000334033735B8
S224015F60000137B55F32FA00C1043F0437B500013735005A34033735000137B55F3EFA00C1
S224015F80C1043F0437F551A4B61437B500013735005A34033735000137B55F42FA00C10465
S224015FA03F0437F551A437F851E4B61437B500013735005A34033735000137B55F46FA0067
S224015FC0C1043F0427F7000000035FF00000601A0001600EFFFF602E3405274F17F5519E24
S224015FE0B700273551A2850237BD5FC6FA02E81837F551A437F851E4BF0437FF51E451A451
S224016000B02837F551A4BC22273551A4B01C273151A4BC16273551A4B010273351A437F5DB
S22401602051A437F851E4BF0237FF51E451A4FA015F4AF50F37BD51AA379D27F5377551A4B8
S22401604027742774375D277A9500DD02379D277AFA02E532CC003F0427F73405274F27F6DA
S224016060B72A37B50003FA00C25CF50F37BD51AA379D8502377551A427742774375D277AD8
S2240160809500DD02379D277AFA02E532FA0203FECC003F0427F70008000260E460EE60F6E2
S2240160A0616660F861666166613E0000000061663405274F37F5319637F051A837B8001402
S2240160C0B50637FF319651A8FA0203FE8502B602CC003F0427F7FA0203B4850237BD60967C
S2240160E0FA02E81837B5FFFFFA015FD8B07A37B50001FA015FD8B070F50F37BD51AA379D52
S224016100377551A427742774375D37550000950237380001B61C37B84E00B61617F551E261
S224016120B60AFA014F6837B50005FA00A492B038FA014F02B0328502FA00A492B02AF50F1B
S22401614037BD51AA379D377551A427742774375D37550000950237380001B60637B85DC0B0
S224016160B600FA015F248502FA00A492CC003F0427F737F53198FC01BE062735319827F50A
S224016180FA015FD817F55172B71A37F53198B61417F55172173351723705FCFDBD0627F578
S2240161A0FA015FD81735517227F7000161B600000000000178E60020090A003B2F2E2E000A
S2240161C022220000000161D6000161D3000161D025780025580025750000000161E50001DA
S2240161E061E24F4E004F46460000000161F6000161F2594553004E4F000000016207000139
S2240162006202545255450046414C5345002A2A2A20455620445833382000636F6D6D616E6E
S22401622064206D6F646520656E7465726564202A2A2A0000FA016D903735000137B5620DCA
S224016240FA009CAE3735000F37B5525A27735252277352563735000137B5621AFA017268B7
S224016260F50F27FA3735000137B561AA277351F237AC27FA173552123735000137B56288BB
S2240162802773532227F727F7340C274F3820317F39C000263A0400260052F501CA01C50193
S2240162A017F85212B23AF50127FA17F561BC277A37AC27FA277A3705FA009B2EF50F37BDFC
S2240162C051F2379DC5013705277B27742774375D9500DD02379D375500009502FA009CAE84
S2240162E00301B0B637B5003EFA009B2E3735000F37B5525A277352523735000137B563082C
S22401630027735322351827F734043FFC274F27F5FA0167AA27F6378701423820317F37355A
S224016320000137B561B734033735000F37B5525AFA02E1723F04277537B1525A3733000FCD
S22401634027735256F50127FA17F561BB277A37AC27FA277A3705340127715256FA02E4904F
S2240163603F028A02374A0000B6FE27F6B708850037FA5252850237FA525437F5525837F084
S224016380525437F5525637F25252B43E37F55254FCFF37FA525437F5525237B3FFFF37FA31
S2240163A0525217FD5254379DD500370534013735000137B561B7FA02E4903F022776B6B634
S2240163C027F6B6B227335254B6002733525237F5525217FD5254379D150037F5525617FD23
S2240163E05258379DD500F840B60E27335258B60027335256F50117FA51E6B000173551E61B
S22401640037F5525617FD5258379DD500F8EBB61A27335258B6002733525627715256FA0191
S224016420C1AE27735256F50117FA51E7B000173551E737F5525837F0525437F5525637F292
S2240164405252B40A3735000137B5646E27735322B0083735000137B5628827735322CC04C0
S2240164603F0627F7252E337300256325730034043FF0274F3735000137B56288277353226B
S224016480F50F37BD51F2379D17F55212370527F427F437DD3755000095028A0E374A000CA9
S2240164A037F5525617FD5258379DD500F83F378700CA2771525634033735000137B5646444
S2240164C03403275C3D0637AD3705277B37DCFA02B5CC3F083735000137B561B73403F50182
S2240164E027FA17F561BC277A37AC27FA277A370534013735000137B564693403275C37ADD1
S2240165003705277B37DCFA02B5CC3F0A275C340837AD34013D0637AD3705277B37DCFA02D2
S224016520E0F03F04275C27FF37DD37DDB4FE3D011506850CCD0E379D950A9708B66C37F59A
S224016540525617FD5258379DF50127FAD50017F861BC277A37AC27FA277AB74E373500012B
S22401656037B561BD3403275C3D0637AD3705277B37DCFA02E0AE3F0437860096B02C850CAC
S224016580CD0E379D950A9708B70A37550008950AFA016CA2378000AC37B50001340137450A
S2240165A0000C850EFA016D543F023780009627715256277352183735000137B561B7340300
S2240165C027715256FA02E0F03F04277537F1525837735256277352143735000137B561B735
S2240165E0340327715214FA02E1723F04277537F15216377352142773525637F5521417FDAA
S2240166005216379D15003735000137B5664C27735322B02E3735000137B561C034032771E2
S2240166205256FA02E0AE3F04B60837F5525617FD5258379D150027F534013745000C850E3A
S224016640FA016D543F02CC103F1227F734043FFC274FF50127FA17F561BC277A37AC27FA1E
S224016660277A3705340127715218FA02E4903F028A02374A00008700B7068500CD02379DD6
S2240166801500B00837F552148A0037F552168A02850037F85218B620850237F8521AB61807
S2240166A0F50F27FA3735000137B561AA277351F237AC27FA173552123780008C373500010A
S2240166C037B561BD340327715218FA02E0AE3F04B60817F55212B76E17315212B0682771F5
S2240166E05218FA017656F50F37BD51F2379D17F55212370527F427F437DD9500DD02379D16
S224016700950A9708B72E277152183403F50F37BD51F2379D17F552123705277B2774277484
S224016720375D9500DD02379D37550008950AFA0169243F0427F6B60EFA0172AC3735000112
S22401674037B5628827735322B052850237F05216850037F25214B4188500CD02379DD50158
S224016760B70E374500008502FC013733000027735218B02837F5525837F0525437F5525691
S22401678037F25252B40A3735000137B5646E27735322B0083735000137B562882773532224
S2240167A0CC043F0627F70820080034053FFC274FF564CA01FA009AE827F63787015C0101AC
S2240167C037870156FA009D64CA03B7E4F808B754F80AB7DCF80D3787008EF8EB378700C2E7
S2240167E037F5525437B0532137F5525237B2000FB4BE37F5525217FD5254379DC5032733AC
S2240168005254B60027335252DA003A200026FFA4C507B70637B5002AFA009B2EB092C503AF
S2240168203705FA009B2EB0883735000F37B5525A37F05254377252523784FF7637F55254EC
S22401684037B0000137FA525437F5525237B2000037FA52523A200026FF5A3735000137B5B3
S22401686067A6FA009CAE3780FF4817F50026F920B700FA016D9037F5525217FD5254379D6B
S224016880150017F5533DB70E17F551E6B6083735000F37B5525AFA0090DE37B5FFFFCC0446
S2240168A03F0827F737F5525437B0532137F5525237B2000FB41437F5525217FD5254379D52
S2240168C0C50327335254B60027335252DA000502C502F8043784FEDAFA009AE827F6B7307F
S2240168E00101B72C37F5525437B0532137F5525237B2000FB41AFA009D64277A37F552527E
S22401690017FD5254379D277A27335254B60027335252DA000302B0B43780FE9627F5CC0414
S2240169203F0827F734073FFA274F8508CD0A379D950297003787015805013735000137B526
S22401694061C48A04374A0002850437B061D0850237B20001B4388502CD04379D3755000045
S224016960950234038508CD0A379D375500009502FA02E1A03F042776B6FE27F6B702F5010B
S224016980CA01B00A8504FC048A04B4B827030002B0B2C501378700848508CD0A379D950680
S2240169A09704B7763735000F37B551EC34033755000095023403374500108512FA02B734CA
S2240169C03F08FCFFB670850837FA51EECD0A17BD51F0379D9504DD06379D27F5FA02E5320D
S2240169E037F551EE8808B60237F551F0880AB74637F551EE17FD51F0379D3755000095022B
S224016A003403374500108512FA02E0AE3F04B62637F551EE8A0837F551F08A0AB02885080A
S224016A20CD0A379D3755000095023403374500108512FA02E0AE3F04B70C850AFC0C8A0A6D
S224016A40B400270300083780FEDE8508CD0A379D950A9708B70E95069704B7089504DD060B
S224016A60379D27F5FA02E532F50F37BD51F2379D1733521217F55212370527F427F437DD5A
S224016A8037450008850A9A02375A000037B50001B0FE27F5CC063F0C27F7340F274F37F5D9
S224016AA051EC800C8A00850C880EB23A850E800C8800B53237F551EC340137F551EE17FDBF
S224016AC051F0379D37550000950234038504CD06379D375500009502FA02B5CC3F068504A3
S224016AE037FA51EE850637FA51F08500CC023F0827F73405274F37FA51EA850837FA51E859
S224016B00CC003F0427F72E2E2E0034073FF2274F05013735000137B561C48A04374A000241
S224016B20850437B061D0850237B20001B4388502CD04379D37550000950234038510CD1257
S224016B40379D375500009502FA02E1A03F042776B6FE27F6B702F501CA01B00A8504FC044D
S224016B608A04B4B827030002B0B2C5013787010C8510CD12379D95069704378700FE950423
S224016B80DD06379D37B50001FA02E53237F551EA37F851E8B26434018510CD12379D37554A
S224016BA000009502340337450018851AFA02B5CC3F068A0C3735000137B56B063403850CE4
S224016BC02775811A37430018FA02B5CC3F04810C8A0C37F551E834018510CD12379D375595
S224016BE0000095023403850C2775811A37430018FA02B5CC3F06810C8A0C3780009A85109C
S224016C00CD12379D375500009502340337450018851AFA02E0D03F048502CD04379D375587
S224016C2000009502340337450018851AFA02E1A03F048A08374A0006B6FE27F6B72E850237
S224016C40CD04379D375500009502FA02E4B68A0A850A2701000A27F6B7128506CD08379D61
S224016C60F53F27030008B60027030006DA00B0DC37450018851AFA02E4B68A0CB0188510A0
S224016C80CD12379D375500009502340337450018851AFA02B5CC3F048A0C850CCC0E3F149A
S224016CA027F73407373FFF0A274FF520CA06275C3D07340837AD3401374500F885FAFA0191
S224016CC06B0A3F04FC018A0485FAFC0C8AFAB400270300F885F8CDFA379D95029700B7404D
S224016CE0F52C37450004270300047C0627CA275C3D06370537AD8A008D02850427758102A5
S224016D00374300003403374500F885FAFA016B0A3F0481048A0485FAFC0C8AFAB4B2270368
S224016D2000F8B0AC275C3D0637AD3705277B37DCFA0172BACCF6373F00FC27F76E6F742074
S224016D4079657420696D706C656D656E746564202E2E2E003407274F37DC277A379D9506A9
S224016D609704B716C50B3705277A8502CD04379D9504DD06379D277AFA02E532B0083735A4
S224016D80000137B56D3CFA0172BACC003F0627F737B5000DFA009B2E3A080026000837B5E9
S224016DA0000AFA009B2E27F725690000340F274F27050000275C340837AD3401373500012A
S224016DC037B56DA8340327715256FA02B7343F08FCFFB618850037B1008037B80100B40CA1
S224016DE08504CD06379DC501DA0037B50001B002FA0172AC27F5CC023F0827F72569000028
S224016E00340F274F27050000275C340837AD34013735000137B56DFC340327715256FA027A
S224016E20B7343F0837B80001B61CC50D27F88800BE14C50F27F88800BD0C8504CD06379D99
S224016E40C501DA0037B50001B002FA0172AC27F5CC023F0827F725750000340F274F270506
S224016E600000275C340837AD34013735000137B56E56340327715256FA02B7343F08FCFF77
S224016E80B614850037B80100B40C8504CD06379DC501DA0037B50001B002FA0172AC27F549
S224016EA0CC023F0827F725750000340F274F27050000275C340837AD34013735000137B5E9
S224016EC06EA6340327715256FA02B7343F08FCFFB61AC50D37058800B212C50F8800B50CB1
S224016EE08504CD06379DC501DA0037B50001B002FA0172AC27F5CC023F0827F74F464600DA
S224016F003407274F27715256FA0176563735000137B56EFC340327715256FA02E0AE3F04AC
S224016F20B60A8502CD04379D150037B50001B006374500028504FA016E5ACC003F0627F7AE
S224016F4025780000340F274F27050000275C340837AD34013735000137B56F4034032771FA
S224016F605256FA02B7343F08FCFFB60C8504CD06379DC501DA0037B50001B002FA0172ACF0
S224016F8027F5CC023F0827F725690000340F274F27050000275C340837AD340137350001E4
S224016FA037B56F88340327715256FA02B7343F08FCFFB60C8504CD06379D85009A0037B54B
S224016FC00001B002FA0172AC27F5CC023F0827F725750000340F274F27050000275C340852
S224016FE037AD34013735000137B56FD0340327715256FA02B7343F08FCFFB60C8504CD061C
S224017000379D85009A0037B50001B002FA0172AC27F5CC023F0827F725750000340F274F1D
S22401702027050000275C340837AD34013735000137B57018340327715256FA02B7343F08C0
S224017040FCFFB6188500880CB512880EB20E277A8504CD06379D277A9A0037B50001B00280
S224017060FA0172AC27F5CC023F0827F74F4646003407274F27715256FA01765637350001A2
S22401708037B5706C340327715256FA02E0AE3F04B60C8502CD04379D2715000037B50001C7
S2240170A0B006374500028504FA016FD4CC003F0627F72566000034073FFC274F27F5277571
S2240170C08A02374A0000275C340837AD34013735000137B570B2340327715256FA02B734EC
S2240170E03F08FCFFB614374500008506CD08379D85029A02375A000037B50001B002FA0180
S22401710072AC27F5CC043F0A27F72566000034073FFC274F275C340837AD3401373500013C
S22401712037B5710A340327715256FA02B7343F08FCFFB634374500008502276C3E0EFA027A
S224017140E662BD24374500008502276C3E12FA02E662BE14374500008506CD08379D8502CD
S2240171609A02375A000037B50001B002FA0172AC27F5CC043F0A27F7340F274F27715256D8
S224017180FA0176560501C501C811B426850CCD0E379DC5013705277B27742774375D375569
S2240171A000009502340327715256FA02E0AE3F04B7000301B0CCC501C811B40E277A85042C
S2240171C0CD06379D277ADA0037B50001B002FA0172AC27F5CC023F0827F73407274F37B5E3
S2240171E0000234013735000137B561DA3403374500028504FA017178CC003F0C27F734072C
S224017200274F37B5000234013735000137B561EA3403374500028504FA017178CC003F0CF2
S22401722027F73407274F37B5000234013735000137B561FA3403374500028504FA01717880
S224017240CC003F0C27F73407274F850A3401277152563403374500028504FA02E14A37B5ED
S2240172600001CC003F0C27F7340F274F37450004850627030006B6002703000437DC277A46
S224017280379DD500CA01B7043705FA009B2EB0D837B5000DFA009B2E37B5000AFA009B2EBD
S2240172A0CC023F0827F73B203F2000003735000137B572A6FA01726827F7340F274FF501C8
S2240172C0CA01C50117F85212B22C37B5002FFA009B2EF50F37BD51F2379DC5013705277B35
S2240172E027742774375D9500DD02379D375500009502FA009CAE0301B0C437B50020FA0091
S2240173009B2E374500048506FA017268CC023F0827F73405274F3716B700F501CA03F5011F
S22401732037BD61DA379DC5033705277B27742774375D375500009502FA0172BACC003F047B
S22401734027F73405274F3716B700F501CA03F50137BD61EA379DC5033705277B27742774AE
S224017360375D375500009502FA0172BACC003F0427F73405274F3716B700F501CA03F50190
S22401738037BD61FA379DC5033705277B27742774375D375500009502FA0172BACC003F04FB
S2240173A027F72569000034053FFA274F27F834013735000137B573A23403275C37AD370597
S2240173C0277B37DCFA02B5CC3F06275C37AD3705277B37DCFA0172BACC063F0A27F72575DE
S2240173E0000034053FFA274F370534013735000137B573DE3403275C37AD3705277B37DCF5
S224017400FA02B5CC3F06275C37AD3705277B37DCFA0172BACC063F0A27F74F4646003405D8
S224017420274F3716B60A3735000137B5741AFA0172BAB004C5033705FA0173E2CC003F049E
S22401744027F725303258000034053FFA274F370534013735000137B574423403275C37AD23
S2240174603705277B37DCFA02B5CC3F06275C37AD3705277B37DCFA0172BACC063F0A27F79B
S2240174802569000034053FF8274F34013735000137B574803403275C37AD3705277B37DC61
S2240174A0FA02B5CC3F06275C37AD3705277B37DCFA0172BACC083F0C27F725750000340575
S2240174C03FF8274F34013735000137B574BA3403275C37AD3705277B37DCFA02B5CC3F06EC
S2240174E0275C37AD3705277B37DCFA0172BACC083F0C27F74F4646003405274F27F6B60A63
S2240175003735000137B574F4FA0172BAB0028502FA0174BECC003F0427F7256C69003407B5
S2240175203FF4274F34033735000137B5751A3403275C37AD3705277B37DCFA02B5CC3F082A
S224017540275C37AD3705277B37DCFA0172BACC0C3F1227F7256700252E2A660034073FD89E
S224017560274F8532BD0237B80008BF323745002A852C34033735000137B575543403275CC7
S22401758037AD3705277B37DCFA02B5CC3F08275C37AD3705277B37DCFA0172BACC283F2E6C
S2240175A027F73745002A852CCD32340B3735000137B575573403275C37AD3705277B37DC5E
S2240175C0FA02B5CC3F0AB0C23407274F37B500013401374500028504FA01755CCC003F08B4
S2240175E027F73407274F37B500033401374500028504FA01755CCC003F0827F7252D2E2AE4
S22401760073003407373FFF36274F85D437B800C8B30237B500C88AD4374500CC85CECDD482
S224017620340B3735000137B575FC3403275C3D0137AD3705277B37DCFA02B5CC3F0A275C25
S2240176403D0137AD3705277B37DCFA0172BACCCA373F00D027F734073FFC274F8A02374AF7
S22401766000008500CD02379DD500B71A3705FA02E4CA277A8500CD02379D277ADA002703E2
S2240176800002B6DA27030000B0D4374500068508CC043F0A27F7000176C10001831C000086
S2240176A00000000176BA0001836800000000000000000000000000000000555345522575CE
S2240176C00046414354257500000177A400017CF4000000000001779D00017D9C0000000030
S2240176E00001779200017E08000000000001778400017C2A000000000001777500017C8E58
S224017700000000000001776900017E5A000000000001775800017F06000000000001774992
S22401772000017F70000000000001774000000000000176960000000000000000000000008E
S22401774050524F474C495354005448524553484F4C445F554E49540054454D504552415401
S2240177605552455F554E49540054454D50455241545552450044454C41595F4F55545F55B0
S2240177804E49540044454C41595F494E5F554E49540050524F474E554D42455200434F4E13
S2240177A04649470050524F474E414D4500000001781100017FDA000000000001780C00012A
S2240177C0801400000000000178070001804E0000000000017801000180A60000000000011E
S2240177E077F6000183A80000000000000000000000000000000053494C454E544D4F4445F6
S224017800005052494E540044554D50004C4F41440053544F524500000001785400017BA801
S224017820000000000001784D00017BB8000000000001784800017BC8000000000000000043
S22401784000000000000000004543484F0050524F4D5054004C494E454645454400000001E4
S22401786078E300017A2000000000000178DE00017A8C00000000000178D800017AF60001EB
S2240178808530000178D200017B3E00000000000178CD00000000000176C8000178C5000065
S2240178A00000000177AE000178BE0001842400000000000000000000000000000000444533
S2240178C05649434500434F4D4D414E44004D495343004F5554257500494E53554D00494E9B
S2240178E02575005655000001792600017A36000000000001791E00000000000178180001C2
S224017900791600000000000196380000000000000000000000005345525649434500434F60
S2240179204D434F4E4600494425750056550034043FE4274F3735000137B5792B3403275C74
S2240179403D0137AD3705277B37DCFA02E0D03F042705001A851A37B80006378C0084FA0004
S224017960897C8A18C518CA17851AFCFEB60EC5173705277BF506277D3711B6F627FBCA16F0
S224017980851AFCFDB610C517370527FD27FD27FD27FD3705F60CC116CA16851AFCFCB60E8B
S2240179A0C5173705277BF506277D3711B6F627FBCA15851AFCFBB610C517370527FD27FDB7
S2240179C027FD27FD3705F60CC115CA15C517F63FCA17F7403745001A7C0327CA2703001AF3
S2240179E03780FF6EC516F770CA09C515F770CA0A050B17F551E6B70E275C3D0137AD37053A
S224017A00277B37DCFA0090DEB00C275C3D0137AD3705277B37DCFA017268CC1C3F1E27F7B9
S224017A203716B700FA01792E27F7000F521C000000000001785E3716B70E37B500FF3401F6
S224017A4037B50001FA016AF23F02B02E37B500FF3735000134033735000137B57A2AFA0136
S224017A606A9A3F04277AF50F27FA277A37FA522C277A37AC27FA277AFC0137FA532A27F794
S224017A80000F522E00000000000185003716B70E37B50002340137B50001FA016AF23F0211
S224017AA0B02C37B500023735000134033735000137B57A80FA016A9A3F04277AF50F27FAF7
S224017AC0277A37FA523E277A37AC27FA277A37FA5328F50117FA100237B5000137BD000151
S224017AE0340937B5008237F05328FA0083EA3F041735100227F737B5000237FA5328F5017D
S224017B0017FA100237B5000137BD0001340937B50082FA0083EA3F0437B5000137BD000123
S224017B20340937B50081FA0083EA3F041735100227F7000F522E0000000000018684371688
S224017B40B70E37B50004340137B50001FA016AF23F02B02C37B500043735000134033735D4
S224017B60000137B57B32FA016A9A3F04277AF50F27FA277A37FA523E277A37AC27FA277AB5
S224017B8037FA5328F50117FA100237B5000137BD0001340937B5000537F05328FA0083EA01
S224017BA03F041735100227F73705340137B50008FA017BD83F0227F73705340137B500048D
S224017BC0FA017BD83F0227F73705340137B50020FA017BD83F0227F734053FD4274FC5350C
S224017BE0B70EC52F37058A0017F500268600FA017312B02C275C3D0337AD3705277B37DC54
S224017C00FA0171DA27F6B718C503B708C52F17F7002617FA0026B008C52F371017F6002620
S224017C2017FA0026CC2C3F3027F7340D274F3716B71EF50F37BD0164379D17F5517427F888
S224017C40277B27742774375D375500009502FA0172BAB03027715256FA01765637B500068F
S224017C6034013735000F37B501643403275C3D0137AD3705277B37DCFA0171783F0627F6EA
S224017C80B702C50117FA5174CC023F0627F7340D274F3716B71EF50F37BD0164379D17F542
S224017CA0517327F8277B27742774375D375500009502FA0172BAB03027715256FA0176563E
S224017CC037B5000634013735000F37B501643403275C3D0137AD3705277B37DCFA017178FA
S224017CE03F0627F6B702C50117FA5173CC023F0627F7200034053FEC274F37B500108A0017
S224017D00C517B710850034013735000F37B533EAFA0176023F02B07285003401275C3D0329
S224017D2037AD3705277B37DCFA0172463F0227F6B758275C3D0337AD3705277B37DCFA02B4
S224017D40E4B68800B41A3735000137B57CF23403275C3D0337AD3705277B37DCFA02E08635
S224017D603F04B0CA8500275C37DD1503275C3D03340837AD34013735000F37B533EAFA0274
S224017D80E0D03F04F50117FA517217FA33E437B5FFFF37FA5782CC143F1827F7340D274FF8
S224017DA03716B71EF50F37BD0054379D17F533FB3705277B27742774375D37550000950276
S224017DC0FA0172BAB03827715256FA01765637B5000834013735000F37B500543403275CE9
S224017DE03D0137AD3705277B37DCFA0171783F0627F6B704C50117FA33FBB002F50717FAA5
S224017E0033FBCC023F0627F7340D274F3716B70637F5004AFA0174BEB02A37B5005037BD8F
S224017E2000013409275C37AD3705277B37DCFA01701C3F0427F6B70C850037FA004AF50106
S224017E4017FA517217FA33E4CC023F0627F73FE66666C0800000430C000034053FF8274F89
S224017E603716B72637B50020FA02E7DA8A02374A0000F501379E2771004E37BE7E4EFA028E
S224017E80E6BA276CFA02E620FA0175C8B06EF50127FA27717E5637DC37AC27FA37DC34036D
S224017EA0F50127FA27717E5237DC37AC27FA37DC3403275C3D0437AD3705277B37DCFA0148
S224017EC0710E3F0827F6B73437B5FFE0FA02E7DA8A02374A0000374500048506276CFA029F
S224017EE0E62037ECF501379E37EC37BE7E4EFA02E9502773004EF50117FA517217FA33E495
S224017F00CC083F0C27F7340D274F3716B71EF50F37BD017C379D17F54F983705277B277490
S224017F202774375D375500009502FA0172BAB03627715256FA01765637B500023401373546
S224017F40000F37B5017C3403275C3D0137AD3705277B37DCFA0171783F0627F6B708C5010B
S224017F6017FA4F98F50117FA5172CC023F0627F7340D274F3716B71EF50F37BD0184379DDE
S224017F8017F500523705277B27742774375D375500009502FA0172BAB03627715256FA016A
S224017FA0765637B5000334013735000F37B501843403275C3D0137AD3705277B37DCFA0117
S224017FC071783F0627F6B708C50117FA0052F50117FA5172CC023F0627F7340D274F371669
S224017FE0B62837B5001E37BD00013409275C3D0137AD3705277B37DCFA016EAA3F0427F658
S224018000B708C501370537FA0048FA00E510CC023F0627F7340D274F3716B62837B50050E2
S22401802037BD00013409275C3D0137AD3705277B37DCFA016EAA3F0427F6B708C50137053E
S22401804037FA0048FA00EC72CC023F0627F7340D274F3716B62A37B5001E340127F53401A4
S224018060275C3D0137AD3705277B37DCFA016EAA3F0427F6B70AF50117FA533EC501370596
S224018080FA01B7CACC023F0627F72F2F2F2F20557365722050726F6772616D2025326920BA
S2240180A02F2F2F2F000034053FDC274F3716B67A37B5001E37BD00013409275C3D2337ADB4
S2240180C03705277B37DCFA016EAA3F0427F6B75AC523370534013735000137B5808A340332
S2240180E0275C3D0537AD3705277B37DCFA02B5CC3F06275C3D0537AD3705277B37DCFA0189
S2240181007268F50F37BD34E0379D373DFF1C370537AD8A008D02C52375E437242775370662
S224018120BAFE2770810237430000FA00DA5ECC243F2827F7252E2A73002F494425752F4D84
S2240181406973632F50726F676C6973742F46616374257520000034053FAA274F37BD021151
S2240181608D00C559378700B2F50F27FA37F55250277A37AC27FA277A37350212372627752C
S22401818037B14BB737330002340B3735000137B581343403275C3D2537AD3705277B37DC45
S2240181A0FA02B5CC3F0A17F551E6B75CF50F27FA37F55250277A37AC27FA277AFC013775BB
S2240181C0532A34033735000137B581393403275C3D0337AD3705277B37DCFA02B5CC3F083F
S2240181E0275C3D25340837AD34013DDE37AD3705277B37DCFA02E0863F04275C3D0337AD03
S2240182003705277B37DCFA0090DEB00C275C3D2537AD3705277B37DCFA0172BACC563F5AA7
S22401822027F7252E2A73002F494425752F4D6973632F50726F676C6973742F5573657225A3
S2240182407520000034053FAA274F37BD00E38D00C559378700B2F50F27FA37F55250277A65
S22401826037AC27FA277A373500E43726277537B134E13733000F340B3735000137B5822258
S2240182803403275C3D2537AD3705277B37DCFA02B5CC3F0A17F551E6B75CF50F27FA37F57A
S2240182A05250277A37AC27FA277AFC013775532A34033735000137B582273403275C3D0377
S2240182C037AD3705277B37DCFA02B5CC3F08275C3D25340837AD34013DDE37AD3705277BE8
S2240182E037DCFA02E0863F04275C3D0337AD3705277B37DCFA0090DEB00C275C3D2537AD3B
S2240183003705277B37DCFA0172BACC563F5A27F7000F524000018156000000003716B70EDB
S22401832037B50002340137B50001FA016AF23F02B02437B50032373500013403373500018C
S22401834037B58310FA016A9A3F04277AF50F27FA277A37FA525037AC27FA27F7000F524059
S22401836000018244000000003716B70E37B50002340137B50001FA016AF23F02B02437B5B6
S224018380001E3735000134033735000137B5835CFA016A9A3F04277AF50F27FA277A37FA03
S2240183A0525037AC27FA27F734053FFC274F3716B70817F5533F3705FA017312B04C275C24
S2240183C03D0337AD3705277B37DCFA0171DA27F6B738C50317FA533FF524CA0217F5533F42
S2240183E0B71AC50237058A0017F50026860037FA5326C502371017F6002617FA0026B00A85
S22401840017F55327C60217F7002617FA0026CC043F0827F745562044583338002573205698
S2240184202573000034053FAC274F3735000137B584148A02374A0000C557B7543735000073
S22401844037B54476340337450000850234033735000137B5841C3403275C3D0437AD3705EB
S224018460277B37DCFA02B5CC3F0C17F551E6B70E275C3D0437AD3705277B37DCFA0090DE70
S224018480B012275C3D0437AD3705277B37DCFA0172BAB000FA0172ACCC543F5827F70001B5
S2240184A084FB0001876000000000000184F60001881800000000000184F1000188BC000078
S2240184C00000000184EB0001895C00000000000184E6000189E0000000000000000000006B
S2240184E00000000000004741494E00534C4F5045005155414C004652455100545950450031
S2240185000001852A00018AD0000000000001852400018CAA00000000000000000000000069
S2240185200000000044454C4159004551257500000001854800018CAA000000000000000091
S224018540000000000000000044454C4159000001857700018B4400000000000185720001E0
S2240185608BE40000000000000000000000000000000046524551005459504500000185A7E9
S22401858000018C840001854E000185A000018C900001854E000000000000000000000000D9
S2240185A04C4F504153530048495041535300000185FF0001917400000000000185F9000110
S2240185C0926A00000000000185F2000191EE00000000000185EA0001930A00000000000093
S2240185E00000000000000000000052454C454153450041545441434B00524154494F0054E9
S2240186004852455348000001863200019382000000000001862A000193F4000000000000D2
S2240186200000000000000000000052454C454153450054485245534800000001868000015D
S22401864095D8000000000001867D000195F00000000000018679000196080000000000017D
S224018660867600019620000000000000000000000000000000004849004D4944004C4F003B
S224018680535542000001875B00018B0A0000000000018755000000000001857C0001874FBB
S2240186A000018D62000000000001874600018E16000000000001874000018EB80000000042
S2240186C0000187390001900A000000000001872E00000000000185AE0001872600000000A0
S2240186E0000186060001871E000194640000000000018719000194F4000000000001871482
S224018700000000000001863A0000000000000000000000004C454453004D55544500524F8E
S2240187205554494E47004C494D4954455200434F4D50524553534F52004C455652454C00BF
S2240187404C4556454C00504F4C41524954590044454C415900584F564552004551257500F4
S224018760340D274F3716B730F50F37BD0074379DF50F37BE57DC379E37F553303735000E9E
S224018780372637EDE50027F8277B27742774375D375500009502FA0172BAB06A277152563E
S2240187A0FA017656F507CA0037F5533037B8000ABCFE0100C500370534013735000F37B526
S2240187C000743403275C3D0137AD3705277B37DCFA0171783F0627F6B72CF50F37BD57DCFE
S2240187E0379D37F553303735000E3726277BC50127DA37F55330FA01EE0437F55330340130
S22401880037B50001FA012B5A3F02CC023F0627F741A00000469C400034053FFC274F371639
S224018820B71CF50F37BD57DE379D37F553303735000E372637DD375500009502FA0175C869
S224018840B06CF50127FA2771881437DC37AC27FA37DC3403F50127FA2771881037DC37AC0D
S22401886027FA37DC3403275C37AD3705277B37DCFA01710E3F0827F6B734F50F37BD57DC3B
S224018880379D37F553303735000E372637DD3745000085029A04375A000237F55330FA0186
S2240188A0EE0437F55330340137B50001FA012B5A3F02CC043F0827F73ECCCCCC34053FFCE3
S2240188C0274F3716B71CF50F37BD57E2379D37F553303735000E372637DD3755000095023A
S2240188E0FA0175C8B06CF50127FA2771881037DC37AC27FA37DC3403F50127FA277188B887
S22401890037DC37AC27FA37DC3403275C37AD3705277B37DCFA01710E3F0827F6B734F50FCB
S22401892037BD57DC379D37F553303735000E372637DD3745000085029A08375A000637F534
S2240189405330FA01EE0437F55330340137B50001FA012B5A3F02CC043F0827F7340D274F23
S2240189603716B71AF50F37BD57DD379D37F553303735000E3726277B27D527F8FA0173E240
S224018980B046275C3D0137AD3705277B37DCFA016E5AC501F806B700F80CB632F50F37BD23
S2240189A057DD379D37F553303735000E3726277BC50127DA37F55330FA01EE0437F553306F
S2240189C0340137B50001FA012B5A3F02CC023F0627F7FA0172ACB0F0C14000004140000042
S2240189E034053FFC274F3716B71CF50F37BD57E6379D37F553303735000E372637DD375538
S224018A0000009502FA0175C8B06CF50127FA277189DC37DC37AC27FA37DC3403F50127FAD9
S224018A20277189D837DC37AC27FA37DC3403275C37AD3705277B37DCFA01710E3F0827F6A0
S224018A40B734F50F37BD57DC379D37F553303735000E372637DD3745000085029A0C375A52
S224018A60000A37F55330FA01EE0437F55330340137B50001FA012B5A3F02CC043F0827F783
S224018A80000F5240000000000001849E3716B71017F5532C3705340137B50001FA016AF2B8
S224018AA03F02B02617F5532C37053735000134033735000137B58A80FA016A9A3F04277AE8
S224018AC0F50F27FA277A37FA525037AC27FA27F73405274FF50517FA532CC5033705FA019D
S224018AE08A8C37F55328373500053726277AF50F27FA277A37F15250277A37AC27FA277A6E
S224018B0037FA5330CC003F0427F73405274FF50417FA532CC5033705FA018A8C37F553287A
S224018B2027F427F4277AF50F27FA277A37F15250277A37AC27FA277AFC0A37FA5330CC00FC
S224018B403F0427F7340D274F3716B730F50F37BD00D8379DF50F37BE57AC379E37F5532EA1
S224018B6037350006372637EDE50027F8277B27742774375D375500009502FA0172BAB05A38
S224018B8027715256FA01765637B5001234013735000F37B500D83403275C3D0137AD37053E
S224018BA0277B37DCFA0171783F0627F6B72CF50F37BD57AC379D37F5532E37350006372686
S224018BC0277BC50127DA37F5532EFA01F1F837F5532E340137B50002FA012B5A3F02CC0236
S224018BE03F0627F734053FFC274F3716B71CF50F37BD57AE379D37F5532E373500063726B5
S224018C0037DD375500009502FA0175C8B06CF50127FA2771881437DC37AC27FA37DC340317
S224018C20F50127FA2771881037DC37AC27FA37DC3403275C37AD3705277B37DCFA01710EB4
S224018C403F0827F6B734F50F37BD57AC379D37F5532E37350006372637DD3745000085025D
S224018C609A04375A000237F5532EFA01F1F837F5532E340137B50002FA012B5A3F02CC04CB
S224018C803F0827F737F5532827F437FA532E27F737F5532827F4FC0137FA532E27F7447A8A
S224018CA000003FF54FDF4461000034053FFC274F3716B726F50F37BD5790379D37F5532839
S224018CC027F427F437DD37550000F501379E950237BE8C9EFA02E6BAFA0175E2B076F5012D
S224018CE027FA27718CA637DC37AC27FA37DC3403F50127FA27718CA237DC37AC27FA37DC1B
S224018D003403275C37AD3705277B37DCFA01710E3F0827F6B73EF50F37BD5790379D37F50C
S224018D20532827F427F437DD37450000F501379E850237BE8C9EFA02E9509A02375A000019
S224018D4037F55328FA01F8AA37F55328340137B50003FA012B5A3F02CC043F0827F7000008
S224018D60000034053FFC274F3716B726F50F37BD579C379D37F5532827F427F437DD37559D
S224018D800000F501379E950237BE8C9EFA02E6BAFA0175E2B076F50127FA27718CA637DC44
S224018DA037AC27FA37DC3403F50127FA27718D5E37DC37AC27FA37DC3403275C37AD3705C1
S224018DC0277B37DCFA01710E3F0827F6B73EF50F37BD579C379D37F5532827F427F437DD55
S224018DE037450000F501379E850237BE8C9EFA02E9509A02375A000037F55328FA01F8CABA
S224018E0037F55328340137B50004FA012B5A3F02CC043F0827F7340D274F3716B72AF50FA1
S224018E2037BD0138379DF50F37BE5955379E37F5532837EDE50027F8277B27742774375D74
S224018E40375500009502FA0172BAB05227715256FA01765637B5000234013735000F37B52F
S224018E6001383403275C3D0137AD3705277B37DCFA0171783F0627F6B724F50F37BD59551F
S224018E80379DC5013775532827DA37F55328FA02092A37F55328340137B50007FA012B5AE5
S224018EA03F02CC023F0627F7C31600004F4646004F46460040C0000034053FFC274F371674
S224018EC0B764F50127FA342037AC27FAF50F37BD595A379D3775532827742774375D375506
S224018EE000009502350237788EA8B60037F88EAA37DC37AC27FA37DCB60C3735000137B557
S224018F008EACFA0172BA378000ECF50F37BD595A379D3775532827742774375D375500004B
S224018F209502FA0175C8378000CC27715256FA0176563735000137B58EB0340327715256C4
S224018F40FA02E0AE3F04B63EF50F37BD595A379D37F5532827F427F437DDF50127FA27712B
S224018F608EA837EC37AC27FA37EC9A02375A000037F55328FA02092A37F55328340137B5A0
S224018F800007FA012B5A3F02B06AF50127FA27718EB437DC37AC27FA37DC3403F50127FA80
S224018FA027718EA837DC37AC27FA37DC3403275C37AD3705277B37DCFA01710E3F0827F646
S224018FC0B732F50F37BD595A379D37F5532827F427F437DD3745000085029A02375A000002
S224018FE037F55328FA02092A37F55328340137B50007FA012B5A3F02CC043F0827F74F463B
S2240190004600C2C8000042C8000034053FF8274F3716B764F50127FA342037AC27FAF50FAF
S22401902037BD595A379D3775532827742774375D375500009502350237788EA8B60037F89A
S2240190408EAA37DC37AC27FA37DCB60C3735000137B58FFEFA0172BA37800110F50F37BD19
S224019060595A379D3775532827742774375D375500009502FA0175C8378000F0F50127FA59
S2240190802771900637DC37AC27FA37DC3403F50127FA2771900237DC37AC27FA37DC340399
S2240190A0275C3D0437AD3705277B37DCFA01710E3F0827F6378700B4F50F37BD595A379D42
S2240190C037F5532827F427F437DD3755000095028A02374A0000374500048506276CFA02CF
S2240190E0E55637450000F501379E850237BE8EB4FA02E662BF14F50127FA27718EB437DC0F
S22401910037AC27FA37DC8A02374A0000B02637450000F501379E850237BE8EA8FA02E66212
S224019120BC12F50127FA27718EA837DC37AC27FA37DC8A02374A0000F50F37BD595A379DC0
S22401914037F5532827F427F437DD3745000085029A02375A000037F55328FA02092A37F5E6
S2240191605328340137B50007FA012B5A3F02CC083F0C27F7340D274F3716B71AF50F37BD7B
S2240191805186379D37F55328373500063726277B27D527F8FA0173A6B04A27F537BDFFE2EC
S2240191A03409275C3D0137AD3705277B37DCFA016E003F0427F6B72CF50F37BD5186379D87
S2240191C037F55328373500063726277BC50127DA37F55328FA0141AE37F55328340137B551
S2240191E00005FA012B5A3F02CC023F0627F7340D274F3716B71AF50F37BD5188379D37F5CC
S2240192005328373500063726277B27D53705FA0173E2B04C37B50064340127F53401275C7F
S2240192203D0137AD3705277B37DCFA016EAA3F0427F6B72CF50F37BD5188379D37F5532873
S224019240373500063726277BC50127DA37F55328FA0141AE37F55328340137B50005FA0177
S2240192602B5A3F02CC023F0627F7340D274F3716B730F50F37BD0140379DF50F37BE518629
S224019280379E37F5532837350006372637EDE5013705277B27742774375D375500009502A8
S2240192A0FA0172BAB05A27715256FA01765637B5000534013735000F37B501403403275CE8
S2240192C03D0137AD3705277B37DCFA0171783F0627F6B72CF50F37BD5187379D37F5532801
S2240192E0373500063726277BC50127DA37F55328FA0141AE37F55328340137B50005FA01D7
S2240193002B5A3F02CC023F0627F7340D274F3716B718F50F37BD518A379D37F553283735C3
S22401932000063726277B2795FA0174BEB04A37B503E7340127F53401275C37AD3705277B9E
S22401934037DCFA01701C3F0427F6B72CF50F37BD518A379D37F55328373500063726277B6B
S2240193608500279A37F55328FA0141AE37F55328340137B50005FA012B5A3F02CC023F066F
S22401938027F7340D274F3716B716F50F37BD5176379D377553282774277427D527F8FA01D2
S2240193A073A6B04627F537BDFFE23409275C3D0137AD3705277B37DCFA016E003F0427F60B
S2240193C0B728F50F37BD5176379DC501377553282774277427DA37F55328FA0148C437F517
S2240193E05328340137B50006FA012B5A3F02CC023F0627F7340D274F3716B714F50F37BD0C
S2240194005178379D37755328277427742795FA0174BEB04637B503E8340127F53401275C8D
S22401942037AD3705277B37DCFA01701C3F0427F6B728F50F37BD5178379D8500377553284A
S22401944027742774279A37F55328FA0148C437F55328340137B50006FA012B5A3F02CC0204
S2240194603F0627F7340D274F3716B72AF50F37BD0154379DF50F37BE578C379E37F5532825
S22401948037EDE50027F8277B27742774375D375500009502FA0172BAB05027715256FA01AD
S2240194A0765637B5000434013735000F37B501543403275C3D0137AD3705277B37DCFA0131
S2240194C071783F0627F6B722F50F37BD578C379DC5013775532827DA37F55328FA01F8CA61
S2240194E037F55328340127F5FA012B5A3F02CC023F0627F7340D274F3716B70C37F553280E
S224019500FC01FA020C4EFA0173A6B03637B50001340127F53401275C3D0137AD3705277B02
S22401952037DCFA016E003F0427F6B716C501B70837F55328FC01FA020BCEB00637F5532821
S224019540FC01FA020B7ECC023F0627F7340D274F3716B718F50F37BD516E379D37755328CD
S22401956027D5CA01C60BCA013705FA017312B05E275C3D0137AD3705277B37DCFA0171DADC
S22401958027F6B74AC501B710F50F37BD516E379D3775532827D5C70BCA01B014C50B3710F4
S2240195A0277AF50F37BD516E379D277A3775532827D6CA01C5013705340137F55328FA020F
S2240195C000CE3F0237F55328340127F5FA012B5A3F02CC023F0627F73405274F37B50001F0
S2240195E03401C5033705FA01954CCC003F0627F73405274F37B500023401C5033705FA0150
S224019600954CCC003F0627F73405274F37B500043401C5033705FA01954CCC003F0627F751
S2240196203405274F37B500083401C5033705FA01954CCC003F0627F7000196A8000197CC9A
S22401964000000000000196A100019760000000000001969D000197040000000000019697D6
S22401966000019B400000000000019691000197EC000000000001968C000198D800000000C8
S22401968000000000000000000000000053494E4500415544494F00535441525400564552A8
S2240196A0004F4E54494D45004F4E434F554E5400000196F900019C80000196F000019CC819
S2240196C0000196E800019C94000196E100019CA2000196D800019D1E4D494449544553548F
S2240196E000454550434C5200494E49544D454D00424F4F544C4F4144005245534554005669
S2240197002573200034053FB0274F3716B7303735000037B5447634033735000137B596FF82
S2240197203403275C37AD3705277B37DCFA02B5CC3F08275C37AD3705277B37DCFA0172BA51
S224019740B000FA0172ACCC503F5427F70000003C25326C7568203A20253032756D696E00D7
S22401976034053FDA274F3716B758F501379E2771318437BE974CFA02E9D48A00F501379EC1
S2240197802771318437BE974CFA02E9F08A04374A000285003401850434033735000137B5E5
S2240197A097503403275C3D0637AD3705277B37DCFA02B5CC3F0A275C3D0637AD3705277B9C
S2240197C037DCFA0172BACC263F2A27F73716B70637F531882775FA01751E27F7C3160000C0
S2240197E04F4646004F46460040C00000340D274F3716B73CF50127FA342037AC27FA2771AF
S22401980001903502377897DCB60037F897DE37DC37AC27FA37DCB60C3735000137B597E042
S224019820FA0172BA3780009027710190FA0175C83780008427715256FA01765637B5000124
S2240198408A00850037B80004BE06FA02058827030000B0EA3735000137B597E4340327714C
S2240198605256FA02E0AE3F04B612F50127FA277197DC37DC37AC27FA37DC27730190B03648
S224019880F50127FA277197E837DC37AC27FA37DC3403F50127FA277197DC37DC37AC27FAFA
S2240198A037DC34033735000F37B50190FA01710E3F0827710190FA02080ACC023F0627F737
S2240198C025752025342E31662025352E31660025752025662025660034053FDE274F371662
S2240198E0B7382771533634032771533217FD533A340B3735000137B598C03403275C37ADCF
S2240199003705277B37DCFA02B5CC3F0E275C37AD3705277B37DCFA0172BA378000EAF50170
S22401992027FA277197DC37DC37AC27FA37DC277353362735533A27715256FA01765637F58C
S22401994052568A1E37F552588A20277527F5340337B10128FA0077FC3F04277527F5340392
S22401996037B101CCFA0077FC3F04277527F5340337B10153FA0077FC3F04277527F53403B2
S22401998037B101F7FA0077FC3F043735000F37B55336340337B55332340337B5533A3403B2
S2240199A03735000137B598CF34033745001E8520FA02B7343F10F501379E2771533637BE54
S2240199C097E8FA02E662BF10F50127FA277197E837DC37AC27FA37DC2773533637F5533ABB
S2240199E037B80001B51C37B80004B21627715336340327715332340317F5533B3705FA0168
S224019A009A243F08B000FA0172ACCC223F2627F74120000041A000003F0000004000000040
S224019A20473B800034053FF2274F3735007F37B5FFFFFA02E8B28A02374A00003745001A30
S224019A40F501379E851C37BE97E8FA02E64237ECF501379E37EC37BE9A14FA02E9503403DC
S224019A60F50127FA27719A1037DC37AC27FA37DCFA02B3563F04276CFA02E6BA37ECF501CD
